:020000040800F2
:1000000000000524E5A90008719D0008739D000803
:10001000759D0008779D0008799D0008000000008C
:1000200000000000000000000000000091420108F4
:100030007B9D000800000000314301089543010842
:1000400035AA000835AA000835AA000835AA000814
:1000500035AA000835AA000835AA000835AA000804
:1000600035AA000835AA000835AA00087D9D0008B9
:100070008D9D00089D9D0008AD9D0008BD9D000858
:1000800035AA000835AA000835AA0008CD9D000849
:10009000DD9D0008ED9D0008FD9D000835AA0008C3
:1000A00035AA000835AA000835AA000835AA0008B4
:1000B00035AA000835AA000835AA000835AA0008A4
:1000C00035AA000835AA000835AA00080D9E0008C8
:1000D00035AA000835AA000835AA00081D9E0008A8
:1000E00035AA000835AA00080000000035AA00085B
:1000F00035AA00082D9E000835AA000835AA000878
:1001000035AA000835AA000835AA000835AA000853
:1001100035AA00083D9E000835AA000835AA000847
:1001200035AA000835AA000835AA00084D9E000827
:100130005D9E000835AA000835AA00086D9E0008DB
:1001400000000000000000000000000000000000AF
:1001500035AA000835AA000835AA000835AA000803
:1001600035AA000835AA0008859E0008959E00085B
:1001700035AA0008A59E000835AA00080000000066
:1001800035AA000835AA000835AA000835AA0008D3
:1001900035AA000835AA000835AA000835AA0008C3
:1001A00035AA000835AA000835AA0008000000009A
:1001B00035AA000835AA000835AA000835AA0008A3
:1001C00035AA000835AA0008000000000000000061
:1001D000000000000000000035AA00080000000038
:1001E000000000000000000000000000000000000F
:1001F000000000000000000035AA000835AA000831
:1002000035AA000835AA00080000000035AA000839
:1002100035AA000835AA000835AA000835AA000842
:1002200035AA00080000000035AA00080000000000
:1002300035AA000835AA00080000000035AA000809
:1002400035AA000835AA000835AA000835AA000812
:1002500035AA000835AA000835AA000835AA000802
:1002600035AA000835AA000835AA000835AA0008F2
:1002700035AA000835AA000835AA000800000000C9
:1002800035AA000835AA000835AA000835AA0008D2
:100290000000000035AA000835AA00080000000090
:1002A0000000000035AA000835AA000835AA000899
:1002B000B59E000835AA000835AA0008C59E0008AA
:0C02C000D59E000835AA000835AA0008E9
:1003000010B5054C237833B9044B13B10448AFF34F
:1003100000800123237010BDF80D002400000000B0
:10032000781C020808B5034B1BB103490348AFF31F
:10033000008008BD00000000FC0D0024781C0208AD
:10034000F0B44C1E4F2C41D8DFE804F028282828B0
:10035000404040403E3E283E3E3E3E3E3E3E3E3ECB
:100360003E3E3E402A2A2A2A2A2A2A2A283E3E3E61
:100370003E3E403E2A292840282A2A3E2940403E27
:100380003E3E28282828283E28283E2840403E3E39
:100390003E4040403E3E3E282A282A2AB2B1ABB118
:1003A000D0E90545AC4211DA0669270106EB0415D0
:1003B0004FF0000C0134C5F804C04461F1552846E3
:1003C000C5E90223F0BC7047002AE9D10025284680
:1003D000F0BC704710B4C3681C78522C0A460FD08A
:1003E0004F2C03D008465DF8044B7047C16A0331B7
:1003F000C16220210133C3605DF8044B00239FE7F5
:10040000C16A0231C1621F21F4E700BF002963D035
:1004100038B505460C462378013B4F2B37D8DFE82B
:1004200003F03131315036363B3B313131313131EE
:1004300031313131313131313136313131313131A7
:1004400031313131282831313631313131373131A3
:10045000313131363B31313131313131313131317D
:100460003131363631373737373631313131313155
:100470003131A3681B78052B04D1D5F8383101330D
:10048000C5F83831D5F81C31B3F5006F08DD38BD3B
:10049000A468002CBFD138BDE468002CBBD1FAE7BA
:1004A0000133C5F81C31A1682846FFF7AFFFE168AA
:1004B0002846FFF7ABFFD5F81C31013BC5F81C31CE
:1004C00038BDD5F844310133C5F84431D5F81C3175
:1004D000B3F5006FDBDCE3E7704700BF7AB32DE9CB
:1004E000F0410A440D460446D0F80011571E013D64
:1004F0004FF0000809E00B46BD4201F10101C4F8CC
:100500000011E65484F8046117D0FF2915F8016F33
:10051000F1D1D4E9423284F8FF8020469847D4F8DC
:1005200028310133C4F8283100230121BD42C4F829
:100530000011E65484F80461E7D1BDE8F08170470A
:100540002DE9F041026815786E2D07462CD0A5F1F3
:100550003003092B33D84FF0000EDFF868C00020BD
:100560006FF0004802E0B0EBD10F19DC01323A60C5
:100570001478A4F1300300EB8000A8EB0301DBB298
:1005800005EB4006092BACFB01012546A6F1300026
:10059000E9D9BEF1000F01D0C6F13000BDE8F0810D
:1005A0004FF0FF30BDE8F081531C03605578A5F192
:1005B0003002092A03D81A464FF0010ECDE7002079
:1005C000ECE700BFCDCCCCCC38B5D0E905329342B6
:1005D0000FDA026902EB031419010025656001338B
:1005E0004225436155540C30FFF7AAFFA060204616
:1005F00038BD0024204638BD10B5C3681A785F2A7C
:1006000004460DD06E2A0DD00C30FFF799FF013053
:1006100008D4E3681A785F2A04D10133E36010BD7F
:100620000020FAE74FF0FF3010BD00BFC3681A7812
:10063000542A19D1013370B5C3600446FFF7DCFFBB
:10064000021E0FDBD4E905318B420BDA216901EB85
:1006500003101D01002646600133052663614E55D7
:10066000826070BD002070BD0020704770B50446E8
:100670000C30FFF765FF051E3EDDE66863689B1BD7
:100680009D4237DCA26873195207E36004D5725D9E
:10069000242A04BF0133E360092D12DCD4E90532BA
:1006A000934227DA206900EB0310002201334260F5
:1006B0006361FEB1C0E90265002343600370A0627C
:1006C00070BD1B49082230461BF054FE30B9337A06
:1006D0002E2B13D05F2B11D0242B0FD0D4E9053251
:1006E0009A4207DD206900EB0310002201334260CB
:1006F0006361DFE70020E2E7002070BD737A4E2BD4
:10070000ECD1E26AD4E905311632551B8B42E56221
:10071000F0DA2269074D02EB0310591C1B016161DD
:1007200000214160D1541523C0E90253C7E700BF3F
:10073000643B0208703B020830B5C368856A044612
:100740001878422883B00A4610D10133E36020466E
:100750000192FFF78BFF019A03464C212046FFF7D9
:10076000EFFDE368197842290246EED01046A562F3
:1007700003B030BD2DE9F843C3681A78532A30D14D
:100780005A1CC2605A78044692B39A1CC2605A78C6
:100790005F2A42D0A2F13000C3B2092B24D8002135
:1007A0000DE0303B99421CD8E1680A78481C1AB128
:1007B000E0600A785F2A39D0A2F130001946C0B251
:1007C00001EBC1030928A2F1410502EB8303E8D93B
:1007D000192D06D801EBC10302EB8303373B994285
:1007E000E2D90020BDE8F883A2F14103192BD6D944
:1007F000A36803F00803002B14BF0125002500D1D6
:10080000B1B9354B742103F1A80001E013F81C1FA6
:10081000914214D08342F9D1E3E70023226A9A423D
:10082000DFD9E26952F82300BDE8F8830133F5E728
:10083000E3681B78433B012B98BF0D46E1E75E69F7
:10084000002E42D0D4E905208242D3F818C041DA04
:1008500027694FEA021E07EB02114FF0000901322F
:100860004FF01808C1F80490626107F80E80C1E9E2
:10087000026CA16235B3D3E90351E36A82420B44AF
:10088000E36225DA236903EB0210160100274760B3
:100890000132182762619F55C0E90251E3681B7855
:1008A000422B9FD101462046FFF746FF002898D0F3
:1008B000D4E90832934294DAE1695A1C41F82300E2
:1008C00022628FE7D3E90151D7E7D4E90520D1E7C8
:1008D0000020E3E70021CCE7681D020838B5044694
:1008E00029B9C3681A787AB15A1CC2601978682984
:1008F00019D0762908D104F10C052846FFF720FE0F
:10090000E3681A785F2A01D0002038BD0133E36024
:100910002846FFF715FEE3681A785F2AF4D1013301
:10092000E360012038BD04F10C00FFF709FEF2E797
:10093000C3681A785F2A01D00120704710B55A1C8D
:10094000C2605A785F2A044605D00C30FFF7F8FDE4
:10095000C043C00F10BD023340F80C3FFFF7F0FD5D
:10096000002809DB092805DDE3681A785F2A03D12E
:100970000133E360012010BD002010BD28B909E05B
:10098000002908DDC068013940B103782F2BF7D06A
:10099000002070477047FBD180687047704700BFE8
:1009A0000346D0F8100130B1096843680029D868BF
:1009B00000DBE3E770470122C3F81821704700BF4E
:1009C000002943D038B505460C4623784C2B33D844
:1009D000DFE803F030323232322730383832323208
:1009E00032323232323232323232323230323232E9
:1009F00032323232323232323232323032323232D9
:100A000030323232323230383232323232323232C4
:100A100032323232323030323232303030323230C2
:100A2000300004F108012846FFF7BAFF10B103783F
:100A30002F2B00D0002038BDA1682846FFF7C0FF4B
:100A40000028F8D1E468002CBFD1F3E700207047FC
:100A5000F0B514465268A5684B1C1344AB4283B0F2
:100A60000E46074611D8E5686DB9D4E9000339464A
:100A70001844324608F0BCF8D4E9003233449D549F
:100A800061683144616003B0F0BDE268002AFAD1C8
:100A900055B16D00AB42FCD8206829461BF09CFD87
:100AA00038B12060A560DEE7022B4FF00205F0D8D8
:100AB000F2E7019020681BF09BF9019B0122C4E939
:100AC0000033C4E90232DEE72DE9F04FC268157841
:100AD00085B000238D420446039300F028820F4620
:100AE000994603AE4FF00108D4F830A0C4F8308026
:100AF00013784C2B7FD0542B00F09C80732B4DD05F
:100B0000662B24D15378702B00F09980204601F099
:100B1000DBFC0546002800F087800378322B00F0CC
:100B2000B280342B00F060810AD8332B08D183685F
:100B3000032B05D8DFE813F031015D010400040048
:100B4000C4F830A00025284605B0BDE8F08FA3F119
:100B50003001092935D8204601F08AFE05460028D3
:100B600062D0E3681A78492A00F0A180C4F830A066
:100B70002A4600232E212046FFF7E2FB30600028A2
:100B800041D0E2681378BB4200F10C06ACD1039D62
:100B900001322846E26005B0BDE8F08F5378722B31
:100BA00000F0E580702BB1D10232E260204600F007
:100BB0000BFA002302464B212046FFF7C1FB0546F6
:100BC0001DE06F2B24D0692B7ED153786C2B9DD1E7
:100BD0000232E26000255078002800F0968145211D
:100BE0002046FFF771FF2A46034631212046FFF7D2
:100BF000A7FB054603E0204601F088FF0546C4F840
:100C000030A0002DB4D10025284605B0BDE8F08FF6
:100C100053786E2B7FF47AAF0232E260204601F007
:100C200027FE054600289CD12846C4F830A005B010
:100C3000BDE8F08F2046FFF7F9FC0546DFE7931C7F
:100C4000E3609378542B5FD02046FFF7D5FC6FF01C
:100C5000004398423FF474AF431C3FF471AF01303E
:100C6000D4E905329342BFF66BAF2269190102EB5A
:100C700003154FF0060C0133C5F80490636102F8C8
:100C800001C0A86072E78068E26A8168036802397F
:100C90000A44E2621A78732A25D0D0F80CB0BBF16E
:100CA000030F3FF64DAFDFE80BF0783380AF013331
:100CB000E360204600F0A8FB2A46034604212046B4
:100CC000FFF73EFB05469AE7742B7FF41FAF53787E
:100CD0006C2B7FF41BAF0232E260204600F0FCFF79
:100CE000E268054677E759787429D6D199780029C2
:100CF000D3D1204600F0F0FF03462A463721204694
:100D0000FFF71EFB05467AE70332E2600020A7E703
:100D10001978702920D06D291ED04FF0000B732A4E
:100D200012D15A78502A0FD19B786BB9204600F027
:100D30006BFB0346BBF1000FDFD01A46392120467A
:100D4000FFF7FEFA0346D8E7204600F03DF90346D8
:100D5000BBF1000FF1D1D0E758788842DDD1E168CE
:100D600008785F28DBD10131E1601A78D5E70232DB
:100D7000E260204600F0B0FF0546204601F078FD15
:100D8000E3681978492900F0C48003462A46012106
:100D90002046FFF7D5FA054631E72A4600233621DB
:100DA0002046FFF7CDFA054629E7AA681268517870
:100DB000632900F0CD801A78662A00F0D980204699
:100DC000019300F001F9019B83461A78632A72D1DE
:100DD00059786C296FD1997800296CD1452120462A
:100DE000FFF772FE024675E0E3681A785F2A00F0AA
:100DF000A780204600F0E8F82A460346372120461F
:100E0000FFF79EFA0546FAE6712A17D15A78752A35
:100E100014D19A7892B9204600F0D6F8834620463D
:100E200000F0D2F802462046019200F0CDF8019A77
:100E3000034670BBC4F830A0054684E61A78662ADB
:100E400000F09D806E2A7FF47BAE5B78772B02D01A
:100E5000612B7FF475AE5F212046FFF735FE834698
:100E6000204600F039FFE36819784529024600F072
:100E7000A680702900F0958069297FF461AE5B78C7
:100E80006C2B7FF45DAE0190204600F09DF8019A36
:100E900003463C212046FFF753FA5A4603463B21BE
:100EA0002046FFF74DFA2A4603463A212046FFF72F
:100EB00047FA0546A3E6642A1AD15978742917D14E
:100EC0009978A9B9204601F0D3FCE368197849293B
:100ED000024658D0134639215A462046FFF730FAC9
:100EE0002A46034638212046FFF72AFA054686E6B9
:100EF000702A05D15A78742A02D19B78002BE1D050
:100F0000204600F061F80246E4E7C4F830A0054648
:100F100019E601330190E360204600F075FA019A6A
:100F2000034604212046FFF70BFA03462EE7013261
:100F3000C2602E211A4605B0BDE8F04FFFF700BA97
:100F40000133E36045212046FFF7BEFD0346D4E6AA
:100F50001278A2F16301012903D9723A012A3FF6FE
:100F60002AAF2046019300F0B7FE019B83462CE791
:100F70002046019301F0A8FA019B834625E720460D
:100F800001F0A2FA4AE701330190E360204600F045
:100F90003BFA019A034604212046FFF7D1F90246A5
:100FA00098E7597869297FF4CBAD02330190E3606B
:100FB00045212046FFF788FD019A034669E7013382
:100FC000E360002365E700BFC26813784C2B00F094
:100FD0008B80542B00F08A80F0B5732B83B00446CD
:100FE00052D0662B30D0A3F1300109290CD820460D
:100FF00001F03EFC0546002872D0E3681A78492AC1
:1010000076D0284603B0F0BD6F2B4BD0692B7DD135
:1010100053786C2B00F09780204601F055FA054676
:1010200000285DD00378322B42D0342B00F07F8132
:1010300056D8332B54D18368032B51D8DFE813F0F3
:10104000C700F300500050005378702BE4D1931C7C
:10105000C3609378542B00F01181FFF7CDFAC3439E
:1010600033F000433CD00130D4E90532934237DA03
:10107000226902EB0315190100266E600133062672
:1010800063615654A860BCE75378722B4AD0702B2A
:10109000C2D10232C260FFF797FF002302464B2104
:1010A00020462EE053786E2BB6D10232C2609EE706
:1010B0008168E36A8A680E68023A1344E36233780F
:1010C000732B4FD17278742A4CD1B278002A49D14F
:1010D000204600F001FE2A4603463721204610E054
:1010E0000025284603B0F0BD01F010BDFFF79EBA01
:1010F0000133E360204600F087F92A4603460421C5
:10110000204603B0BDE8F040FFF71AB9742B83D135
:1011100053786C2B80D10232E26000F0DDFDE26892
:10112000054613E00232C26000F0D6FD05462046B7
:1011300001F09EFBE368197849291AD003462A4634
:1011400020460121DDE70232E26000255378002BC2
:10115000C6D045212046FFF7B7FC2A460346312179
:101160002046CEE7CF68032FBAD8DFE807F0301368
:10117000356101330190E360204600F045F9019AA2
:10118000034604212046FFF7DBF82A4603460121E7
:101190002046B6E73278702A79D06D2A77D00027BA
:1011A000732B6FD17378502B6CD1B378002B69D12E
:1011B000204600F029F903462FB11A46392120466E
:1011C000FFF7BEF803462A462046372199E72A460C
:1011D00020460023362194E7AB681B685A78632ABF
:1011E00000F0B9803378662B00F0C3802046FFF70B
:1011F000EBFE07463378632B7BD172786C2A78D16B
:10120000B278002A75D145212046FFF75DFC0246E1
:10121000134639213A462046FFF792F82A460346FC
:10122000382120466DE72046FFF7CEFE0346CAE789
:10123000712B37D17378752B34D1B37893BB20469B
:10124000FFF7C2FE06462046FFF7BEFE07462046D1
:10125000FFF7BAFE034600283FF442AF3A463C216E
:101260002046FFF76DF8324603463B212046FFF744
:1012700067F82A4603463A21204642E70332C26015
:101280000020F1E62046FFF79FFE034694E77178C1
:10129000914284D1E26811785F2981D10132E26004
:1012A00033787CE73378662B6FD06E2B7FF418AFE2
:1012B0007378772B02D0612B7FF412AF5F21204629
:1012C000FFF702FC0646204600F006FDE3681978A9
:1012D0004529074669D070295BD069297FF400AFA2
:1012E0005B786C2B7FF4FCAE2046FFF76DFE034667
:1012F000B4E7642B28D17278742A25D1B2781ABB4E
:10130000204601F0B5FAE3681978492902467FF4CE
:101310007FAF01330190E360204600F075F8019A39
:10132000034604212046FFF70BF8024670E7E36806
:101330001A785F2A7FF477AF0133E36045212046B6
:10134000FFF7C2FB03463EE7702B17D02046FFF79E
:101350003BFE02465CE71B78A3F16302012A03D936
:10136000723B012B3FF63EAF204600F0B5FC07462E
:1013700040E7204601F0A8F807463BE77378742B56
:10138000E4D1B378002BBBD0E0E7204601F09CF815
:1013900058E75A78692A7FF4A3AE0233E360452107
:1013A0002046FFF791FB034658E70133E360002333
:1013B00054E700BF38B5C26813784C2B1DD00446E3
:1013C00005D8493B012B13D8BDE838404EE0582BD7
:1013D0000ED101320123056BC2600363FFF7F4FDF8
:1013E000E36825631A78452A0BD10133E36038BDE1
:1013F0002046BDE8384000F06FBCBDE8384001F041
:1014000085BB002038BD00BF70B5C368866A1A78F6
:10141000452A82B004461FD00023019301AD09E0A4
:10142000FEF78EFF286000F10C0560B1E3681A78C2
:10143000452A0BD02046FFF7BDFF024600232F218F
:101440002046002AECD1002002B070BD0198A662AF
:101450000133E36002B070BD5A1C0023C2602F212B
:101460001A4602B0BDE87040FEF76ABFC1680A784C
:10147000493A012A02D80131C160C5E7002070470E
:101480002DE9F043C2681378472B83B0044601D09E
:10149000542B34D1E16A01F11403E3621378542B25
:1014A0005DD0472B40F0A680531CE3605378002B9F
:1014B00000F0A080931CE3605378562B00F2B680B6
:1014C000402B40F29780413B152B00F29380DFE8E0
:1014D00013F017019100910091009100910091008B
:1014E0009100910091009100910091009100910074
:1014F00091009100240191003001910041010E46BC
:1015000000F020FA0546002874D0002E77D0A3689A
:10151000DB0774D42B784D2BA3F11C01A3F14F02F0
:1015200000F0D68000F2D280042940F2D180022B54
:1015300061D1EA6813784D2BA3F11C00A3F14F0190
:1015400003D000F2AF81042855D89268EA6013787E
:101550004D2BA3F11C00A3F14F01F2D1F5E7531C71
:10156000E3605378002B45D0931CE3605378413BF4
:10157000352B3FD8DFE813F033013E0016013E0063
:101580003E000E013E0006018E0186013E003E0037
:101590003E003E003E003E003E003E007E017401E3
:1015A0003E006A0162013E003E003E003E003E00F9
:1015B0003E003E003E003E003E003E004B013E002D
:1015C0003E003E003E003B013E003E003E003E002D
:1015D0003E003E003E003E003E003E003E003E001B
:1015E0003E00F600D4E905039842C0F27281E36838
:1015F0000B44E3600025284603B0BDE8F083E368B0
:101600001B78002BF7D0452BF5D029460B78042BFF
:1016100000F0738154D94D2BA3F14F0202D059D958
:10162000012A5AD889680029F0D157E0722BE1D1FC
:1016300004F10C00FEF784FF0128DBDDE3681A7873
:10164000002AD7D05F1CE7601B785F2BD2D1002225
:10165000451E90464FF041093B78002BCAD0242B01
:1016600040F024817B78532B00F05E815F2B00F0EB
:101670005981242BBED11946D4E90503984280F242
:1016800055812669070106EB00130130C3F8048079
:10169000606106F80790E76899600237023DE760ED
:1016A000002A00F0288140212046FEF749FE02462C
:1016B00000289FD0002DCFDC204600233F2127E0CB
:1016C000022B0AD1C9680029A0D107E0012A92D8CB
:1016D000AD681FE71C3B042BA4D90021204601F074
:1016E0006DF8002886D036B92B78022B03D1037809
:1016F000292B08BF866003462A462046032107E0BF
:1017000000212046FFF7BCFE002302461721204699
:1017100003B0BDE8F043FEF713BE204600F012F917
:1017200001902046FEF750FF019A034616212046FD
:10173000EEE79378002120462BB1D31CE360937829
:101740006E2B00F0F880FFF79BFE00230246492134
:101750002046DDE7204600F0F5F80023024613217D
:101760002046D5E776212046FFF7B8F800283FF459
:1017700041AF00212046FFF783FE002302461021DF
:101780002046C5E7204600F0DDF80023024614217C
:101790002046BDE7204600F09FFA002302460E21B6
:1017A0002046B5E7204600F097FA054604F10C0004
:1017B000FEF7C6FE0028FFF61DAFE3681A785F2A21
:1017C0007FF418AF0133E360204600F085FAE36A46
:1017D000591D0246E1622B4620460B2198E7204620
:1017E000FFF7E8FD002302463021204690E76821FC
:1017F0002046FFF773F800283FF4FCAE0021204696
:10180000FFF73EFE002302460F21204680E700211D
:101810002046FFF763F800283FF4ECAE0021204695
:10182000FFF75CF800283FF4E5AE00212046FFF703
:1018300027FE002302461121204669E7204600F0DA
:1018400081F8002302461521204661E70F31E1624D
:10185000204600F041FA002302460921204657E7BE
:101860000A31E162204600F037FA002302460A21DD
:1018700020464DE7204600F02FFA002302460D21B6
:10188000204645E7204600F027FA002302461221B1
:1018900020463DE7204600F01FFA002302460C21B7
:1018A000204635E701293FF6A6AE4EE63E4600212A
:1018B00007E016F8013F002B3FF494AE242B3FF4D1
:1018C00091AE0131A942F4DBD4E9050383427FF7ED
:1018D0008EAE236903EB00130130C3F8048060610E
:1018E00083F80080E0689F604718C3F80480D960DF
:1018F0006D1AE760D4E61A46DCE68B6863B11978A6
:10190000082901F1FF3209D806293FF6E6AE012A7F
:1019100002D8DB68002BF2D10121DFE6353918BF90
:101920000121DBE62E21A7E62F21A5E6E36802339D
:10193000E36000255FE6FFF7A3FD002302464A218E
:101940002046E5E62DE9F047C26813784E3B84B0A7
:1019500004460C2B08D8DFE803F028070707071315
:10196000072107070707760000F082FFE3681B786E
:10197000492B054600F0A980284604B0BDE8F08751
:101980005378742B00F0AB800021FEF7F3FEE36880
:101990001B78492B0546EFD12046F0E000F068FFA8
:1019A0000546284604B0BDE8F0870132C26003A9AD
:1019B000012200F043FE0746002800F08B80002142
:1019C0002046FEF707FDE1680E7880462EB3DFF86B
:1019D00004934FF0000A442E6AD0A6F13003DBB224
:1019E0001C2B40F2FD80A6F16103192B00F2FA8056
:1019F000204600F03DFF0546BAF1000F06D0012158
:101A00002B4652462046FEF79BFC0546532E08D136
:101A1000E168AA460E78002EDDD100253D60ABE7D7
:101A20000546E1680E78452E00F08C80002DF4D03C
:101A3000D4E908329342F0DAE269581C42F82350A4
:101A4000AA462062E6E70132C2600021FFF718FDD6
:101A5000054600283ED0E368197845293AD15A1C3A
:101A6000E2605978732900F0F680642900F09180D3
:101A70002046FFF767FF034650B10278462A07D099
:101A8000482A05D001902046FEF752FF019B08B37B
:101A90002A78032A05D1EA681178292904BF002190
:101AA00091602A4620460221FEF74AFC054663E77C
:101AB0004B7803F0DF03542B204652D000F0D8FEC1
:101AC0000546BAF1000F9AD1ABE718B1D4E9083254
:101AD00093424EDB0025284604B0BDE8F087D0E9EC
:101AE000053102328B42C26080F2B38002697748CE
:101AF00002EB0315591C1B01616100216960D1547F
:101B00000323C5E90203204600F0B2FE2A4603463D
:101B100001212046FEF714FCE36AE2680333E36226
:101B20001378492B05467FF427AF0028D2D0D4E99B
:101B300008329342CEDAE1695A1C41F8230022624E
:101B400020461CE0152329FA03F3DB075AD520466B
:101B500000F08EFE002D3FF463AFAA46012105463A
:101B60004EE700F0B9F80546BAF1000F7FF447AF31
:101B700057E7E1695A1C41F8230020462262FFF72B
:101B800075FC2A46034604212046FEF7D9FB05468C
:101B9000F2E60233E3602046FEF72EFD071E99DBD6
:101BA0002046FFF7CFFE064628B10378462B02D029
:101BB000482B40F08480D4E905239A4265DA2169F4
:101BC00001EB021310014FF0000CC3F804C0013206
:101BD0004FF0470C626101F800C0C3E9026757E7A4
:101BE0005546B0E7552E32D0532E66D101212046FE
:101BF000FEF7C0FD0546BAF1000F7FF400AFE168C3
:101C0000AA4607E7492E42D0542E4CD0452E09D083
:101C10004D2E7FF402AF002D3FF4FFAE0131E160A5
:101C2000AA46F7E63D60002D3FF454AFB8F1000F2F
:101C300004D0039BC8F80830CDF80C80E3681A780C
:101C4000452A7FF447AF0133039DE36094E6554690
:101C50007DE7002557E70233E3602046FEF768FE84
:101C600000283FF437AFD4E905239A420DDA216901
:101C7000174E01EB0213501C1201606100205860E6
:101C800088540E22C3E9026202E7002300E7002D18
:101C90003FF4C3AE0131E1602046FFF7B5FBAA4631
:101CA00004210546ACE62046FEF7C0FCAA460546E0
:101CB000BAF1000F7FF4A3AEB3E65546A4E7204681
:101CC000FEF736FE00287FF476AF03E7983B020864
:101CD000883B0208FF0308102DE9F041C1680B782A
:101CE000722B82B0044658D0562B56D04B2B54D072
:101CF000442B00F09E80A3F130024A2A00F290802B
:101D0000DFE812F02D012D012D012D012D012D01F6
:101D10002D012D012D012D018E008E008E008E00D3
:101D20008E008E008E0001028E0044018E008E0017
:101D3000600166018E008E008E008E008E004102D2
:101D40002D01740182018E0090019E01C201E90102
:101D50008E008E008E008E002D018E008E008E0073
:101D60008E008E008E001001100110011001100174
:101D7000100110011001100110018E00100110015E
:101D8000100110018E008E008E0010011001520112
:101D900010011001100110011001002201A92046BC
:101DA00000F04CFC054600283AD0E3681B78462B2F
:101DB00020463AD0FFF790FF2860002830D0037803
:101DC0001F3B012B05D8019A836882602A68019223
:101DD0002B60019D25B3D4E90832934220DAE169F2
:101DE0005A1C284641F82350226202B0BDE8F08117
:101DF0000123056B0363FFF7E7F825630246002321
:101E000043212046FEF79CFA0546019040B1E36865
:101E10001A782AB15A1CE2601B78452B00F0A78083
:101E20000025284602B0BDE8F08100F0EBFC2860F8
:101E3000C3E74B7803F0DF024F2AAED0773B012B8C
:101E4000ABD94B1CC3604B78002BE9D08B1CC36013
:101E50004B78463B302BE3D801A252F823F000BF69
:101E6000B7210008211E0008211E0008211E0008BD
:101E7000211E0008211E0008211E0008211E000846
:101E8000211E0008211E0008211E0008211E000836
:101E9000211E0008211E0008F11D0008211E000857
:101EA000211E0008211E0008211E0008211E000816
:101EB000211E0008211E0008211E0008211E000806
:101EC000211E0008211E0008211E000853220008C0
:101ED000211E00082D220008F7220008CD2200084C
:101EE000A3220008211E000879220008D32300083D
:101EF000211E0008211E0008211E0008211E0008C6
:101F0000AB230008211E000895230008211E0008AD
:101F1000211E00086B230008F11D00084123000862
:101F200007230008D4E90525BF48613B03EB830381
:101F3000AA4200EB830380F2AB82206900EB02151A
:101F4000160100276F6001322727626187555868A4
:101F5000E26AAB6001310244E160E26261E720467F
:101F6000FFF7F0FC05460190002D3FF459AFD4E98E
:101F700008329342BFF654AFE16941F82350019D06
:101F80005A1C2846226202B0BDE8F0810131E160AE
:101F90002046FFF7A1FE0023024625212046FEF73A
:101FA000CFF905460190DFE70131E1602046FEF7F9
:101FB0005DFB0023024628212046FEF7C1F90546B5
:101FC0000190D1E7204600F01DFC05460190CBE7CB
:101FD0000131E1602046FFF77FFE00230246262103
:101FE0002046FEF7ADF905460190BDE70131E160FD
:101FF0002046FFF771FE0023024624212046FEF70B
:102000009FF905460190AFE70131E1602046FFF7F7
:1020100063FE0023024622212046FEF791F9054681
:102020000190A1E70131E1602046FFF755FE002352
:10203000024623212046FEF783F90546019093E7E7
:102040004B78A3F13002092A05D95F2B03D0413B1D
:10205000192B00F2E28100212046FEF78BFBE3689A
:1020600001901A78492A05467FF4DBAE0133E3601C
:102070002046FFF7C9F92A46034604212046FEF709
:102080005FF9054601906FE72046FEF7CFFAE66854
:1020900001903378492B05467FF466AF636B002BC4
:1020A00040F0C88100283FF4BBAED4E908218A4241
:1020B000BFF6B6AEE16941F8220001322262327801
:1020C000493A012A05D80136E6602046FFF79CF917
:1020D00003462A46D1E70131E1602046FEF7C6FA01
:1020E000E36801901A78492A054600F07B81204672
:1020F000FFF7F2FD019B024621212046FEF720F961
:102100000546019030E74D1CE5604B785F2B00F0F1
:102110006781303B092B00F272812B46194601334F
:10212000E3601A78303A092AF8D9D4E905208242C6
:10213000A3EB0507BFF674AED4F810C000200CEB7B
:10214000021602F1010E874270604FEA0212C4F8D3
:1021500014E07FF765AE70600CF80200C6E9025724
:102160004A785F2A7FF45CAE1D460135E560204663
:10217000FFF7B2FD324603462A212046FEF7E0F87B
:1021800005460190F0E60131E1602046FFF7A4FD2D
:10219000054600283FF444AE2046FFF79DFD034668
:1021A00000283FF43DAE2A462B212046FEF7C8F812
:1021B00005460190D8E6D0E90532934280F26C8161
:1021C000006900EB03121D010026566001332C2626
:1021D0006361019246558B78303BDBB2092B94BF8B
:1021E00001230023938103D804F10C00FEF7A8F922
:1021F0002046019DFFF770FD019BA8609B68002BA6
:102200003FF40EAE04F10C00FEF79AF9E268137881
:1022100013B1531CE3601378019DA3F17302534281
:102220005341EB81FDE500BF2C1E0208D0E90532C9
:102230009342BFF6F5AD0269994E02EB0315591CA6
:102240001B01416100210E206960D154C5E9026083
:10225000E7E5D0E905329342BFF6E2AD0269914E5F
:1022600002EB0315591C1B01416100210420696028
:10227000D154C5E90260D4E5D0E90532934280F239
:1022800007810269884902EB031500206860581C29
:102290001B0160612720D054E36AA9600433E36224
:1022A000BFE5D0E90532934280F2F28002697F49AE
:1022B00002EB031500206860581C1B016061272099
:1022C000D054E36AA9600933E362AAE5D0E9053294
:1022D000934280F2DD800269754902EB031500200C
:1022E0006860581C1B0160612720D054E36AA96014
:1022F0000A33E36295E5D0E90532934280F2C88063
:1023000002696C49D4E78B785F2B00F0B780FEF749
:102310005BF90546002D3FF483ADE3681A785F2A28
:102320007FF47EAD0133E3602046FFF7D5FC2A46FB
:1023300003462D212046FEF703F80546019013E6DB
:10234000D0E90532934280F2A38002695A4902EB38
:10235000031500206860581C1B0160612720D054C1
:10236000E36AA9600733E3625BE5D0E90532934293
:1023700080F28E800269514902EB031500206860EB
:10238000581C1B0160612720D054E36AA960083300
:10239000E36246E5FFF7A0FC002302464B212046FE
:1023A000FDF7CEFF05460190DEE5D0E90532934208
:1023B0006EDA0269424902EB031500206860581C7E
:1023C0001B0160612720D054E36AA9601133E362E6
:1023D00027E5D0E9053293425ADA02693949CBE759
:1023E0000026C2E60133E3602046FFF70DF82A46D7
:1023F000034604212046FDF7A3FF019077E6012361
:10240000256B23632046FEF7DFFD25630646002883
:102410003FF406ADE3681A78A3E62046FFF792FA88
:102420000546019000283FF4FBAC0378182B7FF49D
:102430009EADF6E4731CE3602046D4F81480276A4E
:10244000E56AFEF7E1FFE3681A78492A034606D0F9
:10245000E562E660019DC4F81480276284E5019A74
:10246000002A3FF4DDACD4E908108142BFF6D8ACB5
:10247000E569481C45F821202062FEE5033101236F
:10248000056BC1600363FEF79FFD2563054641E7C9
:10249000002301939B68FFDE00231B70FFDE00BF5B
:1024A000A43B02089C3B020870200208342002086A
:1024B0005C200208482002088420020898200208B4
:1024C000C0200208AC200208F8B5C3681F78064691
:1024D0005FBB4FF0000E394D432100228B1A03EBF6
:1024E000D37302EB6303180105EB031C2C5820780F
:1024F000B84206D094BF5A1C19468A42EED1002039
:10250000F8BD60787045F5D1D6E905329342F6DA28
:10251000326902EB031019010024446001333224B4
:1025200073615454C0F808C0F8BD5A1CC26093F8D7
:1025300001E01F78BEF1000F02D1762FCBD0C8E7A3
:102540009A1CC260762F93F801E01BD1AEF13004E3
:10255000E3B2092BBFD8FEF789F8D6E905318B42E3
:102560000246CCDA316901EB03105F1C002545609F
:102570001B017761002AC2D033264560CE54C0E9E2
:102580000242F8BD632FA6D1BEF1760FA3D1D0E9E8
:102590000C34B3FA83F35B094363FFF79DFB736B62
:1025A000024633B1002335213046FDF7C9FE74637E
:1025B000F8BD34213046FDF7C3FEF8E7D420020809
:1025C00030B5C26883B000230193137823B3044667
:1025D00001AD11E04F2B16D0FFF77EFB0246002322
:1025E0002E212046C2B1FDF7ABFE2860A0B1E26803
:1025F000137800F10C054BB1452B204606D02E2B4D
:1026000004D0522BE6D15378452BE5D1019818B16F
:10261000C36823B103B030BD002003B030BD826871
:1026200011782729F6D19268117C0929F2D15168D5
:10263000E26A521AE2628360ECE700BF2DE9F04FD4
:10264000D0F80CC0171E9CF8003083B004460D462D
:1026500015BF4FF01E0A4FF01B0A4FF01D094FF037
:102660001A0914BF4FF01C084FF019080E464FF01E
:10267000010B722B15D0562B13D04B2B11D0442BA2
:1026800006D00FB9462B5DD0304603B0BDE8F08FC1
:102690009CF8012002F0DF014F2902D0773A012A8D
:1026A000EFD80CF10102722BE26016D0562B2CD021
:1026B0004B2B24D09CF80130002B3ED00CF10203B0
:1026C000E3609CF80110782951D06F2923D1E36A87
:1026D0000933E3624F21002304E0E36A0933E36234
:1026E0004146002300222046FDF72AFE306020B339
:1026F000D4F80CC000F108069CF80030B9E7E36A92
:102700000633E36251460023ECE7E36A0933E362F0
:1027100049460023E6E74F293CD1D4E90B3209337F
:10272000E362C4F830B0204601910092FEF74CFC01
:10273000009A01992263034628BB0026304603B065
:10274000BDE8F08FAE429FD01D241E201C2105E065
:10275000192A15D003F10805AE4295D02B681A78D6
:102760001A2A0AD01B2AF3D118702B68F2E7E36A01
:102770001133E3624D210023B4E71C702B68E9E7B5
:1027800019702B68E6E7E26810784528D5D1013248
:10279000E260A7E77729D0D1E36A0633E3622046F7
:1027A000FFF70EFF03460028C7D0E26811784529DD
:1027B000C3D10132E260502194E700BF70B5C36815
:1027C0001A784A2A05461AD081B12846FFF784FABA
:1027D000044690B12846FFF7F3FE034668B122464F
:1027E00028462921BDE87040FDF7AABD28460C46C1
:1027F000FFF7E6FE03460028F1D1002070BD01334B
:10280000C360E2E710B50446806810F480200BD165
:10281000A26BB2F5006F06D8511CE368A16319786A
:10282000462907D0A26310BDE3681A78462A01D072
:10283000002010BD5A1CE2605A78592A04BF0233A6
:10284000E36001212046FFF7B9FF01462046FDF76E
:10285000C1FDE3681A78452A04BF0133E360A36829
:1028600018BF00205B03DED4A26B013ADAE700BF99
:10287000F8B5C2681378A3F13001092904464FD98D
:10288000A3F16101192914D86F2B04D153786E2B51
:1028900004BF0232C2602046FFF716FE054610B1A3
:1028A0000378322B49D0E368197842293FD0284673
:1028B000F8BDA3F1430101296CD94C2B5AD0552BFB
:1028C00063D153786C2B00F0D080742B5DD1531CF6
:1028D000C360517874295BD10232C260FDF78CFE6F
:1028E0000028C0F2EF80D4E90532934280F2EA80FA
:1028F00022691E0102EB031500210133482769609C
:1029000063619755D4E908329342A86080F2DA8077
:10291000E169E26841F82350013323621178C4E78A
:10292000FDF7A4FEE368197842290546BFD1294680
:102930002046BDE8F840FDF7FFBE8268E36A916873
:10294000126807330B44E36213786C2BABD15378D6
:10295000692BA8D19378002BA5D12046FDF786FEE0
:102960002A46034637212046FDF7EAFCE368054680
:1029700019789AE70132C260FDF778FE054620B16A
:102980002046FDF7D5FF00288DD100252846F8BD4B
:1029900000258AE7806A18B1017851B3182928D038
:1029A000432B30D15378492B00F09080A3F13101B3
:1029B0000429EAD8303B0232DEB2E260D4E90531C4
:1029C0008B4280F29780216901EB031503F1010C22
:1029D00000276F601B01C4F814C0002800F090802D
:1029E0004FF0070C6F6001F803C02E72E860117899
:1029F0005BE7C168E36A0B44E362117843290B4645
:102A0000D0D04429C4D15178303905292AD8DFE8FB
:102A100001F0031D262923204FF0010CD4E90531D4
:102A2000951C8B42E56062DA216901EB03155F1C9E
:102A300000266E601B01676100285ED008276E606B
:102A4000CF5485F808C0E86091782EE74FF0020C6B
:102A5000E4E74FF0050CE1E74FF0040CDEE74FF040
:102A6000030CDBE7194600251FE7531CC3605178B0
:102A70006C298DD10232C260FFF7A2FDE3680646E1
:102A800008B31978452983D10133E3602046FDF767
:102A9000B3FD002816DBD4E90532934212DA22692D
:102AA0001F0102EB0315002101334FF0460C696052
:102AB000636102F807C0D4E908329342C5E90260B5
:102AC000FFF626AFE36819780025EEE6531CE360B5
:102AD0009378A3F13101042915D80332E260303B29
:102AE0002046DEB2FFF7F8F8A06AE26866E7917860
:102AF0000025DAE611780025D7E691780546D4E678
:102B000011780546D1E651780025CEE6F8B5C268C1
:102B100013784C2B31D1531CC36051785F29054683
:102B200033D05A290CD10133EB6000212846FEF73F
:102B3000A7FCEB681A78452A1FD10133EB60F8BD7A
:102B4000FFF7CAF8C8B10378272B06D183681A7C2F
:102B50001AB15A68EB6A9B1AEB62EA6814786E2C19
:102B60000DD03D21452C39D0134603E0EB601C7895
:102B7000452C12D00133002CF8D10020F8BD531C95
:102B8000EB6054783E211A46ECE7931CC3609278C0
:102B90005A2A18BF0020CED1C5E79C1AD5E9056393
:102BA0009E4219DAD5F810C000270CEB061306F187
:102BB000010EBC425F604FEA0616C5F814E00BDD5B
:102BC0005F600CF80670C3E9022402462846FDF750
:102BD000B7FBEB681A78AEE70023F6E70024DDE7E1
:102BE0002DE9F04F044697B0002A74D05368012BAA
:102BF000154670DCD0F81C21B2F5806F6BDC0E46F8
:102C0000591C6960D0F81871D0F82C11029502F1A6
:102C1000010C02A8C4F81CC10391C4F82C01002FB8
:102C200040F0D88095F800C0BCF1500F01F216803A
:102C3000DFE81CF0E707200120018C03710818046D
:102C4000BE07B1078C07660740071A07F406CE06D1
:102C50008D06670641061B06F505CF05A905830508
:102C60005D0537050D05FB00FB00FB00D800D80013
:102C7000D800D800D800D800D80008020802D80030
:102C8000D8004A023E0222027802DE01DC02DE01A6
:102C90009A019A0175093009B009D70814080A0980
:102CA000FD0838032D03720A620AFB01FB0157017C
:102CB00057013C0A2A0A080AD909EB0AC50A9F0AE1
:102CC000790A1408E804C2049C0442044608D800A7
:102CD0001B08D800D8000123C4F8183117B0BDE88C
:102CE000F08FAA6893681B685978632902F05284B0
:102CF00005F10C033146204603F044FE0746002848
:102D000042F04084AB681A78322A02F0DC849B6877
:102D1000C949186806F018F8EB6820B99A68117864
:102D2000032902F019869A683146204603F0DAFD3D
:102D3000AF68C249BB68D3F80080404606F004F88B
:102D40008146002842F0B084D4F80031FF2B0ED128
:102D500084F8FF0019462046D4E942329847D4F857
:102D60002831C4F800915A1CC4F828214B46591C3C
:102D70005B22C4F80011E25484F80421EB68314668
:102D8000DA682046FFF72CFFD4F80031FF2B0FD173
:102D90000026194684F8FF60D4E94232204698475D
:102DA000D4F82831C4F800615A1CC4F828213346ED
:102DB0005D22591CC4F80011E25484F80421AB6868
:102DC0001A78322A02F02E856B68D4F81C210399F8
:102DD000013B013AC4F82C116B60C4F81C2117B0F8
:102DE000BDE8F08F0022D4E94431CDE9061506A9EB
:102DF000C4F814110021CDE90813A946002A36D0E1
:102E000031462046FFF7ECFE089B002B01F0688559
:102E1000069BC4F814310FB1C4F810816B68D4F864
:102E20001C210399013B013AD4E7D4F814E173461D
:102E3000BEF1000F0ED0996849B95A681278A2F114
:102E40001900022802F2EB81944502F0DB811B6835
:102E5000002BF0D1A94606ABC4F81431D4F81031D8
:102E6000CDF818E00022CDE90823CDF81C90D9F860
:102E70000820C5E7AA6831462046FFF7B1FE16F0E4
:102E8000040A02F0DA80D4F80031FF2B0FD10027BA
:102E9000194684F8FF70D4E9423220469847D4F8A6
:102EA0002831C4F800715A1CC4F828213B462E2250
:102EB000591CC4F80011E25484F80421D5F80C80A0
:102EC00098F80030472B02F0F68142463146204602
:102ED000FFF786FE6B68D4F81C210399013B013A89
:102EE00078E7AA681378272B01F06E870027D4F8BB
:102EF0000011FF290ED14FF00008D4E9423284F8C6
:102F0000FF8020469847D4F82831AA68013341460B
:102F1000C4F828312823481CC4F800016354204613
:102F200084F804313146FFF75BFED4F80031FF2B03
:102F300001F07487591C2922C4F80011E25484F866
:102F400004212B783E2B02F03182082F02F0BD8045
:102F5000EA6831462046FFF743FE6B68D4F81C212F
:102F60000399013B013A35E7AA681AB13146204678
:102F7000FFF736FEEB68002B02F02C81D4F800310D
:102F8000FD2B0ED90027E75419462046D4E94232DA
:102F90009847D4F82831C4F800715A1CC4F8282185
:102FA0003B46DFF89C904FF02C0809F1010B4FF0E5
:102FB000000A19460CE00B460131CB45C4F800115C
:102FC00004F8038084F8048101F0AB8419F8018FC0
:102FD000FF29F0D1D4E9423284F8FFA02046984777
:102FE000D4F828310133C4F8283101210023E4E763
:102FF000D4E9443106AA0020CDE90615C4F814210D
:103000000890EA68099331462046FFF7E9FD089BDE
:10301000002B01F0FC866B68D4F81C210699C4F8DB
:103020001411013B0399013AD4E60123C4F8183185
:103030006B68013BCEE600BF943D0208983D020854
:103040006C3D0208D4F82031D5F808902BB999F8D6
:103050000070052F02F0C3811F4699F80030232B22
:1030600001F096842A789A4201F09284242B02F08F
:103070001783D4F814E1EDE6B30601F12F86AA68B0
:10308000002A02F0DD8016F0400026F0600602F013
:10309000E080D4F81431314605F10C02204603F0EB
:1030A000DBF86B68D4F81C210399013B013A91E6E7
:1030B000AA6831462046FFF793FD6B68D4F81C21BF
:1030C0000399013B013A85E616F0040641F0648459
:1030D000AF68D7E9007000283FF47CAE3844D4F8DC
:1030E000001100F1FF39013FB04609E00B46013104
:1030F000B945C4F80011E65484F8046101F0CE85A6
:10310000FF2917F8016FF1D1D4E9423284F8FF802A
:1031100020469847D4F828310133C4F828310121DA
:103120000023E5E7D4E9443E0DF118097146002279
:10313000CDF800E0CDF818E0CDE908230795C4F8F4
:103140001491CE46002902F094844FF00108B44651
:10315000009FC3464E4617E0BB689BB9B8F1030F0A
:1031600002F2728097E80F00AAF1400E8EE80F007D
:103170004AF8406C09EB0816C4F8146108F101081C
:10318000C7F808B03F683FB17B681B78193B022B3A
:1031900016AB03EB081ADFD9EA686146204666469B
:1031A000FFF71EFD089B009AC4F81421BBB9B8F1C3
:1031B000010F0CD009EB08180AAF58F80C2C314657
:1031C000A8F11008204602F041FD4745F5D1D4F89A
:1031D0001431314605F10802204603F06DFA6B68A0
:1031E000D4F81C210399013B013AF3E5B5F90E30FF
:1031F000002B41F04587AA68D84B9168994201F0AD
:10320000498531462046FFF7EBFCD4F80031FF2B0F
:103210000FD10026194684F8FF60D4E942322046D7
:103220009847D4F82831C4F800615A1CC4F8282102
:1032300033462022591CC4F80011E25484F80421BA
:10324000B5F90C30002B41F0C684C54F984607F104
:1032500005095F260BE00B460131B945C4F80011A2
:10326000E65484F8046101F0AE8417F8016FFF2979
:10327000F1D1D4E9423284F8FF8020469847D4F84F
:1032800028310133C4F8283101210023E5E7EB6838
:103290001B78392B3FF425AD0123C4F818316B6836
:1032A000013B97E5D5E9028798F80030322B01F011
:1032B0001386342B42F0EE83D4F80031FF2B10D16B
:1032C0004FF00009194684F8FF90D4E942322046B5
:1032D0009847D4F82831C4F800915A1CC4F8282122
:1032E0004B46591C2822C4F80011E25484F80421EA
:1032F000D8F8082031462046FFF772FCD4F8003198
:10330000FF2B10D14FF00008194684F8FF80D4E954
:10331000423220469847D4F82831C4F800815A1C1C
:10332000C4F8282143462922591CC4F80011E2544C
:1033300084F804213A463146204603F0D3FA6B68FC
:10334000D4F81C210399013B013A43E5D4F8143128
:10335000D5F8088000930023C4F81431B8F1000FA9
:1033600002F0C2800DF11809D4F810E11F4618468A
:103370004A46C2E90038C2E9020E98F800104D2909
:10338000A1F11C0AA1F14F0C07F10107134601F04E
:10339000DD8200F26087BAF1040F41F2D782022980
:1033A000C4F8142116D1D8F80C8098F80030472BB7
:1033B00002F0578309EB071C98F800304D2BA3F15E
:1033C0001C01A3F14F0201F0EB8601F2E68604290D
:1033D00041F2E68698F80030042B04D1CDE904E8E8
:1033E00004ABC4F81031EA6831462046FFF7F8FB19
:1033F00098F80030042B02D1049BC4F8103109EB7B
:1034000007174FF02008AA4657F8085CE5B9D4F82A
:103410000011FF290BD1D4E9423284F8FF50204635
:103420009847D4F8283101332946C4F828314B1C79
:10343000C4F8003157F80C2C04F8018020463146BE
:1034400084F8048102F002FC103FB945DCD1009BF6
:10345000C4F8143155466B68D4F81C210399013B1C
:10346000013AB7E4D4F82031002B01F08C833D4FB2
:10347000D4F8001107F1040961264FF000080BE0B1
:103480000B460131B945C4F80011E65484F80461D3
:1034900001F0CB8317F8016FFF29F1D1D4E9423253
:1034A00084F8FF8020469847D4F828310133C4F8C7
:1034B000283101210023E5E7A9682046FDF780FABD
:1034C0004FF0000A002802F0878103782F2B41F08B
:1034D0004D828368002B01F04982C0680AF1010A1D
:1034E0000028F2D1AB681A460AF1FF3300939046E8
:1034F000A146019503E00137BA4541F30882C9F8B6
:103500002471424631464846FFF76AFB009B9F42C2
:10351000F1DA154CD9F8001104F1010B2C250BE060
:103520000B460131A345C9F8001109F8035089F889
:103530000451E0D014F8015FFF29F1D14FF00003EE
:1035400089F8FF304846D9E942329847D9F82831FE
:103550000133C9F8283101210023E3E7CC1E02081A
:103560005C3D0208E43B02086C3D0208DFF8F8838A
:10357000D4F8001108F1190A6E274FF000090BE08A
:103580000B460131C245C4F80011E75484F80471B8
:1035900001F0148118F8017FFF29F1D1D4E94232FA
:1035A00084F8FF9020469847D4F828310133C4F8B6
:1035B000283101210023E5E7DFF8B083D4F80011BA
:1035C00008F1150A74274FF000090BE00B46013192
:1035D000C245C4F80011E75484F8047101F0E18099
:1035E00018F8017FFF29F1D1D4E9423284F8FF9025
:1035F00020469847D4F828310133C4F828310121F6
:103600000023E5E7D74FD4F8001107F10D097B2619
:103610004FF000080BE00B460131B945C4F800112A
:10362000E65484F8046100F08B8717F8016FFF29D6
:10363000F1D1D4E9423284F8FF8020469847D4F88B
:1036400028310133C4F8283101210023E5E7D5E909
:10365000026000283FF4BEAB3044D4F8001100F102
:10366000FF39013E4FF0000809E00B460131B1453A
:10367000C4F80011E75484F8047101F03881FF297F
:1036800016F8017FF1D1D4E9423284F8FF80204658
:103690009847D4F828310133C4F828310121002398
:1036A000E5E7DFF8CC82D4F8001108F1100A6827AA
:1036B0004FF000090BE00B460131C245C4F8001180
:1036C000E75484F8047100F0888718F8017FFF2917
:1036D000F1D1D4E9423284F8FF9020469847D4F8DB
:1036E00028310133C4F8283101210023E5E7DFF850
:1036F0008482D4F8001108F1140A72274FF00009EF
:103700000BE00B460131C245C4F80011E75484F8C0
:10371000047100F0CA8718F8017FFF29F1D1D4E9BC
:10372000423284F8FF9020469847D4F8283101337C
:10373000C4F8283101210023E5E7DFF83C82D4F802
:10374000001108F1180A54274FF000090BE00B464E
:103750000131C245C4F80011E75484F8047100F047
:10376000978718F8017FFF29F1D1D4E9423284F814
:10377000FF9020469847D4F828310133C4F8283107
:1037800001210023E5E7DFF8F481D4F8001108F106
:10379000150A54274FF000090BE00B460131C245D2
:1037A000C4F80011E75484F8047100F0648718F835
:1037B000017FFF29F1D1D4E9423284F8FF902046FD
:1037C0009847D4F828310133C4F828310121002367
:1037D000E5E7DFF8AC81D4F8001108F1120A672799
:1037E0004FF000090BE00B460131C245C4F800114F
:1037F000E75484F8047100F0318718F8017FFF293D
:10380000F1D1D4E9423284F8FF9020469847D4F8A9
:1038100028310133C4F8283101210023E5E7DFF81E
:103820006481D4F8001108F10E0A6A274FF00009EC
:103830000BE00B460131C245C4F80011E75484F88F
:10384000047100F0FE8618F8017FFF29F1D1D4E958
:10385000423284F8FF9020469847D4F8283101334B
:10386000C4F8283101210023E5E7DFF81C81D4F8F2
:10387000001108F1190A63274FF000090BE00B460D
:103880000131C245C4F80011E75484F8047100F016
:10389000CB8618F8017FFF29F1D1D4E9423284F8B0
:1038A000FF9020469847D4F828310133C4F82831D6
:1038B00001210023E5E7DFF8D480D4F8001108F1F6
:1038C000100A76274FF000090BE00B460131C24584
:1038D000C4F80011E75484F8047100F0988618F8D1
:1038E000017FFF29F1D1D4E9423284F8FF902046CC
:1038F0009847D4F828310133C4F828310121002336
:10390000E5E7DFF88C80D4F8001108F1140A6E277F
:103910004FF000090BE00B460131C245C4F800111D
:10392000E75484F8047100F0658618F8017FFF29D8
:10393000F1D1D4E9423284F8FF9020469847D4F878
:1039400028310133C4F8283101210023E5E7DFF8ED
:103950004480D4F8001108F10F0A74274FF00009D1
:1039600026E000BF483E0208383D02083C3D020800
:10397000243D02080C3D0208F03C0208D83C020835
:10398000C43C0208B43C0208983C0208843C02088B
:10399000803C02086C3C02080B460131C245C4F869
:1039A0000011E75484F8047100F0808718F8017F53
:1039B000FF29F1D1D4E9423284F8FF90204698479C
:1039C000D4F828310133C4F8283101210023E5E778
:1039D000DFF86485D4F8001108F1110A74274FF05C
:1039E00000090BE00B460131C245C4F80011E75451
:1039F00084F8047100F04D8718F8017FFF29F1D198
:103A0000D4E9423284F8FF9020469847D4F8283110
:103A10000133C4F8283101210023E5E7DFF81C85D4
:103A2000D4F8001108F10C0A74274FF000090BE0DC
:103A30000B460131C245C4F80011E75484F8047103
:103A400000F00D8718F8017FFF29F1D1D4E9423247
:103A500084F8FF9020469847D4F828310133C4F801
:103A6000283101210023E5E7DFF8D484D4F80011E0
:103A700008F1170A63274FF000090BE00B460131EC
:103A8000C245C4F80011E75484F8047100F0BD8603
:103A900018F8017FFF29F1D1D4E9423284F8FF9070
:103AA00020469847D4F828310133C4F82831012141
:103AB0000023E5E7DFF88C84D4F8001108F1070A49
:103AC00056274FF000090BE00B460131C245C4F800
:103AD0000011E75484F8047100F08A8618F8017F19
:103AE000FF29F1D1D4E9423284F8FF90204698476B
:103AF000D4F828310133C4F8283101210023E5E747
:103B0000DFF84484D4F8001108F10A0A76274FF050
:103B100000090BE00B460131C245C4F80011E7541F
:103B200084F8047100F0578618F8017FFF29F1D15D
:103B3000D4E9423284F8FF9020469847D4F82831DF
:103B40000133C4F8283101210023E5E7D4F800113E
:103B5000FF290CD10027D4E9423284F8FF702046B7
:103B60009847D4F8283101333946C4F828317E23E8
:103B70004A1CC4F80021635484F80431EA683146D1
:103B80002046FFF72DF86B68D4F81C210399013B00
:103B9000013AFFF71FB9EA6831462046FFF720F8DF
:103BA0006B68D4F81C210399013B013AFFF712B965
:103BB000D5F80880B8F1000F40F06A87DD4FD4F8DF
:103BC000001107F1030974260BE00B460131B945DA
:103BD000C4F80011E65484F8046100F0CC8717F8AB
:103BE000016FFF29F1D1D4E9423284F8FF802046E9
:103BF0009847D4F828310133C4F828310121002333
:103C0000E5E716F0040640F0F286D5E902700028D8
:103C10003FF4E0A83844D4F8001100F1FF39013F27
:103C2000B04609E00B460131B945C4F80011E6542D
:103C300084F8046101F04A80FF2917F8016FF1D17F
:103C4000D4E9423284F8FF8020469847D4F82831DE
:103C50000133C4F8283101210023E5E70123C4F82A
:103C600018316B68013BFFF7B5B8DFF8E082AA684E
:103C700031462046FEF7B4FF08F1070AD4F80011D8
:103C800020274FF000090BE00B460131C245C4F874
:103C90000011E75484F8047100F0328518F8017FB0
:103CA000FF29F1D1D4E9423284F8FF9020469847A9
:103CB000D4F828310133C4F8283101210023E5E785
:103CC000DFF88C82AA6831462046FEF789FF08F1AA
:103CD000040AD4F800115B274FF000090BE00B46F3
:103CE0000131C245C4F80011E75484F8047100F0B2
:103CF000338518F8017FFF29F1D1D4E9423284F8E5
:103D0000FF9020469847D4F828310133C4F8283171
:103D100001210023E5E700237207D4F81481D4F8C9
:103D20004871D5F80890C4F81431C4F8485107D543
:103D300099F8003023B9D9F80C20062A01F05E85E5
:103D40004A4631462046FEF74BFF94F804313C2B9F
:103D500001F0A480D4F80011FF290DD14FF0000923
:103D6000D4E9423284F8FF9020469847D4F82831AD
:103D700001334946C4F828313C234A1CC4F80021C9
:103D8000635484F80431EA6831462046FEF728FF80
:103D900094F804313E2B01F06480D4F80011FF291F
:103DA0000CD10026D4E9423284F8FF6020469847BF
:103DB000D4F8283101333146C4F828313E234A1C57
:103DC000C4F80021635484F804316B68D4F81C21D2
:103DD0000399C4F81481C4F84871013B013AFEF715
:103DE000F9BFDFF87081D4F8001108F1080A6F27D5
:103DF0004FF000090BE00B460131C245C4F8001139
:103E0000E75484F8047100F02E8218F8017FFF292E
:103E1000F1D1D4E9423284F8FF9020469847D4F893
:103E200028310133C4F8283101210023E5E7AA68CD
:103E30003146204602F01AFD6B68D4F81C21039924
:103E4000013B013AFEF7C6BFDFF80881D4F8001144
:103E500008F1080A6F274FF000090BE00B4601310B
:103E6000C245C4F80011E75484F8047100F07B8265
:103E700018F8017FFF29F1D1D4E9423284F8FF908C
:103E800020469847D4F828310133C4F8283101215D
:103E90000023E5E7D5E902281AB131462046FEF7AE
:103EA0009FFED4F80031FF2B0DD10027194684F86E
:103EB000FF70D4E9423220469847D4F828315A1C82
:103EC000C4F828213B46581C7B27C4F80001314622
:103ED000E7544246204684F80471FEF781FED4F888
:103EE0000011FF290CD10026D4E9423284F8FF608A
:103EF00020469847D4F8283101333146C4F8283198
:103F00004A1C7D23C4F80021635484F804316B6893
:103F1000D4F81C210399013B013AFEF75BBFDFF89F
:103F20003880D4F8001108F11D0A74274FF00009F9
:103F300020E000BFE83D0208583C0208483C020867
:103F4000243C0208183C02080C3C0208583E0208B7
:103F5000B43B02087C3D0208EC3B02080B460131F1
:103F6000C245C4F80011E75484F8047100F01C82C3
:103F700018F8017FFF29F1D1D4E9423284F8FF908B
:103F800020469847D4F828310133C4F8283101215C
:103F90000023E5E7D5F80890D34FD9F80880D4F886
:103FA000001107F1070B6F264FF0000A0BE00B46DC
:103FB0000131BB45C4F80011E65484F8046100F0F7
:103FC0005F8117F8016FFF29F1D1D4E9423284F8FB
:103FD000FFA020469847D4F828310133C4F828318F
:103FE00001210023E5E7AA68C04906A818F04AFDA8
:103FF00006A805F025F8002800F0A08106AED4F848
:10400000001106EB00094FF0000809E00B460131F2
:10401000B145C4F80011E75484F8047100F08E81B2
:10402000FF2916F8017BF1D1D4E9423284F8FF80F0
:1040300020469847D4F828310133C4F828310121AB
:104040000023E5E7D4F800012E7AFF2814D14FF0C1
:104050000008D4E94232014684F8FF8020469847A0
:10406000D4F828016B68D4F81C210399471CC4F8C4
:1040700028714046013B013A471CC4F800712654A0
:1040800084F80461FEF7A6BEAA6831462046FEF712
:10409000A7FDEA6831462046FEF7A2FD6B68D4F81A
:1040A0001C210399013B013AFEF794BEDFF84082E0
:1040B000D4F8001108F10D0A6A274FF000090BE04F
:1040C0000B460131C245C4F80011E75484F804716D
:1040D00000F03C8118F8017FFF29F1D1D4E9423288
:1040E00084F8FF9020469847D4F828310133C4F86B
:1040F000283101210023E5E7EB6818783B2804D13B
:10410000DB681B783C2B01F0B1810123C4F8183126
:104110006B68013BFEF75EBE0123C4F818316B6883
:10412000013BFEF757BEDFF8CC81D4F8001108F14F
:10413000070A7B274FF000090BE00B460131C2450F
:10414000C4F80011E75484F8047100F0548118F8A1
:10415000017FFF29F1D1D4E9423284F8FF90204653
:104160009847D4F828310133C4F8283101210023BD
:10417000E5E7DFF88481D4F8001108F11B0A67270E
:104180004FF000090BE00B460131C245C4F80011A5
:10419000E75484F8047100F0218118F8017FFF29A9
:1041A000F1D1D4E9423284F8FF9020469847D4F800
:1041B00028310133C4F8283101210023E5E7DFF875
:1041C0003C81D4F8001108F11C0A67274FF0000960
:1041D0000BE00B460131C245C4F80011E75484F8E6
:1041E000047100F0EE8018F8017FFF29F1D1D4E9C5
:1041F000423284F8FF9020469847D4F828310133A2
:10420000C4F8283101210023E5E7DFF8F480D4F871
:10421000001108F1090A64274FF000090BE00B4672
:104220000131C245C4F80011E75484F8047100F06C
:10423000628118F8017FFF29F1D1D4E9423284F874
:10424000FF9020469847D4F828310133C4F828312C
:1042500001210023E5E7BCF1010F40F27783C4F8A8
:104260001421FFF7B7B8EA6831462046FEF7B8FCDC
:104270006B68D4F81C210399013B013AFEF7AABDF3
:10428000D9F804603378613B192B1AD8FF290DD176
:104290000026D4E9423284F8FF6020469847D4F8DB
:1042A0002831C4F800610133C4F82831D4F8002162
:1042B0002023511CC4F80011A35484F80431D9F808
:1042C00004604346F21812F8012C202A08BF08F1B6
:1042D000FF33002B01F0D382013ED4F8001106EB2E
:1042E00003094FF0000817E0703D0208D03B0208B8
:1042F000C83D0208383E0208183E0208F83D020890
:10430000D83D02080B460131B145C4F80011E7540D
:1043100084F8047100F0F382FF2916F8017FF1D1CF
:10432000D4E9423284F8FF8020469847D4F82831F7
:104330000133C4F8283101210023E5E76B68D4F884
:104340001C210399013B013AFEF744BDAA6831469E
:104350002046FEF745FC6B68D4F81C210399013B0D
:10436000013AFEF737BDD4F8483133B1D4F8102103
:10437000079306AB0692C4F81031AA681378042B91
:1043800000F0C68431462046FEF72AFCD4F84831B6
:1043900013B1069BC4F810316B68D4F81C21039943
:1043A000013B013AFEF716BDAA6831462046FEF7EA
:1043B00017FC6B68D4F81C210399013B013AFEF706
:1043C00009BDAA6831462046FEF70AFC6B68D4F89E
:1043D0001C210399013B013AFEF7FCBCAA68314657
:1043E0002046FEF7FDFB6B68D4F81C210399013BC6
:1043F000013AFEF7EFBCD4F82031AA68D34F01335D
:104400003146C4F820312046FEF7EAFBD4F82031CB
:10441000D4F80011013BC4F8203107F10109292625
:104420004FF000080AE00B460131B945C4F800110D
:10443000E65484F8046111D017F8016FFF29F2D116
:10444000D4E9423284F8FF8020469847D4F82831D6
:104450000133C4F8283101210023E6E7EA68BC49AA
:10446000013206A818F00EFB06A804F0E9FD10B30F
:1044700006AED4F8001106EB00094FF0000808E082
:104480000B460131B145C4F80011E75484F80471BA
:1044900013D0FF2916F8017BF2D1D4E9423284F817
:1044A000FF8020469847D4F828310133C4F82831DA
:1044B00001210023E6E7D4F80011FF290CD10026E2
:1044C000D4E9423284F8FF6020469847D4F8283176
:1044D00001333146C4F828314A1C7D23C4F8002139
:1044E000635484F804316B68D4F81C210399013BB0
:1044F000013AFEF76FBC3146AA682046FEF770FB12
:10450000D4F80011FF290CD10026D4E9423284F8F6
:10451000FF6020469847D4F8283101333146C4F86B
:1045200028314A1C2923C4F80021635484F804313B
:104530006B68D4F81C210399013B013AFEF74ABC91
:10454000AA688349013206A818F09CFA06A804F06C
:1045500077FD10B306AED4F8001106EB00094FF05A
:10456000000808E00B460131B145C4F80011E754DA
:1045700084F8047113D0FF2916F8017BF2D1D4E935
:10458000423284F8FF8020469847D4F8283101331E
:10459000C4F8283101210023E6E7D4F80011FF29EF
:1045A0000CD10026D4E9423284F8FF6020469847B7
:1045B000D4F8283101333146C4F828314A1C7D2310
:1045C000C4F80021635484F804316B68D4F81C21CA
:1045D0000399013B013AFEF7FDBBAA68314620462C
:1045E000FEF7FEFA6B68D4F81C210399013B013AEF
:1045F000FEF7F0BBAA6831462046FEF7F1FA6B6879
:10460000D4F81C210399013B013AFEF7E3BBAA68E9
:1046100031462046FEF7E4FA6B68D4F81C21039972
:10462000013B013AFEF7D6BBAA6831462046FEF7A9
:10463000D7FA6B68D4F81C210399013B013AFEF7C5
:10464000C9BBAA6831462046FEF7CAFA6B68D4F89F
:104650001C210399013B013AFEF7BCBBAA68314615
:104660002046FEF7BDFA6B68D4F81C210399013B84
:10467000013AFEF7AFBBAA6831462046FEF7B0FA12
:104680006B68D4F81C210399013B013AFEF7A2BBE9
:10469000AA6831462046FEF7A3FA6B68D4F81C21BD
:1046A0000399013B013AFEF795BBDFF8A880EA6861
:1046B00031462046FEF794FA08F1040AD4F80011B6
:1046C00020274FF000090BE00B460131C245C4F82A
:1046D0000011E75484F8047100F0F58018F8017FA8
:1046E000FF29F1D1D4E9423284F8FF90204698475F
:1046F000D4F828310133C4F8283101210023E5E73B
:104700003146EA682046FEF76BFAD4F80011FF291B
:104710000CD10026D4E9423284F8FF602046984745
:10472000D4F8283101333146C4F828314A1C5D23BE
:10473000C4F80021635484F804316B68D4F81C2158
:104740000399013B013AFEF745BB00BF443E020816
:10475000D03B0208043D02083146EA682046FEF7D5
:104760003FFAD4F80011FF290CD10026D4E94232D7
:1047700084F8FF6020469847D4F828310133314649
:10478000C4F828314A1C5D23C4F80021635484F81E
:1047900004316B68D4F81C210399013B013AFEF700
:1047A00019BBAA6831462046FEF71AFA6B68D4F89E
:1047B0001C210399013B013AFEF70CBBAA68314664
:1047C0002046FEF70DFA6B68D4F81C210399013BD3
:1047D000013AFEF7FFBAAA6831462046FEF700FA12
:1047E0006B68D4F81C210399013B013AFEF7F2BA39
:1047F000AA6831462046FEF7F3F96B68D4F81C210D
:104800000399013B013AFEF7E5BADFF8B885AA68DB
:1048100031462046FEF7E4F908F1030AD4F8001106
:104820002D274FF000090AE00B460131C245C4F8BC
:104830000011E75484F804711ED018F8017FFF2995
:10484000F2D1D4E9423284F8FF9020469847D4F858
:1048500028310133C4F8283101210023E6E7AA6892
:1048600031462046FEF7BCF96B68D4F81C21039949
:10487000013B013AFEF7AEBAEA6831462046FEF740
:10488000AFF96B68D4F81C210399013B013AFEF79C
:10489000A1BAAA6831462046FEF7A2F96B68D4F89F
:1048A0001C210399013B013AFEF794BAAA683146EC
:1048B0002046FEF795F96B68D4F81C210399013B5B
:1048C000013AFEF787BAAA6831462046FEF788F912
:1048D0006B68D4F81C210399013B013AFEF77ABAC0
:1048E0004A463146204601F0B1F9FEF791BA6B68AD
:1048F000D4F81C210399013B013AFEF76BBA6B68AF
:10490000D4F81C210399013B013AFEF763BA019DDB
:10491000D9F81C216B6803994C46013B013AFEF71C
:1049200059BAEA680F4620463146D4F82861FEF7A6
:1049300057F9D4F828319E4200F054846B68D4F8BB
:104940001C210399013B013AFEF744BAD8F80880CC
:10495000B8F1000F00F0C685042F02F110027EF4BA
:1049600008AD0122C4E94532FEF775BDAB681A46B1
:10497000BAF1000F7EF4B8AD6B68D4F81C2103992E
:10498000013B013AFEF726BA2B782F2B00D0A9461F
:10499000D4F814E1FEF75FBAAE68D6E902600028E9
:1049A0003EF418AA3044D4F8001100F1FF39013E5A
:1049B0004FF0000809E00B460131B145C4F8001181
:1049C000E75484F8047100F07981FF2916F8017F1B
:1049D000F1D1D4E9423284F8FF8020469847D4F8D8
:1049E00028310133C4F8283101210023E5E7D5E956
:1049F000026006EB00084645BEF4ECA94FF0000942
:104A000009E04B1CC4F80031675484F80471013686
:104A1000B04540F24B81A8EB0603032B377801DD4C
:104A20005F2F11D0D4F80011FF29EAD1D4E9423226
:104A300084F8FF9020469847D4F828310133C4F811
:104A4000283100210123DDE773785F2BEAD1B378A9
:104A5000552BE7D1F31C9845E4D9002005E0174613
:104A6000984507EB001001F012809A4613F8017B7D
:104A7000A7F130025FFA82FCBCF1090FA7F14101F6
:104A8000EDD90529A7F1610200F2A384373FE7E7DA
:104A9000C94FD4F8001107F1050A7B264FF0000931
:104AA0000AE00B460131BA45C4F80011E65484F817
:104AB000046111D017F8016FFF29F2D1D4E9423215
:104AC00084F8FF9020469847D4F828310133C4F881
:104AD000283101210023E6E7B849424606A817F02D
:104AE000D1FF06A804F0ACFA10B306AED4F800115A
:104AF00006EB00094FF0000808E00B460131B14514
:104B0000C4F80011E75484F8047111D0FF2916F895
:104B1000017BF2D1D4E9423284F8FF8020469847E5
:104B2000D4F828310133C4F8283101210023E6E705
:104B3000D4F80031FF2B0FD10026194684F8FF600E
:104B4000D4E9423220469847D4F82831C4F80061AD
:104B50005A1CC4F828213346591C7D22C4F8001180
:104B6000E25484F804216B68D4F81C210399013BBA
:104B7000013AFEF72FB96B68D4F81C210399013B69
:104B8000013AFEF727B905F108012046FBF708FFB7
:104B90000246002800F0B88403782F2B00F0A98487
:104BA000D4F810713B68C4F8103131462046FEF746
:104BB00017F86B68D4F81C210399C4F81071013BF5
:104BC000013AFEF707B96B68D4F81C210399013B41
:104BD000013AFEF7FFB87A4E5F2706F105094FF05C
:104BE00000080AE00B460131B145C4F80011E75452
:104BF00084F8047111D016F8017FFF29F2D1D4E9AD
:104C0000423284F8FF8020469847D4F82831013397
:104C1000C4F8283101210023E6E76B68D4F81C2191
:104C20000399013B013AFEF7D5B8AA6863490132FE
:104C300006A817F027FF06A804F002FA10B306AE84
:104C4000D4F8001106EB00094FF0000808E00B460D
:104C50000131B145C4F80011E75484F8047111D052
:104C6000FF2916F8017BF2D1D4E9423284F8FF80A3
:104C700020469847D4F828310133C4F8283101215F
:104C80000023E6E76B68D4F81C210399013B013A45
:104C9000FEF7A0B8D4F80011FEF7D2BA6B68D4F8CA
:104CA0001C210399013B013AFEF794B86B68D4F8D4
:104CB0001C210399013B013AFEF78CB86B68D4F8CC
:104CC0001C210399013B013AFEF784B86B68D4F8C4
:104CD0001C210399013B013AFEF77CB826F06001E4
:104CE00005F10C02D4F814310091204601F0B4FA19
:104CF000AA680099002A00F0CA852046FDF770FFD7
:104D00006B68D4F81C210399013B013AFEF762B8A5
:104D1000926831462046FDF763FFD4F8483113B15D
:104D2000069BC4F8103194F804313C2B00F00F8539
:104D3000D4F80031FF2B0FD10027194684F8FF70FB
:104D4000D4E9423220469847D4F82831C4F800719B
:104D50005A1CC4F828213B46591C3C22C4F80011B7
:104D6000E25484F80421AB683146DA682046FDF746
:104D700037FF94F804313E2B00F0CC84D4F8003196
:104D8000FF2B0FD10026194684F8FF60D4E9423288
:104D900020469847D4F82831C4F800615A1CC4F85A
:104DA000282133463E22591CC4F80011E25484F8ED
:104DB0000421FFF7F1BA00BFF03D0208D03B020822
:104DC000643D0208403C020893681F7C062F00F2F5
:104DD000BF81002F3EF48BA8EB6893F80080B8F1F8
:104DE000000F7EF484A8BCF13E0F00F0F486EA6860
:104DF00031462046023FFDF7F3FE042F00F21487F0
:104E0000DFE817F0C606A306960689067C0631463B
:104E10002A46204600F01AFFFEF7FDB80022194688
:104E200084F8FF202046D4E942329847D4F828314C
:104E300001210B442922C4F82831C4F80011227042
:104E400084F804212B783E2B7EF47FA8D4F800212F
:104E50002D23511CC4F80011A35484F80431FEF72B
:104E600074B8D4F80031FF2B0FD10026194684F80E
:104E7000FF60D4E9423220469847D4F82831C4F87C
:104E800000615A1CC4F8282133462022591CC4F85A
:104E90000011E25484F80421FEF77FBFD4F80031FA
:104EA000FF2B10D14FF00009194684F8FF90D4E988
:104EB000423220469847D4F82831C4F800915A1C51
:104EC000C4F828214B462022591CC4F80011E25492
:104ED00084F80421FEF73EBFD8F80830D249D3F851
:104EE00000A0504603F030FF3B7810B9032B00F0D0
:104EF0009E85392B00F08985CC49504603F024FF6C
:104F00008146002800F036859AF80030732B2BD1AB
:104F10009AF80130502B27D19AF8023023BB1E4655
:104F200003E0FF68002F00F0FA823B782F2B40F05F
:104F3000F682BB68002B00F0F2821A784B2A18BF69
:104F40000136EED199682046FBF73AFD034648B199
:104F5000002304E082682AB1C068013310B10278EE
:104F60002F2AF7D01E44DCE742463146204601F0A6
:104F70007DFC9AF80030672B13D19AF80130732B1F
:104F80000FD19AF8023063B93A4631462046FDF710
:104F900027FE6B68D4F81C210399013B013AFDF709
:104FA00019BFA349504603F0CFFE804600287EF487
:104FB000C1A9D4F80031FF2B0ED184F8FF001946A7
:104FC0002046D4E942329847D4F82831C4F8008109
:104FD0005A1CC4F828214346581C4FF0280CC4F82A
:104FE00000013A4604F803C03146204684F804C163
:104FF000FDF7F6FDD4F80031FF2B0FD1002619463E
:1050000084F8FF60D4E9423220469847D4F828312A
:10501000C4F800615A1CC4F828213346591C2922BF
:10502000C4F80011E25484F804216B68D4F81C2100
:105030000399013B013AFDF7CDBE7E4FD4F8001134
:1050400007F102090AE00B460131B945C4F8001125
:1050500004F8038084F804813DF430AFFF2917F889
:10506000018BF0D1D4E9423284F8FFA02046984762
:10507000D4F828310133C4F8283101210023E4E7B2
:105080006D4FD4F8001107F105094FF0000A0AE04E
:105090000B460131B945C4F8001104F8038084F8C7
:1050A00004813EF4A8A8FF2917F8018BF0D1D4E9B8
:1050B000423284F8FFA020469847D4F828310133C3
:1050C000C4F8283101210023E4E7D4F80031FF2B94
:1050D0000FD10027194684F8FF70D4E942322046E8
:1050E0009847D4F82831C4F800715A1CC4F8282114
:1050F0003B46591C5B22C4F80011E25484F8042199
:10510000EA6831462046FDF76BFDD4F80031FF2BED
:105110000FD10026194684F8FF60D4E942322046B8
:105120009847D4F82831C4F800615A1CC4F82821E3
:105130003346591C5D22C4F80011E25484F804215E
:105140006B68D4F81C210399013B013AFDF742BE7C
:10515000072F7DF4CCAEEB68197800297DF4C7AE3B
:10516000D96801297DF4C3AEBCF13D0F7DF4BFAE1B
:105170009B681B78302B00F04A85312B7DF4B7AE4D
:105180002E4904222046FBF7A9F96B68D4F81C21AC
:105190000399013B013AFDF71DBE012A3EF623A902
:1051A000042FACF1100B0CF1100A00F09D819BE86C
:1051B0000F008CE80F0000234AF81C8C4AF8183CBA
:1051C000D8F80880C4F814C14AE905EB0137D44681
:1051D000FEF7F2B86B68D4F81C210399013B013A41
:1051E000FDF7F8BDD4F80031BB427FF4A7AB6B6884
:1051F000D4F81C210399023FC4F80071013B013A25
:10520000FDF7E8BDAA6831462046FDF7E9FC6B686A
:10521000D4F81C210399013B013AFDF7DBBD0F4691
:10522000A946FDF718BE00BF883D02088C3D020864
:10523000B4400208BC3B0208543D0208C03D0208CD
:1052400026F06006FDF725BF0123C4F81831FDF7ED
:10525000C6BF06ABD4F81471C4F81431CDE90750B9
:10526000D4F810310697314620460993FDF7B8FC73
:10527000089F069BC4F81431002F40F0EA83D4F84D
:105280000031FF2B0ED1194684F8FF70D4E9423269
:1052900020469847D4F82831C4F800715A1CC4F845
:1052A00028213B462022591CC4F80011E25484F8FE
:1052B0000421FDF7EEBED24FD4F8001107F10D0A1C
:1052C0004FF0000B09E00B460131BA45C4F800115C
:1052D00004F8039084F8049111D0FF2917F8019B7A
:1052E000F1D1D4E9423284F8FFB020469847D4F88F
:1052F00028310133C4F8283101210023E5E7D8F82B
:105300000C20C049013206A817F0BCFB06A803F028
:1053100097FE18B306AFD4F8001107EB00094FF061
:10532000000B09E00B460131B945C4F8001104F83F
:1053300003A084F804A111D0FF2917F801ABF1D123
:10534000D4E9423284F8FFB020469847D4F8283197
:105350000133C4F8283101210023E5E7AA4FD4F82E
:10536000001107F1030A4FF0000B09E00B46013171
:10537000BA45C4F8001104F8039084F8049111D0E0
:10538000FF2917F8019BF1D1D4E9423284F8FFB02C
:1053900020469847D4F828310133C4F82831012138
:1053A0000023E5E7D8F80880FDF78FBDFF297FF4DB
:1053B0004DAD4FF00008D4E9423284F8FF8020461A
:1053C0009847D4F82831C4F800810133C4F8283153
:1053D0003CE5052A00F26583573FFFF741BBD4E95E
:1053E0004CC7002F40F3D181E646924604E09F422D
:1053F0000EF1080E00F0C8815CF83320914503F1EE
:105400000103F4D1034603E05B68002B00F09382B4
:105410001A68914503D09542F6D18342F4D009F140
:1054200008012046FBF7BCFA8146A0B1002799F895
:1054300000302F2B7DF411AED4F824110029FFF693
:10544000A3AA4846FBF79AFA814600287DF405AEE8
:105450000FB1C4F810810123C4F818316B68D4F877
:105460001C210399013B013AFDF7B4BCAA6805F180
:105470000C033146204601F085FA0746002840F02B
:105480004A82D5E902A2DAF80810D36808685F49B1
:10549000D2F808B0D3E9029803F056FC002840F097
:1054A000FE815A463146204601F01CFA52463146EA
:1054B000204601F0DBF94A463146204601F012FA57
:1054C000534903222046FBF709F84246314620465D
:1054D00001F008FA6B68D4F81C210399013B013AEA
:1054E000FDF778BCC4F814210123C4F81831FDF786
:1054F000B2BFD4F824110029FFF652ABFBF73EFAF5
:10550000024600287FF44CAB0123C4F818316B68C5
:10551000D4F81C210399013B013AFDF75BBC3949E2
:10552000324606A817F0AEFA06A803F089FD08B3C4
:1055300006AED4F8001137184FF0000909E00B4609
:10554000591CB742C4F8001104F8038084F80481A0
:1055500010D0FF2916F8018BF1D1D4E9423284F83A
:10556000FF9020469847D4F828310133C4F82831F9
:105570000023E5E76B68D4F81C210399013B013A4D
:10558000FDF728BC6B68D4F81C210399013B013A54
:10559000FDF720BC1B78A3F16301012903D9723BFD
:1055A000012B3DF6A5AB3146204601F05FF9D4F85A
:1055B0000031FF2B0FD10027194684F8FF70D4E982
:1055C000423220469847D4F82831C4F800715A1C5A
:1055D000C4F828213B46591C3C22C4F80011E2546F
:1055E00084F80421EB680B4F9A6831462046FDF79A
:1055F000F7FA07F10209D4F800114FF0000A15E09C
:10560000C03B0208D03B0208D43B02089C3D020884
:10561000A03D0208903D02080B46591CB945C4F84C
:10562000001104F8038084F8048110D0FF2917F8D2
:10563000018BF1D1D4E9423284F8FFA0204698478B
:10564000D4F828310133C4F828310023E5E7EB68AA
:105650003146DA682046FDF7C3FAD4F80031FF2B53
:105660000FD10026194684F8FF60D4E94232204663
:105670009847D4F82831C4F800615A1CC4F828218E
:105680003346591C2922C4F80011E25484F804213D
:105690006B68D4F81C210399013B013AFDF79ABBD2
:1056A000D9F80820FDF79FBBB549404603F04CFBF5
:1056B000002840F0C881EB683146DA68204601F0E6
:1056C00011F9FDF77CBB9A68916801297DF41FAB45
:1056D000526812783E2A7DF41AABD4F80031FF2BC1
:1056E0000ED184F8FF0019462046D4E9423298478B
:1056F000D4F82831C4F800715A1CC4F828213B465C
:10570000591C2822C4F80011E25484F80421AB6823
:10571000FDF7FDBAD4F80031FF2B0FD10026194652
:1057200084F8FF60D4E9423220469847D4F8283103
:10573000C4F800615A1CC4F8282133462022591CA1
:10574000C4F80011E25484F80421FFF717BBD4F821
:105750000031FF2B0FD10027194684F8FF70D4E9E0
:10576000423220469847D4F82831C4F800715A1CB8
:10577000C4F828213B462022591CC4F80011E254E9
:1057800084F80421FFF7D4BA5246D4F838319F4246
:1057900080F2AA817B1C0CEBC70EC4F834314CF8A4
:1057A0003790D4F810710EF1040E002F00F0A38191
:1057B000D4E95003984200F1010C80F29581D4F8AD
:1057C0003C31C4F840C103EBC00378685860CEF8A0
:1057D00000303F689E46E8E7AA683146204601F05F
:1057E00081F8684903222046FAF778FE6B68D4F8FE
:1057F0001C210399013B013AFDF7ECBA6249D9F843
:10580000080017F0BFF900287EF49AAAEA6831462A
:105810002046FDF7E5F95D4902222046FAF75EFED3
:10582000FEF7D3BA9B689A68012A7DF4CDAA5B681B
:105830001B783E2B7DF4C8AAD4F80031FF2B0FD182
:105840000026194684F8FF60D4E942322046984782
:10585000D4F82831C4F800615A1CC4F82821334612
:10586000591C2922C4F80011E25484F804216B6801
:10587000D4F81C210399013B013AFDF7ABBA6B68E0
:10588000D4F81C210399013B013AFDF7A3BA6B68D8
:10589000D4F81C210399013B013AFDF79BBA3C491E
:1058A00004222046FAF71AFEDBF80830F3B15A4614
:1058B0003146204601F016F8D4F80031FF2B0ED106
:1058C000194684F8FF70D4E9423220469847D4F84C
:1058D0002831C4F800715A1CC4F828213B46202204
:1058E000591CC4F80011E25484F804214A46314698
:1058F0002046FDF775F9B8F1000F14D04246314645
:10590000204600F0EFFF6B68D4F81C210399013B9F
:10591000013AFDF75FBA6B68D4F81C210399013B8B
:10592000013AFDF757BA6B68D4F81C210399013B83
:10593000013AFDF74FBADEF80430D4F81081C4F80C
:10594000103109F108012046FBF72AF881460028AA
:105950003FF47FAD01276AE5D3681B78292B1CBF74
:105960000123C4F8183192683146204600F0BAFF8E
:10597000FDF7DEB939462046FBF722F880B912E080
:10598000943D0208E43D0208D83B0208E03B0208CF
:10599000A43D0208836833B1C06809F1010910B160
:1059A00003782F2BF6D0A4494A4606A817F06AF8C8
:1059B00006A803F045FB00B306AE37184FF0000809
:1059C000D4F8001116F8019BFF290DD1D4E9423219
:1059D00084F8FF8020469847D4F82831C4F8008125
:1059E0000133C4F8283100214B1CB742C4F8003100
:1059F00004F8019084F80491E2D16B68D4F81C217A
:105A00000399013B013AFDF7E5B9BA6831462046F2
:105A100000F068FF42463146204600F027FF6B68E1
:105A2000D4F81C210399013B013AFDF7D3B9BB68B7
:105A30001A78012A7FF460AAFA681278292A08BF26
:105A40001F46FFF759BA3A463146204600F00EFF8E
:105A500031E66B68D4F81C210399013B013AFDF74C
:105A6000B9B9D8F80880B8F1000F3FF43DADFDF7A3
:105A7000A1BCEA6831462046FDF7B2F8089B009ABF
:105A8000C4F81421002B3DF4A2ABFDF7A8BB5F279F
:105A9000FEF7C8BF42463146204600F0E7FEFDF75C
:105AA00049BCD045F3D95F2FF1D1FF283EF6BAAFFC
:105AB000D4F80011FF29C7B20DD1D4E9423284F8DD
:105AC000FF9020469847D4F82831C4F8009101335C
:105AD000C4F8283100214B1CC4F8003156466754E5
:105AE00084F80471FEF793BF0123C4F818316B6882
:105AF000013BFDF76FB9CEF8007090E44F490322E7
:105B00002046FAF7EBFC6B68D4F81C210399013BA3
:105B1000013AFDF75FB94A4902222046FAF7DEFC56
:105B20006B68D4F81C210399013B013AFDF752B987
:105B3000444902222046FAF7D1FC6B68D4F81C21B4
:105B40000399013B013AFDF745B9D4F80031FF2B29
:105B50000FD10026194684F8FF60D4E9423220466E
:105B60009847D4F82831C4F800615A1CC4F8282199
:105B70003346591C6C22C4F80011E25484F8042105
:105B80006B68D4F81C210399013B013AFDF722B957
:105B9000D4F80031FF2B0FD10026194684F8FF609E
:105BA000D4E9423220469847D4F82831C4F800613D
:105BB0005A1CC4F828213346591C7522C4F8001118
:105BC000E25484F804216B68D4F81C210399013B4A
:105BD000013AFDF7FFB8D4F80031FF2B0ED119467A
:105BE00084F8FF80D4E9423220469847D4F828311F
:105BF000C4F800815A1CC4F8282143462D22591CA0
:105C0000C4F80011E25484F80421FFF7F0B80E49FB
:105C100005222046FAF762FC6B68D4F81C21039930
:105C2000013B013AFDF7D6B86B68D4F81C21039903
:105C3000013B013AFDF7CEB8D03B0208B43D020863
:105C4000B03D0208AC3D0208B83D02082DE9F0471E
:105C50001378033B154604460E464D2B4FD8DFE81C
:105C600013F0BD004E004E004E004E004E004E00A0
:105C70004E004E004E004E004E004E004E004E00B4
:105C80004E004E004E004E004E004E004E0053009F
:105C900077009A00530077009A00C200CF00DC0022
:105CA000EF003801460169018C014E004E004E00A4
:105CB0004E0000014E0035024E004E004E004E00D8
:105CC0004E004E004E004E004E004E004E004E0064
:105CD0004E004E004E004E004E004E004E004E0054
:105CE0004E004E004E004E004E004E004E004E0044
:105CF0004E004E004E00B0014E00D401FA012A467B
:105D0000BDE8F047FCF76CBFD84ED0F8001106F1A3
:105D10000808202500270BE00B460131B045C4F8E8
:105D20000011E55484F8045100F0998016F8015FE1
:105D3000FF29F1D1D4E9423284F8FF702046984718
:105D4000D4F828310133C4F8283101210023E5E7D4
:105D5000C74ED0F8001106F10808202500270AE0F8
:105D60000B460131B045C4F80011E55484F80451E4
:105D700075D016F8015FFF29F2D1D4E9423284F8D8
:105D8000FF7020469847D4F828310133C4F82831F1
:105D900001210023E6E7B74ED0F8001106F105080F
:105DA000202500270AE00B460131B045C4F8001158
:105DB000E55484F8045152D016F8015FFF29F2D15E
:105DC000D4E9423284F8FF7020469847D4F828314D
:105DD0000133C4F8283101210023E6E7AA68BDE8B1
:105DE000F047FCF7FDBED0F80031FF2B00F0E68154
:105DF0002022591CC0F80011C25480F804216AE026
:105E0000D0F80031FF2B00F0CA81591C2022C4F8C1
:105E10000011E25484F804216BE0D0F80011FF294E
:105E200000F0AF814A1C2023C4F80021635484F899
:105E30000431EA6831462046BDE8F047FCF7D0BEA1
:105E400011F004060BD1D0F80011FF2900F0F48105
:105E50004A1C2A23C4F80021635484F80431BDE8A5
:105E6000F08790F80431282B0BD0D0F80011FF29CF
:105E700000F0D4814A1C2023C4F80021635484F824
:105E800004317D4FAA6831462046FCF7A9FE07F190
:105E90000208D4F800113A2500260AE00B46013129
:105EA0004745C4F80011E55484F80451D7D017F8D9
:105EB000015FFF29F2D1D4E9423284F8FF60204625
:105EC0009847D4F828310133C4F828310121002340
:105ED000E6E7D0F80011FF2900F080814A1C262354
:105EE000C4F80021635484F80431BDE8F087D0F889
:105EF0000011624E262506F1010800270AE00B4634
:105F00000131B045C4F80011E55484F80451A6D01D
:105F100016F8015FFF29F2D1D4E9423284F8FF700C
:105F200020469847D4F828310133C4F8283101219C
:105F30000023E6E7524ED0F8001106F1070863256A
:105F400000270AE00B4601314645C4F80011E5542C
:105F500084F8045183D016F8015FFF29F2D1D4E907
:105F6000423284F8FF7020469847D4F82831013334
:105F7000C4F8283101210023E6E7424ED0F8001191
:105F800006F10908692500270BE00B460131B045F1
:105F9000C4F80011E55484F804513FF460AF16F8DA
:105FA000015FFF29F1D1D4E9423284F8FF70204625
:105FB0009847D4F828310133C4F82831012100234F
:105FC000E5E7314ED0F8001106F110082025002732
:105FD0000BE00B460131B045C4F80011E55484F8DC
:105FE00004513FF43CAF16F8015FFF29F1D1D4E929
:105FF000423284F8FF7020469847D4F828310133A4
:10600000C4F8283101210023E5E7DFF88080D0F8CB
:10601000003108F1080A20274FF000090AE01A466B
:106020000133D045C4F80031A75484F8047172D00C
:1060300018F8017FFF2BF2D1194684F8FF90D4E9BC
:10604000423220469847D4F828310133C4F8283129
:1060500000220123E5E7DFF83880D0F8003108F1AD
:10606000050A20274FF000091FE000BF643E020828
:10607000703E02087C3E0208C83E0208AC3E0208A0
:10608000B03E0208BC3E0208843E0208983E020868
:10609000A43E02081A460133C245C4F80031A75491
:1060A00084F8047137D018F8017FFF2BF2D119461C
:1060B00084F8FF90D4E9423220469847D4F828313A
:1060C0000133C4F8283100220123E5E7DFF8848199
:1060D000D0F8001108F1090A20274FF000090AE062
:1060E0000A460131C245C4F80011A75484F804716E
:1060F0002FD018F8017FFF29F2D1D4E9423284F879
:10610000FF9020469847D4F828310133C4F828314D
:1061100001210022E6E7EA68002A3FF4A0AEFF2B47
:106120006BD0591C2825C4F800112046E55431468F
:1061300084F80451FCF754FDD4F80011FF2911D064
:106140004A1C2923C4F80021635484F80431BDE8B3
:10615000F0873146AA682046FCF742FDD4F80011CA
:10616000FF29EDD10025D4E9423284F8FF502046C2
:106170009847D4F8283101332946C4F82831012240
:10618000DFE70027D0E9423280F8FF709847D4F863
:10619000283101333946C4F82831012243E600256D
:1061A000194680F8FF50D0E942329847D4F8283198
:1061B0005A1CC4F828212B46012127E60022194643
:1061C00080F8FF20D0E942329847D4F828312022C5
:1061D0000133C4F82831227001217FE60025D4E97B
:1061E000423284F8FF5020469847D4F828310133D2
:1061F0002946C4F82831012271E60027194684F89F
:10620000FF70D4E9423220469847D4F82831EA6832
:10621000591CC4F828113B46012183E70027D0E927
:10622000423280F8FF709847D4F82831013339465C
:10623000C4F8283101221EE6D0E9423280F8FF601E
:106240009847D4F8283101333146C4F82831012267
:10625000FFE500BFCC3E02082DE9F04704460E469C
:1062600017461D46002B62D09A68002A5FD15A68F3
:1062700010781938122857D8DFE800F00A0A0A56B1
:10628000565656560A8989890A0A565656560A009B
:1062900094F80431202B00F08180D4F80031FF2BDA
:1062A00000F0A080591C2022FF29C4F80011E254FC
:1062B00084F8042176D04B1C4FF02809C4F8003133
:1062C00004F801904FF0000AD4F8148184F8049186
:1062D0002A46C4F814A153463146204600F0ACF8D3
:1062E000D4F80021FF2A00F08E80511C2923FF29B9
:1062F000C4F80011A35484F8043126D1002384F893
:10630000FF302046D4E9423298472823237084F88E
:106310000431D4F828313A68591C0123C4F82811F3
:10632000C4F80031D2B921E01B68002B9CD10023B6
:10633000D4F81481C4F8143131462A46204600F0BE
:106340007BF8D4F80011FF29D8D028224B1CC4F8C0
:106350000031625484F804213A682AB1314620465B
:10636000FCF73EFCD4F80031FF2B2BD05A1C29201F
:10637000C4F800213146E0542A4684F80401012380
:10638000204600F059F8C4F81481BDE8F08794F86D
:10639000043103F0FD02282A7FF47CAFD4F8001109
:1063A000FF2988D14FF00008D4E9423284F8FF80F9
:1063B00020469847D4F828310133C4F828314146A3
:1063C000012379E70027194684F8FF70D4E94232A7
:1063D00020469847D4F828315A1CC4F828213B4657
:1063E0000122C4E70022194684F8FF202046D4E9A0
:1063F00042329847D4F8283120220133C4F828319A
:106400002270012157E7114684F8FFA0D4E94232F7
:106410002046984742F62903238084F80491D4F853
:1064200028313A68591C0223C4F82811C4F80031F5
:10643000002A93D19AE700BF002A00F0BB802DE923
:10644000F04F054689B00F461E4614464FF001082E
:1064500019E0A0F11C03042B12D9E368D5F81091C0
:10646000C4F808802928C5F8103157D02A2860D0F0
:10647000022821D039462846FFF7E8FBC5F81091DD
:106480002468002C47D0D5F81821002A43D1A368EE
:10649000002BF5D162681078002EDED14D28EFD0A8
:1064A000D7D94F380128EBD9E368D5F81091C4F853
:1064B0000880C5F81031DDE70026D5F81481926810
:1064C000C5F8146139462846FCF78AFB17F0040A20
:1064D000C5F814813DD0D5F80011FF295CD04A1CC5
:1064E0002E23C5F800216B5485F804316368DC68FD
:1064F0002378472B5FD04D2BA3F14F02A3F11C0152
:1065000024D021D8042921D9224639462846FCF72F
:1065100067FBC5F8109109B0BDE8F08F23680C3215
:1065200039462846FFF798FEC5F8109109B0BDE836
:10653000F08F236808323946284600F0BDF8C5F8C8
:10654000109109B0BDE8F08F012ADDD8A468237846
:10655000D1E7DFF85881D5F8001108F1010B3A2690
:106560000AE00B460131D845C5F80011EE5485F814
:106570000461BBD018F8016FFF29F2D1D5E942328E
:1065800085F8FFA028469847D5F828310133C5F88B
:10659000283101210023E6E7D5E9423285F8FF6082
:1065A00028469847D5F8283101333146C5F82831B7
:1065B000012295E77047DFF8F880D5F8001108F15F
:1065C0000C0B7B264FF0000A0AE00B460131D84540
:1065D000C5F80011EE5485F8046111D018F8016F68
:1065E000FF29F2D1D5E9423285F8FFA02846984725
:1065F000D5F828310133C5F8283101210023E6E719
:10660000E2682949013201A816F03CFA01A802F01B
:1066100017FD18B301AED5F8001106EB000B4FF0D3
:10662000000A09E00B460131B345C5F8001105F831
:10663000038085F8048113D0FF2916F8018BF1D16E
:10664000D5E9423285F8FFA028469847D5F8283189
:106650000133C5F8283101210023E5E7D5F8001101
:10666000DFF850807D2608F1020B4FF0000A0BE0A6
:106670000B460131C345C5F80011EE5485F804619D
:106680003FF464AF18F8016FFF29F1D1D5E9423228
:1066900085F8FFA028469847D5F828310133C5F87A
:1066A000283101210023E5E7D03B0208BC3B02086A
:1066B000C03B0208D43B02082DE9F84F04460E46C1
:1066C00091466BB11D461A469368002B58D012684C
:1066D000002AF9D1134631462A462046FFF7ACFE80
:1066E000D4F80031FF2B57D02022591CC4F80011D8
:1066F000E25484F80421FF291AD05B224B1CC4F811
:106700000031625484F80421D9F800202AB13146BE
:106710002046FCF765FAD4F80031FF2B20D0591C35
:106720005D22C4F80011E25484F80421BDE8F88F1A
:10673000002384F8FF302046D4E9423298475B2397
:10674000237084F80431D4F82831D9F80020591C7A
:106750000123C4F82811C4F80031002AD7D1DEE79C
:106760000025194684F8FF50D4E942322046984764
:10677000D4F828315A1CC4F828212B460121CFE730
:10678000526812782A2A22D131462A462046FFF73B
:1067900053FED4F80011AEE70022194684F8FF201A
:1067A0002046D4E94232984745F620325B2384F8EC
:1067B00004312280D4F82831D9F80020591C022352
:1067C000C4F82811C4F80031002AA0D1A7E7DFF8E7
:1067D0009880D4F800119B4608F1010A20270BE0AD
:1067E0000B46C24501F10101C4F80011E75484F8D9
:1067F000047117D018F8017FFF29F1D1D4E9423292
:1068000084F8FFB020469847D4F828310133C4F803
:10681000283100230121C245C4F80011E75484F84F
:106820000471E7D131462A4600232046FFF704FED3
:10683000D4F80011FF2907D029224B1CC4F80031DD
:10684000625484F804214DE7002384F8FF30204689
:10685000D4E942329847D4F8283129220133C4F8C8
:106860002831227001233FE7E03D02082DE9F04185
:106870001578322D03D0BDE8F041FCF7B1B993682B
:10688000D3E901565EB32E44D0F800110446013E10
:10689000013D00270AE00B46B54201F10101C4F8B1
:1068A000001104F8038084F8048118D0FF2915F83A
:1068B000018FF0D1D4E9423284F8FF702046984726
:1068C000D4F828310133C4F8283100230121B5421E
:1068D000C4F8001104F8038084F80481E6D1BDE80F
:1068E000F08100BF2DE9F0411378012B15460E46CB
:1068F000044620D9312B1ED0062B1CD0D0F80071B5
:10690000FF2F1FD07A1C2823C4F800213146E355FD
:106910002A46204684F80431FCF762F9D4F80011C5
:10692000FF291FD04A1C2923C4F80021635484F88E
:106930000431BDE8F0812A4631462046BDE8F041E9
:10694000FCF74EB94FF00008D0E94232394680F8E2
:10695000FF809847D4F8283101334746C4F82831DE
:106960000122D0E70025D4E9423284F8FF502046C6
:106970009847D4F8283101332946C4F82831012238
:10698000D1E700BF2DE9F04F926812681578662DA7
:1069900083B07AD11B68D3E9028A9AF800303C2B85
:1069A0004FF0FF3308BFDAE902A90C46D0F82411F2
:1069B000C0F824315378019118BF4FF000096C2BB7
:1069C000074600F0A08064D84C2B01D0522B55D143
:1069D000D7F80011FF2900F0E5804A1C2823C7F8EA
:1069E000002138467B545246214687F80431754DC4
:1069F000FFF778FF214642463846FFF737FF05F19B
:106A0000020BD7F800112E264FF0000A0BE00B46C0
:106A1000AB4501F10101C7F80011FE5487F804618C
:106A200017D015F8016FFF29F1D1D7E9423287F865
:106A3000FFA038469847D7F828310133C7F82831E6
:106A400000230121AB45C7F80011FE5487F804610B
:106A5000E7D1424621463846FFF708FF4A4621461D
:106A60003846FFF73FFFD7F80011FF297DD04A1CB9
:106A70002923C7F800217B5487F80431019BC7F80C
:106A80002431012003B0BDE8F08F002003B0BDE841
:106A9000F08F722BF2D1D0F80011FF2974D04A1C6C
:106AA0002823C7F8002138467B545246214687F8F0
:106AB0000431FFF717FF2146434C42463846FFF7A3
:106AC000D5FE04F10308D7F800112E2500260AE0B0
:106AD0000B4601314445C7F80011FD5487F80451B5
:106AE000CCD014F8015FFF29F2D1D7E9423287F800
:106AF000FF6038469847D7F828310133C7F8283166
:106B000001210023E6E7314DD0F8001105F1030B18
:106B100028264FF000090BE00B46AB4501F10101BF
:106B2000C7F80011FE5487F8046117D015F8016FFB
:106B3000FF29F1D1D7E9423287F8FF9038469847CC
:106B4000D7F828310133C7F8283100230121AB459C
:106B5000C7F80011FE5487F80461E7D14246214688
:106B60003846FFF783FE524679E70024D7E94232E0
:106B700087F8FF4038469847D7F828310133214637
:106B8000C7F82831012273E70025D0E9423280F8A6
:106B9000FF509847D7F8283101332946C7F82831E4
:106BA00001227DE70025D7E9423287F8FF503846B9
:106BB0009847D7F8283101332946C7F828310122F0
:106BC0000CE700BFE43D0208E03E0208D83E0208A0
:106BD0002DE9F04FE5B090F80090B9F15F0F00AFEC
:106BE00004468846164600F0F280C4490822204632
:106BF00015F0C8FF48B9237A2E2B00F0D7805F2B01
:106C000000F0D480242B00F0D1804FF0000A204601
:106C100002F016FA22184FEA400B1123FA60BBF576
:106C2000006F4FF00002C7E90434C7E9072BC7E93A
:106C30000C22C7E90E22F862BC60BA623A6400F224
:106C4000AF806D468100A5EB4013073121F00701AD
:106C50009D46ADEB010DBAF1010FC7F824D0BB6121
:106C600000F0C980AAF10201012900F2CA80E17A8C
:106C7000BAF1020F08BF4FF0440904F10B0A18BF24
:106C80004FF045095F29C7F814A000F0A7805046CF
:106C90007B6002F0D5F9BBF1000F7B6840F31A81ED
:106CA000002201215A60F961002800F01381C3E934
:106CB00002A01A701A464946002307F10800F9F7A6
:106CC0003FFB7C698146204602F0BAF923187B61BC
:106CD000235C002B40F09280B9F1000F00F08E8011
:106CE00007F1440420464946C4E94433C4E9493322
:106CF000C4E94633C4E94B33C4E94D33C4E94F33E7
:106D00007B60C4F8003184F80431C4F82031C4F841
:106D10004431C4F80881C4F80C61F9F777FBD4F862
:106D20001C21B2F5006FD4F83821BCBF7B68C4F8D1
:106D30001C31D4F84431012A1046E846B8BF01207E
:106D400003FB02F3A8EBC002012B9546EC46194663
:106D5000B8BF0121ACEBC1018D464A460026112186
:106D60002046C4F84431C4F830C1C4F83CD1C4F85A
:106D70004861FBF735FFD4F80011D4F808316654A8
:106D8000C5462046D4F80C219847D4F81801B0FA2B
:106D900080F04009AD4607F5CA77BD46BDE8F08FE3
:106DA000104607F5CA77BD46BDE8F08F637A442BDD
:106DB00002D0492B7FF429AFA27A5F2A7FF425AF56
:106DC000492B0CBF4FF0020A4FF0030A1FE743782C
:106DD0005A2B7FF40AAF4FF0010A18E7217B5A299A
:106DE0007FF455AF0D34114607F108007C61FAF7C6
:106DF00047FB03465EE7B9F15F0F0AD00020AD46BE
:106E0000C9E707F10800FAF767FF7B6981461B783D
:106E10005FE763785A2BF1D10234514607F108003D
:106E20007C61FAF72DFB3B6913F0010F81464FF0AF
:106E300000025FD0D7F814C09CF800302E2B7FF4EE
:106E400048AF14469CF80130A3F16102192A45D9D4
:106E50005F2B43D0303B092B4CD89CF80010634685
:106E60002E2912D15A78303A092A0ED89A78A2F1EE
:106E70003001092903F1020305D813F8012FA2F10B
:106E800030010929F9D92E2AECD0D7E90701884227
:106E90007B61A3EB0C021FDAB96901EB001300F16F
:106EA000010E002A5C604FEA0010C7F81CE013DDF9
:106EB0005C600C54C3E902C24A464E2107F1080047
:106EC000F9F73EFAD7F814C09CF800302E2B814613
:106ED000B8D0FEE60023EDE60023EDE70CF1020258
:106EE000134612F8011BA1F161001928F8D95F2996
:106EF000F6D0B5E77B691B78EBE600BF643B020880
:106F00002DE9F0411E4684B0002840D00C461546BD
:106F100009B1002A3BD0002329496A46CDE9003354
:106F2000CDE90233FFF754FE002839D0039B009FC0
:106F3000D3B9DDF80880002F3CD02CB3384602F0DE
:106F40007FF82B68984219D2421C3946204601F03E
:106F50004FFE384614F04CFF27460EB10023336035
:106F6000384604B0BDE8F0814FF00108002FE4D1AD
:106F70008EB14FF0FF3333600027F1E7204614F065
:106F800037FFC5F80080E8E7002DFAD1E5E716B134
:106F90006FF0020333600027384604B0BDE8F0818B
:106FA000009814F025FF002EF5D06FF00103336038
:106FB0000027D5E7002EEED0B8F1010FD9D0F4E7C5
:106FC000510A000860B108B539B1FFF701FE002889
:106FD00014BF00206FF0010008BD6FF0020008BD73
:106FE0006FF00200704700BF81F0004102E000BF77
:106FF00083F0004330B54FEA41044FEA430594EA79
:10700000050F08BF90EA020F1FBF54EA000C55EAB3
:10701000020C7FEA645C7FEA655C00F0E2804FEA84
:107020005454D4EB5555B8BF6D420CDD2C4480EA66
:10703000020281EA030382EA000083EA010180EA96
:10704000020281EA0303362D88BF30BD11F0004FE4
:107050004FEA01314FF4801C4CEA113102D040421A
:1070600061EB410113F0004F4FEA03334CEA133355
:1070700002D0524263EB430394EA050F00F0A7806D
:10708000A4F10104D5F1200E0DDB02FA0EFC22FA68
:1070900005F2801841F1000103FA0EF2801843FA5C
:1070A00005F359410EE0A5F120050EF1200E012A4D
:1070B00003FA0EFC28BF4CF0020C43FA05F3C0188B
:1070C00051EBE37101F0004507D54FF0000EDCF104
:1070D000000C7EEB00006EEB0101B1F5801F1BD3AD
:1070E000B1F5001F0CD349085FEA30004FEA3C0CB1
:1070F00004F101044FEA445212F5800F80F09A80A7
:10710000BCF1004F08BF5FEA500C50F1000041EBAA
:10711000045141EA050130BD5FEA4C0C404141EBAE
:107120000101013C28BFB1F5801FE9D291F0000FA9
:1071300004BF01460020B1FA81F308BF2033A3F158
:107140000B03B3F120020CDA0C3208DD02F1140C4F
:10715000C2F10C0201FA0CF021FA02F10CE002F18A
:107160001402D8BFC2F1200C01FA02F120FA0CFC83
:10717000DCBF41EA0C019040E41AA2BF01EB0451CC
:10718000294330BD6FEA04041F3C1CDA0C340EDCCA
:1071900004F11404C4F1200220FA04F001FA02F30D
:1071A00040EA030021FA04F345EA030130BDC4F1CB
:1071B0000C04C4F1200220FA02F001FA04F340EAC0
:1071C0000300294630BD21FA04F0294630BD94F071
:1071D000000F83F4801306BF81F480110134013D58
:1071E0004EE77FEA645C18BF7FEA655C29D094EAC9
:1071F000050F08BF90EA020F05D054EA000C04BF47
:107200001946104630BD91EA030F1EBF0021002031
:1072100030BD5FEA545C05D14000494128BF41F0D0
:10722000004130BD14F580043CBF01F5801130BD34
:1072300001F0004545F0FE4141F470014FF00000BF
:1072400030BD7FEA645C1ABF194610467FEA655C70
:107250001CBF0B46024650EA013406BF52EA033512
:1072600091EA030F41F4002130BD00BF90F0000F00
:1072700004BF0021704730B54FF4806404F132043C
:107280004FF000054FF0000150E700BF90F0000FF5
:1072900004BF0021704730B54FF4806404F132041C
:1072A00010F0004548BF40424FF000013EE700BFEC
:1072B00042004FEAE2014FEA31014FEA02701FBF7C
:1072C00012F07F4393F07F4F81F06051704732F0AE
:1072D0007F4208BF704793F07F4F04BF41F4002105
:1072E000704730B54FF4607401F0004521F0004163
:1072F0001CE700BF50EA010208BF704730B54FF0ED
:1073000000050AE050EA010208BF704730B511F0ED
:10731000004502D5404261EB41014FF4806404F125
:1073200032045FEA915C3FF4D8AE4FF003025FEAAB
:10733000DC0C18BF03325FEADC0C18BF033202EB2F
:10734000DC02C2F1200300FA03FC20FA02F001FA89
:1073500003FE40EA0E0021FA02F11444BDE600BF2C
:1073600070B54FF0FF0C4CF4E06C1CEA11541DBFDB
:107370001CEA135594EA0C0F95EA0C0F00F0DEF8A6
:107380002C4481EA030621EA4C5123EA4C5350EA8B
:10739000013518BF52EA033541F4801143F48013DC
:1073A00038D0A0FB02CE4FF00005E1FB02E506F06D
:1073B0000042E0FB03E54FF00006E1FB03569CF0C2
:1073C000000F18BF4EF0010EA4F1FF04B6F5007FC8
:1073D00064F5407404D25FEA4E0E6D4146EB06063A
:1073E00042EAC62141EA55514FEAC52040EA5E50C3
:1073F0004FEACE2EB4F1FD0C88BFBCF5E06F1ED86D
:10740000BEF1004F08BF5FEA500E50F1000041EBA3
:10741000045170BD06F0004646EA010140EA020050
:1074200081EA0301B4EB5C04C2BFD4EB0C0541EA72
:10743000045170BD41F480114FF0000E013C00F387
:10744000AB8014F1360FDEBF002001F0004170BDAB
:10745000C4F10004203C35DA0C341BDC04F11404C4
:10746000C4F1200500FA05F320FA04F001FA05F250
:1074700040EA020001F0004221F0004110EBD3701D
:1074800021FA04F642EB06015EEA430E08BF20EA49
:10749000D37070BDC4F10C04C4F1200500FA04F3EC
:1074A00020FA05F001FA04F240EA020001F000417E
:1074B00010EBD37041F100015EEA430E08BF20EAF1
:1074C000D37070BDC4F1200500FA05F24EEA020E39
:1074D00020FA04F301FA05F243EA020321FA04F068
:1074E00001F0004121FA04F220EA020000EBD3701F
:1074F0005EEA430E08BF20EAD37070BD94F0000F1F
:107500000FD101F00046400041EB010111F4801F52
:1075100008BF013CF7D041EA060195F0000F18BF03
:10752000704703F00046520043EB030313F4801F3F
:1075300008BF013DF7D043EA0603704794EA0C0FF9
:107540000CEA135518BF95EA0C0F0CD050EA41060F
:1075500018BF52EA4306D1D181EA030101F000418C
:107560004FF0000070BD50EA410606BF10461946B4
:1075700052EA430619D094EA0C0F02D150EA0136C0
:1075800013D195EA0C0F05D152EA03361CBF104601
:1075900019460AD181EA030101F0004141F0FE41A0
:1075A00041F470014FF0000070BD41F0FE4141F424
:1075B000780170BD70B54FF0FF0C4CF4E06C1CEA24
:1075C00011541DBF1CEA135594EA0C0F95EA0C0FD9
:1075D00000F0A7F8A4EB050481EA030E52EA033594
:1075E0004FEA013100F088804FEA03334FF08055B5
:1075F00045EA131343EA12634FEA022245EA1115E2
:1076000045EA10654FEA00260EF000419D4208BF92
:10761000964244F1FD0404F5407402D25B084FEA3F
:107620003202B61A65EB03055B084FEA32024FF4EB
:1076300080104FF4002CB6EB020E75EB030E22BF48
:10764000B61A754640EA0C005B084FEA3202B6EB08
:10765000020E75EB030E22BFB61A754640EA5C00B7
:107660005B084FEA3202B6EB020E75EB030E22BF47
:10767000B61A754640EA9C005B084FEA3202B6EB48
:10768000020E75EB030E22BFB61A754640EADC0007
:1076900055EA060E18D04FEA051545EA16754FEA69
:1076A00006164FEAC30343EA52734FEAC2025FEA87
:1076B0001C1CC0D111F4801F0BD141EA00014FF016
:1076C00000004FF0004CB6E711F4801F04BF0143E7
:1076D0000020B4F1FD0C88BFBCF5E06F3FF6AFAE03
:1076E000B5EB030C04BFB6EB020C5FEA500C50F193
:1076F000000041EB045170BD0EF0004E4EEA113116
:1077000014EB5C04C2BFD4EB0C0541EA045170BD1C
:1077100041F480114FF0000E013C90E645EA060E60
:107720008DE60CEA135594EA0C0F08BF95EA0C0F8E
:107730003FF43BAF94EA0C0F0AD150EA01347FF4D6
:1077400034AF95EA0C0F7FF425AF104619462CE7AD
:1077500095EA0C0F06D152EA03353FF4FDAE104610
:10776000194622E750EA410618BF52EA43067FF461
:10777000C5AE50EA41047FF40DAF52EA43057FF4F1
:10778000EBAE12E74FF0FF3C06E000BF4FF0010CFC
:1077900002E000BF4FF0010C4DF804CD4FEA410C60
:1077A0007FEA6C5C4FEA430C18BF7FEA6C5C1BD02D
:1077B00001B050EA410C0CBF52EA430C91EA030FAE
:1077C00002BF90EA020F0020704710F1000F91EA0B
:1077D000030F58BF994208BF90422CBFD8176FEAD9
:1077E000E37040F0010070474FEA410C7FEA6C5CA7
:1077F00002D150EA013C07D14FEA430C7FEA6C5CAE
:10780000D6D152EA033CD3D05DF8040B704700BFD9
:107810008446104662468C461946634600E000BF27
:1078200001B5FFF7B7FF002848BF10F1000F01BDF9
:107830004DF808EDFFF7F4FF0CBF012000205DF8C4
:1078400008FB00BF4DF808EDFFF7EAFF34BF012049
:1078500000205DF808FB00BF4DF808EDFFF7E0FFE2
:1078600094BF012000205DF808FB00BF4DF808ED33
:10787000FFF7CEFF94BF012000205DF808FB00BF9A
:107880004DF808EDFFF7C4FF34BF012000205DF87C
:1078900008FB00BF4FEA410C7FEA6C5C02D150EA62
:1078A000013C0AD14FEA430C7FEA6C5C02D152EAF8
:1078B000033C02D14FF0000070474FF001007047C9
:1078C0004FEA410212F5001215D211D56FF4787308
:1078D000B3EB625212D94FEAC12343F0004343EAAB
:1078E000505311F0004F23FA02F018BF4042704786
:1078F0004FF00000704750EA013005D111F0004010
:1079000008BF6FF0004070474FF00000704700BFA5
:107910004FEA4102B2F1E04324BFB3F5001CDCF1B1
:10792000FE5C0DD901F0004C4FEAC0024CEA5070E9
:10793000B2F1004F40EB830008BF20F00100704718
:1079400011F0804F21D113F13872BCBF01F000401B
:10795000704741F480114FEA5252C2F11802C2F14D
:10796000200C10FA0CF320FA02F018BF40F00100CE
:107970004FEAC1234FEAD32303FA0CFC40EA0C0080
:1079800023FA02F34FEA4303CCE77FEA625307D1BD
:1079900050EA01331EBF4FF0FE4040F440007047F4
:1079A00001F0004040F0FE4040F40000704700BF8E
:1079B00053B94AB9002908BF00281CBF4FF0FF3156
:1079C0004FF0FF3001F0C0B8ADF1080C6DE904CE06
:1079D00000F006F8DDF804E0DDE9022304B07047AA
:1079E0002DE9F047089D04468C46002B40F083802B
:1079F0008A42174647D9B2FA82F242B1C2F1200058
:107A000024FA00F09140974040EA010C94404FEA7C
:107A10001748230CBCFBF8F61FFA87FE08FB16C1BB
:107A200043EA014306FB0EF1994209D9FB1806F11E
:107A3000FF3080F01981994240F21681023E3B44AA
:107A40005B1AA4B2B3FBF8F008FB103344EA03441A
:107A500000FB0EFEA64509D93C1900F1FF3380F06A
:107A60000581A64540F2028102383C4440EA0640C6
:107A7000A4EB0E0400261DB1D4400023C5E9004349
:107A80003146BDE8F08702B9FFDEB2FA82F2002A81
:107A900050D1CB1B4FEA174E1FFA87F80126B3FBD4
:107AA000FEFC210C0EFB1C3341EA034108FB0CF3E6
:107AB0008B4207D979180CF1FF3002D28B4200F2C9
:107AC000E9808446C91AA3B2B1FBFEF00EFB101187
:107AD00043EA014408FB00F8A04507D93C1900F12E
:107AE000FF3302D2A04500F2D9801846A4EB080467
:107AF00040EA0C40BFE78B4209D9002D00F0B1806D
:107B00000026C5E9000130463146BDE8F087B3FAEA
:107B100083F6002E4AD18B4202D3824200F2B88013
:107B2000841A61EB030101208C46002DA8D0C5E921
:107B3000004CA5E7C2F1200320FA03F6974001FAB2
:107B400002F04FEA174ED9403043030CB1FBFEF66A
:107B50001FFA87F80EFB161143EA014306FB08F1F2
:107B6000994204FA02F409D9FB1806F1FF3C80F0AF
:107B70008D80994240F28A80023E3B445B1A81B27A
:107B8000B3FBFEF00EFB103341EA034100FB08F3A8
:107B90008B4207D9791800F1FF3C73D28B4271D91F
:107BA00002383944CB1A40EA064678E7C6F1200C81
:107BB00003FA06F422FA0CF31C4320FA0CF701FA3C
:107BC00006F34FEA144E21FA0CF11F433B0CB1FBB4
:107BD000FEF91FFA84F80EFB191143EA014109FB73
:107BE00008FA8A4502FA06F200FA06F308D9611883
:107BF00009F1FF3048D28A4546D9A9F1020921444A
:107C0000A1EB0A01BFB2B1FBFEF00EFB101147EA77
:107C1000014700FB08F8B84507D9E71900F1FF3123
:107C20002ED2B8452CD90238274440EA0940A7EBA8
:107C30000807A0FB02894F45C64649461AD317D00C
:107C40005DB1B3EB0E0267EB010707FA0CFCF240E3
:107C50004CEA0202F740C5E9002700263146BDE89C
:107C6000F0872E4628460BE70646E9E61846FDE66D
:107C70004345E5D2B8EB020E69EB04010138DFE7BA
:107C80000846D2E760468DE78146B9E7664675E764
:107C900030464AE7ACF1020C394413E702383C4461
:107CA00024E700BF03685A004CBF43F0004323F0B1
:107CB00000431844704700BF2DE9F84329B34F1E15
:107CC000044615463E464FF0000808EB060101EB5E
:107CD000D171491004EBC1094846FFF7E3FF0346A1
:107CE000C80008308F42204409D0AB4209D8FFF7C2
:107CF000D9FF0138A8420AD201F10108E5E7AB42F9
:107D000005D9884501D04E1EDFE74FF000094846EF
:107D1000BDE8F883012807D0022807D0044B0028CB
:107D20000CBF184600207047024870470248704751
:107D3000D9830008DD830008E183000830B5234BB8
:107D400083B004468D1E3BB301A92846AFF30080E3
:107D5000E8B101992A46FFF7AFFF0146B8B1FFF736
:107D6000A1FF4B68A064012B2BD0002B01F1040074
:107D700023DBFFF797FF0023C4E913030368002BFD
:107D800010DBFFF78FFF2061002003B030BD002320
:107D90000920236103B030BD0D490E48091AC910EE
:107DA0000191D7E7C3F30360FFF7B4FF0028206118
:107DB00014BF0020092003B030BD0123C4E9130320
:107DC000DCE7002323610520DFE700BF000000009F
:107DD000C84A0208304902080368DA0710B50446A9
:107DE00006D49B0700F1480009D500F04BFC23683E
:107DF000590709D51A070ED5DB0613D510BD00F0BB
:107E000039FC23685907F5D404F1D00000F042FC96
:107E100023681A07F0D404F5A87000F043FC236827
:107E2000DB06EBD404F5E870BDE8104000F07EBC42
:107E30000346006800B11844704700BF092070472E
:107E4000704700BF70B504460E46316C2046FFF700
:107E500075FF054688B9336C636132462369214654
:107E6000012098470828F0D0072806D12846316C11
:107E7000FFF7E6FF301D00F0F1FB13F01BFD00BF24
:107E80002DE9F0470D1D064614460FCDADF5727D68
:107E90000DF10C0CACE80F000FCDACE80F000FCDCE
:107EA000ACE80F0095E80F0002ADF768D6F818802F
:107EB0008CE80F0000232B6021E02B6C73614FF4E2
:107EC000F07229467AA800F093FE33697AAA314607
:107ED00050469847889BCDE9005821466B648146FF
:107EE000334632460120B8470446E8B94FF4F072F1
:107EF0007AA9284600F07CFEB9F1080F1BD1296C45
:107F00003046FFF71BFF09345FFA84FA81460028E8
:107F1000D3D0AB6B4AF01001CDE9005832466B6408
:107F200001203346B84708B14FF0090948460DF51E
:107F3000727DBDE8F087B9F1070FF5D12046296CB5
:107F4000FFF77EFF03A800F089FB00BF406C70477D
:107F5000F0B5CB6B0B640E1D0F4605460FCEF9B086
:107F600001AC0FC40FCE0FC40FCE0FC496E80F00A4
:107F70004FF0FF3684E80F00009606E02B696A4652
:107F8000294698470828044608D110992846FFF743
:107F9000D5FE0028F2D0092079B0F0BD6846FFF781
:107FA0001BFF062CF7D139462846FFF74BFF00BFD1
:107FB00030B4DD6BC160826119461D64002230BCA3
:107FC0005EE700BF70B5C66843690B64AEB903696C
:107FD0000A4604460D46014602209847072805D068
:107FE00008280FD129462046FFF72CFF3046296C80
:107FF000FFF726FF281D00F031FB0122FFF740FFAD
:1080000013F058FC13F056FCC2681AB1CA6B0A642C
:10801000002235E79CE700BF704700BF8368014638
:108020000BB1012018477047012912D009D873B944
:108030000F2A0CD800EB820218465368009A13608E
:1080400070470339012994BF0120022070470220A4
:1080500070470846704700BF10B584B0002303ACDA
:108060000A4600941946FFF7DFFF039804B010BDDD
:10807000012912D009D873B90F2A0CD800EB82005D
:10808000009A12684260184670470339012994BF6C
:10809000012002207047022070470846704700BF49
:1080A00010B584B0002303AC039200940A4619462D
:1080B000FFF7DEFF04B010BDF0B5D36B1364151DE0
:1080C0008C4606460FCDADF50F7D17AC0FC40FCD16
:1080D0000FC40FCD0FC495E80F004FF0FF3784E8B1
:1080E0000F006546169710E0FFF7DAFF294616A83D
:1080F000B047034616AA6946082083B9049B9847EF
:10810000052804460CD0092809D026996846FFF7AF
:1081100015FE03466A460C2116A8002BE4D009245C
:1081200016A8FFF759FE20460DF50F7DF0BD00BFE4
:108130002DE9F04FCC6C89B00D4654F8041B069421
:10814000174600F003081E46002B79D00B0CDAB25C
:1081500009048DF81D30022304EB820405918DF88B
:108160001C302B6DB8F1020F08BFAC6B13F001038C
:108170000CD0384605A900F073FB18B9082009B0E7
:10818000BDE8F08F092009B0BDE8F08FD4F800A059
:10819000BAF1000FEDD0019300F008030293022E14
:1081A0004AD0B4F800A0B4F802900434AA6C29F0C4
:1081B000010B0F2138469344FFF74EFF834539D812
:1081C0002AF001025A44824294BF002001204FEA63
:1081D000490303F002030AF0010A43EA0A03012BF0
:1081E00049D0022B32D0002BCCD1B8F1000F02D0F5
:1081F000002840F0CD800434D4F800A0BAF1000F7C
:10820000CDD105A9384600F02BFB0028BAD1019B3F
:10821000002BB3D00F213846FFF71EFF0E21024678
:108220003846FFF73DFF38466A4A0F21FFF738FF0F
:108230000720A8E70020CAE7D4F804900834B5E77F
:10824000090203230591ADF81C308AE7236823F067
:10825000004BB8F1000F45D128B1029A002A5CD03A
:10826000BBF1000F74D0002B00DA04340BF1010BCA
:1082700004EB8B04C0E7B8F1000F19D1B0B1D4E919
:108280000023991C4FEAD2723FF47CAF05F15801EC
:108290000133049100F09080201DFFF7C9FD04AB6D
:1082A0000146284611F09EFF00285BD10834A3E761
:1082B0000D213846D5F82090FFF7CEFE8145F5D147
:1082C000AB6A9C42F2D12046FFF7ECFC0F2102463C
:1082D0003846FFF7E5FE38462A460021FFF7E0FE64
:1082E000072050E70D213846D5F82090FFF7B4FE5F
:1082F000814501D02368B6E7AB6A9C42FAD10422DB
:108300000021C5E90B12A318C5F828B06B632368D8
:108310008B4259DB01230193A8E705F15803CDF8FF
:108320000C8004F1040AB04691461E460DE0049606
:10833000FFF77EFD04AB01460022284611F052FFF4
:1083400009F101090AF1040AE8B9D9455046EED10C
:1083500038460D21FFF780FE049B2862C5E90934E9
:10836000062010E781460D213846FFF775FEB9F16A
:10837000020F286225D12B46049A43F82C2F6B62FA
:10838000AC620620FFE646462368DDF80C806AE70B
:108390002046FFF787FC04340246AC6328461446A7
:1083A00011F080FF00283FF4EDAE384622460F2141
:1083B000FFF776FE0720E6E638460D21FFF74CFE74
:1083C0002862049B6B62DBE70BF1010004EB800089
:1083D0007AE700BF25AE01080023A9E60123A7E63E
:1083E0000223A5E62DE9F0430646C3B015461C4618
:1083F000042900F2B980DFE801F09A53B72903009D
:10840000002C40F0B180102A00F2AE800368D8063C
:1084100000F1F38020AF384600F092F9B06B0023F2
:10842000012404FA03F22A42014604D051F8042B35
:1084300047F8232008460133042BF2D1B0633846B5
:1084400000F074F9002043B0BDE8F083032C40F045
:108450008B8094B204EB1243102B4FEA124500F2CA
:10846000838003681F0700F1D08020AF384600F0FA
:108470003BF907EBC501B56B54B10B46E81A01EBAC
:10848000C401E4001A5843F8042B8B42FAD1254466
:108490003846B56300F006F9002043B0BDE8F0832C
:1084A000012C4FEA124895B25AD0052C5CD108EB4A
:1084B0000509B9F1200F57D8B8F10F0F77D9A946A0
:1084C000002D40F08880B36B6DB320AF4FF00009F2
:1084D00007EBC807043F03EBC50553F8041B47F837
:1084E000041FAB42F9D1B9F1000F0FD06F464146DE
:1084F000102938BF102107EBC101843903EBC905EE
:1085000053F8040B41F8040FAB42F9D1012C00F0F1
:108510008480B8F10F0FB56345D9B9F1000F02D0CF
:10852000684600F0B7F8002043B0BDE8F083DCB93E
:10853000876B2346012094B206F1040C00FA03F283
:108540002242394604D051F8042B4CF823200F4620
:108550000133102BF2D115F40050E4D1B76304E0DD
:1085600008EB0503102B03D9022043B0BDE8F083CC
:10857000B8F10F0FF8D83368DA0706D5304623F084
:10858000030340F8483B00F079F820AF384600F08C
:1085900075F8B36B002D99D11D460435B563384687
:1085A00000F068F8BFE720A800F06CF8B5E7B9F173
:1085B000100F40D9A9F110093368D90708D523F065
:1085C0000103304643F0020340F8483B00F05EF8F8
:1085D000B9F1000F32D033685A0720D4B8F10F0F29
:1085E00025D96F463846C8F1100500F057F8002D20
:1085F000B36B7FF77CAF20AF6AE723F010033360E3
:1086000006F5E87000F09CF804E723F00803036027
:1086100000F5A87000F068F827E720AFBDE7304606
:1086200023F0040340F8D03B00F038F8D6E720A848
:1086300000F02CF8D5E74FF00009BDE7B8F10F0FB7
:108640003FF641AF20AF384600F020F8B36B002D65
:108650007FF43CAF384600F015F864E700F13401D0
:1086600091E838009C46A6464CF8045D90E8FF0F60
:10867000E54600BD90EC210B704700BF80EC210B5C
:10868000704700BF90EC200B704700BF80EC200BC0
:10869000704700BFD0EC200B704700BFC0EC200B30
:1086A000704700BFF0EC0201F0EC0211F0EC022187
:1086B000F0EC0231F0EC0241F0EC0251F0EC02611E
:1086C000F0EC0271F0EC0281F0EC0291F0EC02A10E
:1086D000F0EC02B1F0EC02C1F0EC02D1F0EC02E1FE
:1086E000F0EC02F1704700BFE0EC0201E0EC021197
:1086F000E0EC0221E0EC0231E0EC0241E0EC02515E
:10870000E0EC0261E0EC0271E0EC0281E0EC02914D
:10871000E0EC02A1E0EC02B1E0EC02C1E0EC02D13D
:10872000E0EC02E1E0EC02F1704700BFB0FC018137
:10873000B0FC0191B0FC01A1B0FC01B1704700BFD9
:10874000A0FC0181A0FC0191A0FC01A1A0FC01B151
:10875000704700BFEC4600B52DE900502DE9FF1F22
:108760004FF000032DE90C0001A9FFF7F1FBDDF844
:1087700040E012B0704700BFEC4600B52DE9005054
:108780002DE9FF1F4FF000032DE90C0001A9FFF7B1
:1087900019FCDDF840E012B0704700BFEC4600B5B0
:1087A0002DE900502DE9FF1F4FF000032DE90C00CB
:1087B00001A9FFF729FCDDF840E012B0704700BFC7
:1087C000EC4600B52DE900502DE9FF1F4FF00003E6
:1087D0002DE90C0001ABFFF7EBFBDDF840E012B038
:1087E000704700BFEC4600B52DE900502DE9FF1F92
:1087F0004FF000032DE90C0001AAFFF75DFCDDF846
:1088000040E012B0704700BF027A7AB9437AA3B150
:108810004268013B10B4437213680321141D0172B6
:108820001A024460026010BC180E70470368013AD7
:1088300002721A020260180E7047B020704700BF23
:1088400000B585B003AA0023009219460C22FFF759
:10885000EBFB039805B05DF804FB00BFF0E700BF39
:108860002DE9F043054685B00E464FF0000830462E
:10887000FFF7CAFFB028044600F0B280070620D5F3
:1088800000F0F003802B4DD0902B36D0A02B60D081
:10889000B02B74D0C02B00F08B8000F0F803D02BED
:1088A0000BD100F00702013242F40022052301211E
:1088B0002846FFF797FD0028D9D0092005B0BDE86C
:1088C000F0830DF10C09002319468700CDF80090C4
:1088D0000D222846FFF7A8FBFFB2039BCDF80090BE
:1088E000043760064CBFDF1BFF18002319460D221A
:1088F00028460397FFF7BCFBB9E700F00D030D2BEB
:10890000DBD003AF002300F00F0219460097284682
:10891000FFF78AFB0023009719460D222846FFF730
:10892000A7FBA4E73046FFF76FFF24022043B0F512
:10893000004FC2D004010023A2B219462846FFF717
:1089400051FD0028B9D114F4004F18BF4FF00108B1
:108950008DE7C24302F007034FF47F621A4101071B
:1089600002F47F624FF0000348BF42F48042194690
:108970002846FFF737FD00283FF479AF9DE7B1287F
:1089800033D0B22800F08B80B32839D000F0FC033C
:10899000B42B92D000F007020132012342F40022EE
:1089A00019462846FFF71EFD00283FF460AF84E714
:1089B000C62842D0C7284CD000F0F803C02B5BD0AB
:1089C000C82860D0C9287FF478AF3046FFF71CFF75
:1089D000020300F00F0002F470220130024365E749
:1089E000B8F1000F18D0002068E73046FFF70CFF01
:1089F000024600283FF461AF10F0F003D0D05CE7EE
:108A00003046FFF701FF010300F00F0001F4702171
:108A1000421C01230A43C3E703AC43460E224146EE
:108A200000942846FFF700FB0094284643460F2297
:108A30004146FFF71DFB404640E73046FFF7E4FEA6
:108A4000010300F00F0001F47021421C03230A43CC
:108A5000A6E73046FFF7D8FE024600283FF42DAFC8
:108A600010F0F0037FF429AF04212846FFF7BAFC89
:108A700000283FF4FCAE20E700F00F020132032390
:108A800042F420228CE73046FFF7BEFE00F0F002F1
:108A900000F00F031032013343EA023206E70023ED
:108AA0000DF10C090D221946CDF800902846FFF76C
:108AB000BBFA3046FFF7A8FE02064FF002070CD5BE
:108AC000039B00F07F00B840034430460393FFF758
:108AD0009BFE030607F10707F2D4039BCDF8009035
:108AE00000F07F0403F50172BC40002314441946D2
:108AF0000D2228460394FFF7BBFAB8E610B5C26C06
:108B000084B0536803248DF80C401B0202F1080462
:108B10000846D279019301A902948DF80D20FFF740
:108B20009FFE04B010BD00BF08B5FFF797FE806C34
:108B300008BD00BF08B5FFF791FEC06CC3790233D2
:108B400000EB830008BD00BF704700BF00000000BD
:108B500001F0FF01102A2BDB10F0070F08D010F8EE
:108B6000013B013A8B422DD010F0070F42B3F6D1F2
:108B7000F0B441EA012141EA014122F007047FF00B
:108B800000070023F0E80256083C85EA010586EA62
:108B9000010685FA47F5A3FA87F586FA47F6A5FA9E
:108BA00087F68EB9EED1F0BC01F0FF0102F00702AA
:108BB00032B110F8013B013A83EA010313B1F8D155
:108BC0000020704701387047002D06BF3546033836
:108BD000073815F0010F07D1013015F4807F02BF6F
:108BE000013015F4C03F0130F0BC0138704700BFC0
:108BF000844641EA000313F003036DD1403A41D3A8
:108C000051F8043B40F8043B51F8043B40F8043B66
:108C100051F8043B40F8043B51F8043B40F8043B56
:108C200051F8043B40F8043B51F8043B40F8043B46
:108C300051F8043B40F8043B51F8043B40F8043B36
:108C400051F8043B40F8043B51F8043B40F8043B26
:108C500051F8043B40F8043B51F8043B40F8043B16
:108C600051F8043B40F8043B51F8043B40F8043B06
:108C700051F8043B40F8043B51F8043B40F8043BF6
:108C8000403ABDD2303211D351F8043B40F8043B96
:108C900051F8043B40F8043B51F8043B40F8043BD6
:108CA00051F8043B40F8043B103AEDD20C3205D3A6
:108CB00051F8043B40F8043B043AF9D2043208D09E
:108CC000D2071CBF11F8013B00F8013B01D30B8810
:108CD00003806046704700BF082A13D38B078DD0EE
:108CE00010F003038AD0C3F10403D21ADB071CBFC0
:108CF00011F8013B00F8013B80D331F8023B20F82A
:108D0000023B7BE7043AD9D3013A11F8013B00F862
:108D1000013BF9D20B7803704B7843708B788370EA
:108D200060467047000000000000000000000000E6
:108D30000000000000000000000000000000000033
:108D4000A2EB0300704700BF02780B78012A28BF0E
:108D50009A42F5D16DE9044540EA0104CDE9026784
:108D60006FF0000C4FEA447212B380EA010414F071
:108D7000070F6AD100F0070420F0070004F0030594
:108D800021F007014FEAC505F0E8042314F0040FB1
:108D9000F1E804670CFA05F462EA040266EA0406E4
:108DA0000AD063EA0403624667EA0407664603E002
:108DB000F0E80423F1E8046782FA4CF582EA06043D
:108DC000A4FA8CF46CBB83FA4CF583EA0705A5FA88
:108DD0008CF595B950E9022351E9026782FA4CF506
:108DE00082EA0604A4FA8CF483FA4CF583EA0705B8
:108DF000A5FA8CF52543DBD09CB92DBAB5FA85F4DC
:108E000024F0070427FA04F1DDE9026723FA04F3EA
:108E100003F0FF0001F0FF01FDE80445A0EB0100B5
:108E2000704724BAB4FA84F424F0070426FA04F153
:108E3000DDE9026722FA04F202F0FF0001F0FF010F
:108E4000FDE80445A0EB0100704714F0030F3CD18E
:108E500010F0030428D150F8082B51F8083B82FA8F
:108E60004CF582EA0305A5FA8CF55DB950F8042C9F
:108E700051F8043C82FA4CF582EA0305A5FA8CF518
:108E8000002DE8D02DBAB5FA85F424F0070423FAB2
:108E900004F122FA04F202F0FF0001F0FF01FDE804
:108EA0000445A0EB010070474FEAC40420F0030022
:108EB00050F8082B21F0030151F8083B0CFA04F498
:108EC00062EA040263EA0403C9E710F003041AD05B
:108ED000A1EB040120F00300E40750F8042B06D0B6
:108EE0000FD28B785FFAA2F4E41A06D12BB1CB78BB
:108EF0005FFAB2F4E41A00D11BB920465DF8104BBA
:108F0000704701F1040150F8042BCC0721F0030154
:108F100051F8043B48D824D222F07F4482FA4CF521
:108F200094EA1325A5FA8CF50AD165B951F8043BEA
:108F300084EA0204B4EB036F0ED150F8042BEBE784
:108F40004FEA132355E035F07F454DD10878FDE811
:108F50000445C0F1000070474FEA126203F0FF03BE
:108F600047E002EA1C4482FA4CF594EA1345A5FA5C
:108F70008CF50AD165B951F8043B84EA0204B4EBDC
:108F8000034F0CD150F8042BEBE74FEA134330E0CA
:108F900015EA1C4528D10B884FEA124229E04FEA16
:108FA000124203EA1C4324E002F0FF0482FA4CF56B
:108FB00094EA1365A5FA8CF50AD165B951F8043B1A
:108FC00084EA0204B4EB032F09D150F8042BEBE739
:108FD0004FEA13630DE015F0FF0F05D10B684FEA60
:108FE000122223F07F4304E04FF00000FDE8044527
:108FF000704712BA1BBA82FA4CF482EA0304A4FA4C
:109000008CF5B5FA85F402FA04F203FA04F34FEA98
:109010001260FDE80445A0EB1360704700000000FB
:109020000000000000000000000000000000000040
:109030000000000000000000000000000000000030
:1090400090F800F06DE9024520F007016FF0000C88
:1090500010F0070491F820F040F049804FF0000430
:109060006FF00700D1E9002391F840F000F108000B
:1090700082FA4CF2A4FA8CF283FA4CF3A2FA8CF343
:109080004BBBD1E9022382FA4CF200F10800A4FAAA
:109090008CF283FA4CF3A2FA8CF3E3B9D1E90423FE
:1090A00082FA4CF200F10800A4FA8CF283FA4CF335
:1090B000A2FA8CF37BB9D1E9062301F1200182FAEF
:1090C0004CF200F10800A4FA8CF283FA4CF3A2FAF5
:1090D0008CF3002BC6D0002A04BF04301A4612BA03
:1090E000B2FA82F2FDE8024500EBD2007047D1E906
:1090F000002304F00305C4F100004FEAC50514F095
:10910000040F91F840F00CFA05F562EA05021CBF65
:1091100063EA050362464FF00004A9E700B583B097
:10912000294BD3F8D82042F00102C3F8D820D3F855
:10913000D82002F001020092009AD3F8D82042F021
:109140000202C3F8D820D3F8D83003F00203019309
:10915000019B002205210B2001F0D4FC0B2001F023
:1091600003FD002205210C2001F0CCFC0C2001F0B5
:10917000FBFC002205210D2001F0C4FC0D2001F0B4
:10918000F3FC002205210E2001F0BCFC0E2001F0B2
:10919000EBFC002205210F2001F0B4FC0F2001F0B0
:1091A000E3FC002205213B2001F0ACFC3B2001F058
:1091B000DBFC002205213C2001F0A4FC3C2001F056
:1091C000D3FC03B05DF804FB0044025810B5154809
:1091D000154B036000238360C3600374437483747E
:1091E000032141610A2282611D24C461026241623D
:1091F0008262C4620263436301228263C3630164C7
:10920000042242648164C264036542658365C36568
:1092100002664366826603F0C1F900B910BD00F032
:109220003FFBFBE7180E002400A0004010B51648D5
:10923000164B036000238360C3600374437483741C
:10924000032141610A2282611D24C46102624162DC
:109250008262C462026340F2553242630122826339
:10926000C3630164042242648164C264036542658D
:109270008365C36502664366826603F08FF900B9B1
:1092800010BD00F00DFBFBE7B80E002400A4004069
:1092900010B51648164B036000238360C360037447
:1092A00043748374032141610A2282611D24C461D5
:1092B000026241628262C462026340F2AB62426354
:1092C00001228263C3630164042242648164C26434
:1092D000036542658365C36502664366826603F083
:1092E0005DF900B910BD00F0DBFAFBE7580F002470
:1092F00000D4004030B5BBB0044600213591369112
:10930000379138913991B82206A813F0CFF8236825
:10931000844A934208D0844A93425CD0834A934261
:1093200000F0B0803BB030BD4FF400420023CDE9E7
:1093300006234FF08053219306A805F035FD002841
:1093400038D17B4A136801331360012B35D0794B38
:10935000D3F8E02042F00802C3F8E020D3F8E03070
:1093600003F008030193019B0323359302233693F3
:109370000024379438940923399335A96E4803F0B3
:10938000F1FD22460521132001F0BCFB132001F062
:10939000EBFB22460521152001F0B4FB152001F05E
:1093A000E3FB224605213F2001F0ACFB3F2001F00A
:1093B000DBFBB7E700F074FAC3E75E4BD3F8EC20B1
:1093C00042F48072C3F8EC20D3F8EC3003F48073DD
:1093D0000093009BBBE74FF400420023CDE9062336
:1093E0004FF08053219306A805F0DEFC002838D109
:1093F0004F4A136801331360012B35D04D4BD3F81E
:10940000E02042F00202C3F8E020D3F8E03003F09D
:1094100002030393039B60233593022336930024B6
:10942000379438940923399335A9444803F09AFDB9
:1094300022460521142001F065FB142001F094FB65
:1094400022460521162001F05DFB162001F08CFB61
:10945000224605213F2001F055FB3F2001F084FB0F
:1094600060E700F01DFAC3E7324BD3F8EC2042F47A
:109470008072C3F8EC20D3F8EC3003F480730293CD
:10948000029BBBE74FF400420023CDE906234FF0D7
:109490008053219306A805F087FC88BB244A1368F3
:1094A00001331360012B2ED0224BD3F8E02042F081
:1094B0000802C3F8E020D3F8E03003F00803059376
:1094C000059B4FF440533593022336930024379481
:1094D00038940525399535A9174803F043FD2246F0
:1094E00029469F2001F00EFB9F2001F03DFB224604
:1094F0002946A02001F006FBA02001F035FB11E772
:1095000000F0CEF9CAE70B4BD3F8EC2042F480729E
:10951000C3F8EC20D3F8EC3003F480730493049B7D
:10952000C2E700BF00A0004000A4004000D40040FB
:10953000140E002400440258000C02580004025883
:1095400008B50BF0BDFF01200AF0FDFDFBE70000B0
:10955000034B0360034B0B6080231360704700BF15
:10956000FC110024FC0F002430B589B001AC074D7C
:109570000FCD0FC495E8070084E80700002101A87B
:109580000AF0ACFD024B186009B030BD901C020817
:10959000F80F00242DE9F0478CB0002407940894BC
:1095A00009940A940B945F4BD3F8E02042F0100228
:1095B000C3F8E020D3F8E02002F010020192019AF3
:1095C000D3F8E02042F00402C3F8E020D3F8E02012
:1095D00002F004020292029AD3F8E02042F08002E4
:1095E000C3F8E020D3F8E02002F080020392039A4F
:1095F000D3F8E02042F00102C3F8E020D3F8E020E5
:1096000002F001020492049AD3F8E02042F0020230
:10961000C3F8E020D3F8E02002F002020592059A98
:10962000D3F8E02042F00802C3F8E020D3F8E0309D
:1096300003F008030693069B3B4E22464FF4C041BD
:10964000304603F086FD01220921304603F081FDFA
:10965000DFF8DC8001224FF40041404603F079FD41
:10966000324F22464FF48061384603F072FD4FF4CA
:10967000C04307930125089509940A9407A9304629
:1096800003F070FC09230793089509944FF0030A2F
:10969000CDF828A007A9304603F064FC48F2200367
:1096A000079308940994DFF88C9007A9484603F0C3
:1096B00059FC4FF4A05307934FF48813089309946F
:1096C00007A9404603F04EFC4FF40043079308956A
:1096D0000994CDF828A007A9404603F043FC4FF4B5
:1096E00080660796089509940A9407A9384603F0FE
:1096F00039FC07960226089609940A9407250B95CB
:1097000007A9484603F02EFC702307930896099496
:109710000A940B9507A9384603F024FC0CB0BDE869
:10972000F08700BF0044025800080258000C02589D
:10973000001002580000025808B51548154B036088
:10974000A3F17863A3F57E23A3F24F2343600023A4
:1097500083600122C260036143618361C36103626C
:1097600003F0FEFC50B90021094803F05DFD40B94B
:109770000021074803F086FD30B908BD00F090F8DD
:10978000F1E700F08DF8F3E700F08AF8F5E700BFA5
:10979000501200240058004010B5B6B00446002115
:1097A00031913291339134913591B82202A812F05F
:1097B0007DFE22681C4B9A4201D036B010BD0822B3
:1097C0000023CDE902230023229302A805F0ECFA3E
:1097D00038BB164CD4F8E03043F00203C4F8E03054
:1097E000D4F8E03003F002030093009B4FF4406391
:1097F000319312233293002333933493042335930C
:1098000031A90B4803F0AEFBD4F8E83043F48003F1
:10981000C4F8E830D4F8E83003F480030193019BE6
:10982000CBE700F03DF8D4E7005800400044025870
:109830000004025810B584B00024009401940294EE
:10984000039401F09FF901238DF800308DF8014059
:1098500001941F228DF8082087228DF809208DF8A9
:109860000A408DF80B408DF80C308DF80D308DF8D6
:109870000E408DF80F40684601F0A6F9042001F073
:1098800091F904B010BD000008B50268034B9A427C
:1098900000D008BD01F0FEF8FBE700BF002000404B
:1098A00072B6FEE700B59DB04C22002109A812F067
:1098B000FDFD2022002101A812F0F8FD022004F095
:1098C0008BFB00230093214B9A6922F440429A615A
:1098D0009B6903F440430093009B1C4B9B6913F46A
:1098E000005FFAD0012209924FF480330A930223D9
:1098F000129313930521149160211591169204225D
:10990000179218930823199300231A931B9309A8FD
:1099100004F094FBA8B93F23019303210291002393
:109920000393082304934023059306934FF4806226
:109930000792089301A804F071FF20B91DB05DF8EB
:1099400004FBFFF7ADFFFFF7ABFF00BF0048025875
:1099500000B583B0FFF76EFF01F06EF8FFF7A2FFCE
:10996000FFF718FEFFF7DAFBFFF730FCFFF75EFCAE
:10997000FFF78EFC00F06AF800F052FC00F0D6FC15
:1099800000F034FD00F074FD00F0CCFD00F006FEA8
:1099900000F03AFEFFF7D0FE00F026F80D4C002153
:1099A000204607F019F9236844F620625A6340F212
:1099B000DC5001F081F80CF06DFF074B0093074B72
:1099C000074A084900200BF06BFDFFF7CDFD0AF0B8
:1099D00080FBFEE7F414002460250208202502081D
:1099E000242502082C25020808B51648164B0360EA
:1099F0004FF480034360002383600722C2604FF06E
:109A0000007202614FF0807242614FF080628261A9
:109A10004FF00052C261036243628362C3624FF03F
:109A2000804242638363C363036443648364C364A7
:109A300003654365836506F089F900B908BDFFF742
:109A40002FFFFBE7941300240030014008B51348B2
:109A5000134B03604FF480034360002383600322B1
:109A6000C260036143614FF080628261C36103623F
:109A700043628362C3624FF0804242638363C36385
:109A8000036443648364C36403654365836506F0CC
:109A90005DF900B908BDFFF703FFFBE71C140024C4
:109AA00000380040F0B5BBB0044600213591369136
:109AB000379138913991B82206A812F0F7FC236843
:109AC0006D4A934205D06D4A934200F088803BB0C6
:109AD000F0BD4FF480520023CDE9062300231D93EF
:109AE00006A805F061F9002870D1654BD3F8F02085
:109AF00042F48052C3F8F020D3F8F02002F48052F0
:109B00000092009AD3F8E02042F00802C3F8E02067
:109B1000D3F8E02002F008020192019AD3F8E02085
:109B200042F00202C3F8E020D3F8E03003F0020371
:109B30000293029B802335930227369700253795A1
:109B400038950526399635A94E4803F00BFA1823A7
:109B50003593369737953895399635A94A4803F0A5
:109B600001FA4A484A4B0360252343608560C5607B
:109B70004FF48063036145618561C561056245629B
:109B800001F05AFA28BB414BE3679C634148424BC2
:109B9000036026234360402383600023C3604FF4A7
:109BA0008062026143618361C3610362436201F0C9
:109BB00043FA88B9374BA3679C6300220521232011
:109BC00000F0A0FF232000F0CFFF80E7FFF768FE42
:109BD0008BE7FFF765FED6E7FFF762FEEAE74FF493
:109BE00080520023CDE9062300231D9306A805F02B
:109BF000DBF800283DD1224BD3F8E82042F4804224
:109C0000C3F8E820D3F8E82002F480420392039AD4
:109C1000D3F8E02042F00402C3F8E020D3F8E020BB
:109C200002F004020492049AD3F8E02042F0020207
:109C3000C3F8E020D3F8E03003F002030593059B5E
:109C4000062335930226369600243794389405254A
:109C5000399535A9114803F085F94FF40053359330
:109C6000369637943894399535A9074803F07AF930
:109C70002DE7FFF715FEBEE7003001400038004039
:109C800000440258000C025800040258A412002498
:109C9000580402401C1300247004024000080258BB
:109CA00000B583B00A4BD3F8F42042F00202C3F8A7
:109CB000F420D3F8F43003F002030193019B002257
:109CC0000F216FF0010000F01DFF03B05DF804FBF1
:109CD000004402580F2801D90120704710B58AB0FE
:109CE0000446002201462D2000F00CFF2D2000F03C
:109CF0003BFF1A4B1C601A4BD3F8E82042F48072E9
:109D0000C3F8E820D3F8E83003F480730093009B95
:109D100001A902A804F012FF079BBBB904F0EAFEF8
:109D200003461048A0FB03239B0C013B0E480F4A3F
:109D3000026040F2E732C260436000230361836047
:109D400006F012FD30B101200AB010BD04F0D2FEC1
:109D50004300E6E7044806F061FBF5E71000002445
:109D60000044025883DE1B43A4140024002000405A
:109D7000FEE7FEE7FEE7FEE7FEE7704708B50248AC
:109D800001F042FF08BD00BF2416002408B50248B8
:109D900001F03AFF08BD00BF9C16002408B5024838
:109DA00001F032FF08BD00BF0418002408B50248C6
:109DB00001F02AFF08BD00BF8C17002408B5024837
:109DC00001F022FF08BD00BF1417002408B50248A7
:109DD00002F038FF08BD00BF180E002408B5024885
:109DE00002F030FF08BD00BFB80E002408B50248DD
:109DF00002F028FF08BD00BF180E002408B5024875
:109E000002F020FF08BD00BFB80E002408B50248CC
:109E100006F074F808BD00BF9413002408B502488A
:109E200007F06EFA08BD00BF1019002408B50248FB
:109E300006F047FB08BD00BFA414002408B5024883
:109E400007F05EFA08BD00BFA419002408B5024857
:109E500001F0DAFE08BD00BFA412002408B50248D4
:109E600001F0D2FE08BD00BF1C13002408B5034852
:109E700002F0E8FE024802F0E5FE08BD180E0024DC
:109E8000B80E002408B5024803F04FFD08BD00BF1E
:109E90002071002408B5024803F047FD08BD00BF4B
:109EA0002071002408B5024803F03FFD08BD00BF43
:109EB0002071002408B5024807F022FA08BD00BF4F
:109EC0007C18002408B5024802F0BCFE08BD00BFA3
:109ED000580F002408B5024802F0B4FE08BD00BFC8
:109EE000580F00240120704708B511F0F5FC162327
:109EF00003604FF0FF3008BD08B54FF0FF31FFF7AA
:109F0000F3FFFEE770B50C4616460025B54207DAAA
:109F1000AFF30080214601F8010B01350C46F5E74F
:109F2000304670BD70B50C4616460025B54205DAC0
:109F300014F8010BAFF300800135F7E7304670BD30
:109F40004FF0FF3070474FF400534B6000207047D4
:109F5000012070470020704710B503460C4A0D4998
:109F60000D48006840B10C4800680344521A9342FF
:109F700006D8094A136010BD0748084C0460F2E790
:109F800011F0AAFC0C2303604FF0FF30F3E700BF91
:109F90000000052400040000F0140024D8880024E8
:109FA000224AD2F8883043F47003C2F88830204B3C
:109FB0001B6803F00F03062B06D81D4A136823F015
:109FC0000F0343F0070313601A4B1A6842F00102B3
:109FD0001A6000221A611968174A0A401A60144B65
:109FE0001B6813F0080F06D0114A136823F00F0303
:109FF00043F0070313600F4B00229A61DA611A6283
:10A000000E4999620E49D9620E4919635A639963E0
:10A01000DA6319645A64196821F4802119601A6698
:10A02000094B43F2D2021A60704700BF00ED00E016
:10A0300000200052004402587FEDF6EA00020202BE
:10A040000000FF01800201010040005284B003685B
:10A050001A4A934207D0B3F1804F12D0184A934264
:10A060001DD004B07047174BD3F8F02042F0010226
:10A07000C3F8F020D3F8F03003F001030193019B03
:10A08000EFE7104BD3F8E82042F00102C3F8E820D4
:10A09000D3F8E83003F001030293029BE1E7094B98
:10A0A000D3F8E82042F04002C3F8E820D3F8E830C3
:10A0B00003F040030393039BD3E700BF000001407C
:10A0C000001800400044025802680A4B9A4200D02F
:10A0D000704782B0084BD3F8E82042F00202C3F880
:10A0E000E820D3F8E83003F002030193019B02B0AB
:10A0F000704700BF000400400044025800B58BB018
:10A1000000230593069307930893099303683D4A38
:10A1100093420BD0B3F1804F24D03B4A93423CD0C2
:10A120003A4A934252D00BB05DF804FB384BD3F857
:10A13000E02042F01002C3F8E020D3F8E03003F052
:10A1400010030193019B4FF40853059302230693D8
:10A150000023079308930123099305A92D4802F0D2
:10A1600001FFE0E72A4BD3F8E02042F00102C3F8F8
:10A17000E020D3F8E03003F001030293029B0523B3
:10A180000593022306930023079308930123099361
:10A1900005A9214802F0E6FEC5E71D4BD3F8E020F3
:10A1A00042F00202C3F8E020D3F8E03003F00203EB
:10A1B0000393039B022305930693002207920892C0
:10A1C000099305A9154802F0CDFEACE7104BD3F872
:10A1D000E02042F00202C3F8E020D3F8E03003F0C0
:10A1E00002030493049B4FF4004305930223069358
:10A1F000002207920892099305A9084802F0B2FECE
:10A2000091E700BF0000014000040040001800403A
:10A21000004402580010025800000258000402587E
:10A2200010B59CB000241794189419941A941B9498
:10A230001494159416940D940E940F9410941194F4
:10A240001294139434222146684612F02FF93548AF
:10A25000354B0360446084604FF6FF73C360046154
:10A260004461846106F080FA002846D12D4806F04A
:10A27000ABFA002844D1072317930023189317A99A
:10A28000284806F06DFC00283DD100231493159357
:10A29000169314A9234806F05BFD002836D16023ED
:10A2A0000D9300220E920F9210921192129213921D
:10A2B0000DA91C4806F002FB58BB08220DA919483D
:10A2C00006F0FCFA40BB0023009301930293039332
:10A2D00004934FF400520592069308934FF00072D6
:10A2E00009920A930C9369460E4806F089FDB0B9AD
:10A2F0000C48FFF703FF1CB010BDFFF7D1FAB5E71C
:10A30000FFF7CEFAB7E7FFF7CBFABEE7FFF7C8FAD9
:10A31000C5E7FFF7C5FAD0E7FFF7C2FAD3E7FFF7C3
:10A32000BFFAE5E7F41400240000014000B591B045
:10A3300000230B930C930D930E930F9308930993A3
:10A340000A9301930293039304930593069307934F
:10A3500025484FF080420260436083604FF0FF3237
:10A36000C2600361836106F0FFF958BB1E4806F026
:10A370002BFA50BB07230B9300230C930BA91A480D
:10A3800006F0EEFB20BB002308930A9308A91648A9
:10A3900006F0DEFCF8B960230193002202920392DA
:10A3A000059201A9104806F089FAB8B9082201A956
:10A3B0000D4806F083FAA0B90B48FFF79FFE11B0D5
:10A3C0005DF804FBFFF76CFAD0E7FFF769FAD1E715
:10A3D000FFF766FAD7E7FFF763FADCE7FFF760FA03
:10A3E000E4E7FFF75DFAE7E78C15002400B58BB0D2
:10A3F0000023079308930993009301930293039317
:10A400000493059306931848184A02601722426085
:10A41000836042F20F72C2600361836106F0D4F977
:10A42000C8B900230793099307A90F4806F090FCC9
:10A43000A0B96023009300230193029304930C229C
:10A440006946094806F03AFA58B90748FFF756FE38
:10A450000BB05DF804FBFFF723FAE2E7FFF720FA01
:10A46000E7E7FFF71DFAF0E7D815002400040040E5
:10A4700000B591B000230B930C930D930E930F93A3
:10A48000089309930A93019302930393049305930A
:10A49000069307932148224A0260436083604FF687
:10A4A000FF72C2600361836106F05EF938BB1B482E
:10A4B00006F08AF930BB07230B9300230C930BA9FA
:10A4C000164806F04DFB00BB002308930A9308A929
:10A4D000124806F03DFCD8B9602301930023029393
:10A4E0000393059304220DEB02010C4806F0E6F9F4
:10A4F00088B90A48FFF702FE11B05DF804FBFFF7C8
:10A50000CFF9D4E7FFF7CCF9D5E7FFF7C9F9DBE7D7
:10A51000FFF7C6F9E0E7FFF7C3F9EAE740150024C3
:10A520000018004008B51A481A4B03601A4B4360E4
:10A530004FF4805383604FF40053C3604FF4806343
:10A5400003610C23436100238361C361036243629F
:10A55000836207F0F4FD70B900210D4807F006FF93
:10A5600060B900210A4807F026FF50B9084807F0F3
:10A57000DEFE48B908BDFFF793F9EDE7FFF790F964
:10A58000EFE7FFF78DF9F1E7FFF78AF9F2E700BF90
:10A59000A419002400500040A086010008B5184806
:10A5A000184B03604FF4E133436000218160C160C8
:10A5B00001610C2343618161C16101624162816279
:10A5C0000B460A4607F06CFE70B900210C4807F0F4
:10A5D000CDFE60B900210A4807F0EDFE50B90848E9
:10A5E00007F0A5FE48B908BDFFF75AF9EDE7FFF7F8
:10A5F00057F9EFE7FFF754F9F1E7FFF751F9F2E701
:10A60000101900240048004008B51748174B036094
:10A610004FF4E133436000238360C36003610C2285
:10A6200042618361C36103624362836207F087FD15
:10A6300070B900210C4807F099FE60B900210A4862
:10A6400007F0B9FE50B9084807F071FE48B908BDD7
:10A65000FFF726F9EDE7FFF723F9EFE7FFF720F91A
:10A66000F1E7FFF71DF9F2E77C180024001C014018
:10A67000F0B5BDB0044600213791389139913A9137
:10A680003B91B82208A811F011FF2368824A934237
:10A6900008D0824A934276D0814A934200F01681D4
:10A6A0003DB0F0BD02220023CDE90823002325930D
:10A6B00008A804F079FB00285FD17A4BD3F8E82092
:10A6C00042F48012C3F8E820D3F8E82002F48012A4
:10A6D0000092009AD3F8E02042F00402C3F8E02090
:10A6E000D3F8E02002F004020192019AD3F8E020AE
:10A6F00042F00802C3F8E020D3F8E03003F008038A
:10A700000293029B4FF4805337930227389700251A
:10A7100039953A9508263B9637A9634802F022FC02
:10A7200004233793389739953A953B9637A95F4874
:10A7300002F018FC5E485F4B036041234360856074
:10A74000C5604FF480630361456185614FF4807398
:10A75000C3614FF440330362456200F06DFC78B989
:10A76000534BC4F880309C6300220521352000F053
:10A77000C9F9352000F0F8F992E7FFF791F89CE766
:10A78000FFF78EF8ECE702220023CDE9082300232F
:10A79000259308A804F008FB002873D1414BD3F897
:10A7A000E82042F48022C3F8E820D3F8E82002F43D
:10A7B00080220392039AD3F8E02042F00202C3F809
:10A7C000E020D3F8E02002F002020492049AD3F8C9
:10A7D000E02042F00802C3F8E020D3F8E03003F0B4
:10A7E00008030593059B4FF480433793022738975E
:10A7F000002539953A9507263B9637A92E4802F051
:10A80000B1FB4FF440733793389739953A953B969F
:10A8100037A9264802F0A6FB2848294B03602E23BF
:10A82000436040238360C5604FF4806303614561EA
:10A830008561C5610562456200F0FEFB28BB1F4BC8
:10A84000E3679C631F48204B03602D234360002374
:10A850008360C3604FF48062026143618361C361BE
:10A860000362436200F0E8FB90B9164BC4F88030F5
:10A870009C6300220521272000F044F9272000F0E6
:10A8800073F90DE7FFF70CF888E7FFF709F8D6E74B
:10A89000FFF706F8E9E700BF00500040004800401D
:10A8A000001C01400044025800080258000C0258E5
:10A8B000241600241000024000040258041800244A
:10A8C000400002408C17002458000240012200235F
:10A8D000CDE908230023269308A804F065FA002890
:10A8E0006AD13A4BD3F8F02042F08002C3F8F0204E
:10A8F000D3F8F02002F080020692069AD3F8E02006
:10A9000042F01002C3F8E020D3F8E03003F0100367
:10A910000793079B0423379302273897002539951F
:10A920003A953B932A4E37A9304602F01BFB082389
:10A930003793389739953A950B233B9337A930468F
:10A9400002F010FB2348244B0360762343608560AC
:10A95000C5604FF48063036145618561C5614FF453
:10A9600080330362456200F067FB40BB194BC4F8BB
:10A9700080309C6319481A4B03607723436040235F
:10A9800083600023C3604FF480620261436183618E
:10A99000C3614FF480320262436200F04DFB88B91C
:10A9A0000E4BE3679C63002205219C2000F0AAF86F
:10A9B0009C2000F0D9F873E6FEF772FF91E7FEF7EE
:10A9C0006FFFD3E7FEF76CFFEAE700BF00440258D1
:10A9D000001002589C16002428000240141700247E
:10A9E00070000240DFF834D0FFF7DAFA0C480D4966
:10A9F0000D4A002302E0D458C4500433C4188C42DA
:10AA0000F9D30A4A0A4C002301E013600432A2423F
:10AA1000FBD311F0B9F9FEF79BFF70470000052446
:10AA200000000024F80D0024DC4A0208F80D002480
:10AA3000D8880024FEE7000010B5032000F050F88D
:10AA400003F0F2FD0F498B69C3F303230E4AD35C75
:10AA500003F01F03D8408B6903F00F03D35C03F0AE
:10AA60001F0320FA03F3094A1360094B18600F20F3
:10AA7000FFF730F910B10124204610BD0446FFF75E
:10AA80000FF9F9E70044025868250208080000247D
:10AA900004000024034B1B78034A11680B44136025
:10AAA000704700BF0C000024381A0024014B1868BE
:10AAB000704700BF381A002438B50446FFF7F6FF88
:10AAC0000546B4F1FF3F02D0044B1B781C44FFF74E
:10AAD000EDFF401BA042FAD338BD00BF0C0000249C
:10AAE0000649CB6823F4E0631B041B0C000200F44E
:10AAF000E0600343024A1A43CA60704700ED00E079
:10AB00000000FA0530B4154BDB68C3F30223C3F130
:10AB10000704042C28BF04241D1D062D14D9033B53
:10AB20004FF0FF3505FA04F421EA0401994005FAD3
:10AB300003F322EA03031943002807DB0901C9B222
:10AB4000074B195430BC70470023E9E700F00F00B1
:10AB50000901C9B2034B1954F4E700BF00ED00E04E
:10AB600000E400E014ED00E0002807DB00F01F0225
:10AB7000400901239340024A42F82030704700BF49
:10AB800000E100E0BFF35F8F044A536A23F480338F
:10AB90005362034B00225A60704700BF00ED00E093
:10ABA00090ED00E040F00100054B5860054A536A03
:10ABB00043F480335362BFF34F8FBFF36F8F7047FF
:10ABC00090ED00E000ED00E04378114A93601369D6
:10ABD00023F0010313614368D360017BC37A1B0632
:10ABE00043EA0173817A43EAC143417B43EA8143EB
:10ABF000817B43EA4143C17B43EA0143417A43EA13
:10AC00000123017A43EA410301780B431361704742
:10AC100090ED00E0F0B4876D0468654E654DAC4280
:10AC200018BFB44242D01835AC423FD01835AC42C0
:10AC30003CD01835AC4239D01835AC4236D0183536
:10AC4000AC4233D01835AC4230D005F55675AC4225
:10AC50002CD01835AC4229D01835AC4226D0183546
:10AC6000AC4223D01835AC4220D01835AC421DD0B0
:10AC70001835AC421AD01835AC4217D04E4DAC4204
:10AC800014D01435AC4211D01435AC420ED014356A
:10AC9000AC420BD01435AC4208D01435AC4205D0D0
:10ACA0001435AC4202D01435AC4207D1446E856EE7
:10ACB0006560C46E14B1046F456F656004683C4EF6
:10ACC0003C4DAC4218BFB44252D01835AC424FD0C4
:10ACD0001835AC424CD01835AC4249D01835AC428E
:10ACE00046D01835AC4243D01835AC4240D005F5BB
:10ACF0005675AC423CD01835AC4239D01835AC4210
:10AD000036D01835AC4233D01835AC4230D0183577
:10AD1000AC422DD01835AC422AD01835AC4227D0E1
:10AD2000254E264DAC4218BFB44211D0244DAC4242
:10AD30000ED01435AC420BD01435AC4208D01435CB
:10AD4000AC4205D01435AC4202D01435AC4223D10C
:10AD5000C46D04F01F050124AC407C60046863608E
:10AD60008368402B1FD0036899600368DA6013E0A2
:10AD7000C46D04F01F053F24AC40BC6005682C681E
:10AD800024F480242C60046863608368402B05D021
:10AD9000036899600368DA60F0BC704703689A60E2
:10ADA0000368D960F8E703689A600368D960F3E73D
:10ADB0001000024028000240085402581C54025857
:10ADC0003054025803682749274A934218BF8B42E0
:10ADD0002FD0183293422CD01832934229D01832F7
:10ADE000934226D01832934223D01832934220D077
:10ADF000183293421DD002F55672934219D0183280
:10AE0000934216D01832934213D01832934210D086
:10AE1000183293420DD0183293420AD0183293421E
:10AE200007D01832934204D023F0FF038365806D6E
:10AE3000704710B4D9B210390C4AA2FB0142C2F3D8
:10AE400002120B4CA25CC2655F2907D9094A1A405D
:10AE500004328265806D5DF8044B7047054A1A40E4
:10AE60008265F7E71000024028000240ABAAAAAAB8
:10AE70007825020800FCFFFF83699BB9836A012BD8
:10AE80000AD0022B02D00BB100207047C36A13F026
:10AE9000807F2AD100207047C36AB3F1C07F26D0DB
:10AEA00000207047B3F5005F0AD0836A022B26D9D1
:10AEB000032B26D1C36A13F0807F24D10020704772
:10AEC000836A032B03D8DFE803F01404140A00207C
:10AED0007047C36A13F0807F0DD100207047C36AAA
:10AEE000B3F1C07F09D000207047012070470120D6
:10AEF00070470120704701207047012070470120F2
:10AF00007047002070470120704700000368224905
:10AF1000224A934218BF8B4228D01432934225D044
:10AF20001432934222D0143293421FD014329342EF
:10AF30001CD01432934219D01432934216D0DAB294
:10AF4000103A1749A1FB0212120916491944A829FF
:10AF50001FD9154B13449B000366144B436602F044
:10AF60001F02012303FA02F282667047DBB2083B3C
:10AF70000F4AA2FB03230F4A02EB13129200026650
:10AF80000D4A4266C3F30413012202FA03F38366F7
:10AF900070470832DDE700BF085402581C540258BD
:10AFA000ABAAAAAAF0FBFDBF0082001080080240F5
:10AFB000CDCCCCCC009600168058025801794A1EA0
:10AFC000072A2CD830B40368154D164CA34218BF7D
:10AFD000AB4218D01434A34215D01434A34212D07B
:10AFE0001434A3420FD01434A3420CD01434A3421F
:10AFF00009D01434A34206D00B4B0B449B00C3660C
:10B000000A4B036705E00A4B0B449B00C366094BE0
:10B010000367012303FA02F2426730BC70477047AE
:10B02000085402581C5402583F8200104009024044
:10B030003F9600164059025870B50446FFF736FD9A
:10B04000002C00F0B58105462368AE49AE4A934214
:10B0500018BF8B420CBF0122002250D030318B42EE
:10B060004DD018318B424AD018318B4247D018311D
:10B070008B4244D018318B4241D018318B423ED0A4
:10B0800001F556718B423AD018318B4237D01831C6
:10B090008B4234D018318B4231D018318B422ED0B4
:10B0A00018318B422BD018318B4228D018318B426B
:10B0B00025D09649964A934218BF8B4200F03081C2
:10B0C000944A934200F02C811432934200F028817C
:10B0D0001432934200F024811432934200F0208114
:10B0E0001432934200F01C811432934200F0188114
:10B0F00040236365032384F8353001204AE00221B0
:10B1000084F83510002184F834107ABB824A9342C7
:10B110002CD01832934229D01832934226D01832BC
:10B12000934223D01832934220D0183293421DD03C
:10B1300002F55672934219D01832934216D0183243
:10B14000934213D01832934210D0183293420DD04C
:10B15000183293420AD01832934207D018329342E1
:10B1600004D01A6822F001021A6003E01A6822F083
:10B1700001021A6023681A6812F0010F0BD0FFF762
:10B1800095FC431B052BF5D920236365032384F825
:10B190003530012070BD1A6860481040A168E2682F
:10B1A0000A4321690A4361690A43A1690A43E169C3
:10B1B0000A43216A0A430243616A042900F0968027
:10B1C0006168A1F12905A1F13F00032888BF052D81
:10B1D0000AD9A1F14700012806D9A1F14F0003289F
:10B1E00002D97439032901D842F480121A60266802
:10B1F000756925F00705636A1D43042B08D1A36A0E
:10B200001D43E36A23B12046FFF736FE002872D1C2
:10B2100075612046FFF7D6FDE36D03F01F023F2363
:10B220009340836023683749374A934218BF8B4263
:10B2300042D0183293423FD0183293423CD0183259
:10B24000934239D01832934236D01832934233D0D9
:10B250001832934230D002F5567293422CD01832F5
:10B26000934229D01832934226D01832934223D0E9
:10B270001832934220D0183293421DD01832934294
:10B280001AD01832934217D0204A934214D0143265
:10B29000934211D0143293420ED0143293420BD009
:10B2A0001432934208D01432934205D014329342A0
:10B2B00002D01432934213D12046FFF727FEA36831
:10B2C000802B68D0236E22791A60636EA26E5A605A
:10B2D0006368013B072B61D90023E366236763673B
:10B2E00000206065012384F8353053E7E16A206B64
:10B2F00001430A4364E740236365012084F8350075
:10B3000048E700BF100002402800024008540258DD
:10B310001C54025830540258400002403F8010FE36
:10B32000022284F83520002284F834201A6821494A
:10B330001140A268402A2CD0802A27D00022E06841
:10B3400042EAD002206942EAD002606942EAD002B1
:10B35000A06942EAD002E06942EAD002206A42EAE9
:10B3600010120A431A602268134B1344134AA2FBBB
:10B3700003231B099B00E3652046FFF723FDE26DD5
:10B3800002F01F0101228A4042604BE74FF48042E5
:10B39000D5E71022D3E70023636093E72046FFF749
:10B3A0000DFEE36E00221A60236F626F5A6097E70A
:10B3B0000120EFE60F00FEFFF8ABFDA7CDCCCCCC13
:10B3C000002800F03E8170B5044690F83400012852
:10B3D00000F03981012084F8340094F83500C0B2BF
:10B3E000012807D04FF400636365002384F83430EC
:10B3F000012070BD022084F83500002060652068BF
:10B40000924E934DA84218BFB0422FD01835A84293
:10B410002CD01835A84229D01835A84226D0183586
:10B42000A84223D01835A84220D01835A8421DD0F4
:10B4300005F55675A84219D01835A84216D018350A
:10B44000A84213D01835A84210D01835A8420DD004
:10B450001835A8420AD01835A84207D01835A84296
:10B4600004D0056825F00105056003E0056825F0B6
:10B47000010505602046FFF7CDFB23687349744A38
:10B48000934218BF8B4238D01832934235D01832CD
:10B49000934232D0183293422FD0183293422CD09C
:10B4A0001832934229D01832934226D002F55672B0
:10B4B000934222D0183293421FD0183293421CD0AC
:10B4C0001832934219D01832934216D01832934250
:10B4D00013D01832934210D0183293420DD01A680C
:10B4E00022F00E0242F00A021A60236C93B1226825
:10B4F000136843F0040313600CE01A6822F01E0284
:10B5000042F016021A60236C23B12268136843F0DC
:10B510000803136023684D494D4A934218BF8B427C
:10B5200042D0183293423FD0183293423CD0183266
:10B53000934239D01832934236D01832934233D0E6
:10B540001832934230D002F5567293422CD0183202
:10B55000934229D01832934226D01832934223D0F6
:10B560001832934220D0183293421DD018329342A1
:10B570001AD01832934217D0364A934214D014325C
:10B58000934211D0143293420ED0143293420BD016
:10B590001432934208D01432934205D014329342AD
:10B5A00002D0143293420ED1236E1A6812F4803FF7
:10B5B00003D01A6842F480721A60E36E1BB11A68F5
:10B5C00042F480721A6023682049214A934218BFCE
:10B5D0008B4230D0183293422DD0183293422AD069
:10B5E0001832934227D01832934224D01832934213
:10B5F00021D0183293421ED002F5567293421AD0CF
:10B600001832934217D01832934214D01832934212
:10B6100011D0183293420ED0183293420BD0183208
:10B62000934208D01832934205D01A6842F00102C2
:10B630001A600020DDE61A6842F001021A6000205C
:10B64000D7E6012070470220D3E600BF1000024079
:10B65000280002400854025870B50446FFF726FA45
:10B66000002C00F09181054694F83530DBB2022BB6
:10B6700006D080236365002384F83430012070BD38
:10B6800023688C498C4A934218BF8B4230D01832C1
:10B6900093422DD0183293422AD01832934227D0A9
:10B6A0001832934224D01832934221D01832934258
:10B6B0001ED002F5567293421AD01832934217D018
:10B6C0001832934214D01832934211D01832934258
:10B6D0000ED0183293420BD01832934208D0183251
:10B6E000934205D01A6822F00E021A60266809E01B
:10B6F0001A6822F01E021A602268536923F0800340
:10B700005361266823686B496B4A934218BF8B428A
:10B7100042D0183293423FD0183293423CD0183274
:10B72000934239D01832934236D01832934233D0F4
:10B730001832934230D002F5567293422CD0183210
:10B74000934229D01832934226D01832934223D004
:10B750001832934220D0183293421DD018329342AF
:10B760001AD01832934217D0544A934214D014324C
:10B77000934211D0143293420ED0143293420BD024
:10B780001432934208D01432934205D014329342BB
:10B7900002D01432934204D1226E136823F48073D2
:10B7A000136023684349444A934218BF8B422FD009
:10B7B000183293422CD01832934229D01832934237
:10B7C00026D01832934223D01832934220D0183218
:10B7D00093421DD002F55672934219D0183293420B
:10B7E00016D01832934213D01832934210D0183228
:10B7F00093420DD0183293420AD01832934207D0A8
:10B800001832934204D01A6822F001021A6003E051
:10B810001A6822F001021A60336813F0010F0ED08B
:10B82000FFF744F9431B052BF6D920236365032357
:10B8300084F83530002384F8343001201FE7236872
:10B840001C491D4A934218BF8B4239D0183293428B
:10B8500036D01832934233D01832934230D0183257
:10B8600093422DD0183293422AD01832934227D0D7
:10B8700002F55672934223D01832934220D01832E8
:10B8800093421DD0183293421AD01832934217D0E7
:10B890001832934214D01832934211D01832934286
:10B8A0000ED0A16DE36D03F01F02012393404B60A6
:10B8B0000DE000BF1000024028000240085402586A
:10B8C000A16DE36D03F01F023F2393408B6023685B
:10B8D0002E492F4A934218BF8B4242D018329342CE
:10B8E0003FD0183293423CD01832934239D01832AC
:10B8F000934236D01832934233D01832934230D02C
:10B9000002F5567293422CD01832934229D0183245
:10B91000934226D01832934223D01832934220D03B
:10B92000183293421DD0183293421AD018329342E3
:10B9300017D0184A934214D01432934211D01432C3
:10B9400093420ED0143293420BD01432934208D05B
:10B950001432934205D01432934202D014329342EF
:10B960000BD1636EA26E5A60E36E33B11A6822F493
:10B9700080721A60236F626F5A60012384F8353039
:10B98000002084F834007AE6012078E610000240B6
:10B990002800024008540258002800F0298108B508
:10B9A000024690F83530DBB2022B03D0802343658A
:10B9B000012008BD0368904890498B4218BF83421C
:10B9C0000CBF0121002166D03030834263D0183093
:10B9D000834260D0183083425DD0183083425AD001
:10B9E0001830834257D01830834254D000F5567037
:10B9F000834250D0183083424DD0183083424AD011
:10BA00001830834247D01830834244D018308342E4
:10BA100041D0183083423ED0183083423BD0196861
:10BA200021F00E0119601368A0F5956073498B42EF
:10BA300018BF83426AD072498B4267D018318B425B
:10BA400064D018318B4261D018318B425ED01831EE
:10BA50008B425BD018318B4258D001F556718B4226
:10BA600054D018318B4251D018318B424ED01831FE
:10BA70008B424BD018318B4248D018318B4245D085
:10BA800018318B4242D018318B423FD0196821F0D7
:10BA9000010119603EE0042082F8350081BB584A5C
:10BAA00093422DD0183293422AD01832934227D095
:10BAB0001832934224D01832934221D01832934244
:10BAC0001ED002F5567293421AD01832934217D004
:10BAD0001832934214D01832934211D01832934244
:10BAE0000ED0183293420BD01832934208D018323D
:10BAF000934205D01A6822F001021A60002058E72C
:10BB00001A6822F001021A60002052E7196821F039
:10BB1000010119601368384838498B4218BF8342C5
:10BB200042D018318B423FD018318B423CD0183173
:10BB30008B4239D018318B4236D018318B4233D0FA
:10BB400018318B4230D001F556718B422CD0183110
:10BB50008B4229D018318B4226D018318B4223D00A
:10BB600018318B4220D018318B421DD018318B42B6
:10BB70001AD018318B4217D022498B4214D014317D
:10BB80008B4211D014318B420ED014318B420BD02A
:10BB900014318B4208D014318B4205D014318B42C2
:10BBA00002D014318B4217D1116E0B6823F48073CD
:10BBB0000B60906DD36D03F01F0101238B40436038
:10BBC000536E916E5960D36E33B1196821F4807150
:10BBD0001960136F516F5960012382F835300023CB
:10BBE00082F83430136D2BB1104698470020E0E600
:10BBF000012070470020DCE61000024028000240CF
:10BC00004000024008540258F0B583B004460023B7
:10BC10000193A24B1D68A24BA3FB0535AD0A876DAE
:10BC20003E68D7F800C003689E499F48834218BF0A
:10BC30008B420CBF0120002061D09C4A93425ED011
:10BC4000183293425BD01832934258D01832934244
:10BC500055D01832934252D0183293424FD002F549
:10BC6000567293424BD01832934248D018329342C6
:10BC700045D01832934242D0183293423FD0183206
:10BC800093423CD01832934239D01832934236D086
:10BC90008749884A934218BF8B4212D0864A934202
:10BCA0000FD0143293420CD01432934209D0143284
:10BCB000934206D01432934203D01432934240F0A0
:10BCC00062821A68E16D01F01F010420884010EAC9
:10BCD0000C0F00F0A88212F0040F00F0A48278602C
:10BCE00012F4004F00F05B8212F4803F40F051826A
:10BCF000A36C002B00F047822046984743E2E26D98
:10BD000002F01F0108228A40324241D070BB674ACC
:10BD100093422BD01832934228D01832934225D028
:10BD20001832934222D0183293421FD018329342D5
:10BD30001CD002F55672934218D01832934215D097
:10BD40001832934212D0183293420FD018329342D5
:10BD50000CD01832934209D01832934206D01832D0
:10BD6000934203D01A68C2F3C00202E01A68C2F319
:10BD700080026AB11A6822F004021A60E36D03F0CF
:10BD80001F0208239340BB60636D43F001036365AA
:10BD9000E26D02F01F0226FA02F313F0010F37D012
:10BDA0002368404840498B4218BF83422CD0183149
:10BDB0008B4229D018318B4226D018318B4223D0A8
:10BDC00018318B4220D018318B421DD018318B4254
:10BDD0001AD001F556718B4216D018318B4213D010
:10BDE00018318B4210D018318B420DD018318B4254
:10BDF0000AD018318B4207D018318B4204D0183149
:10BE00008B4201D01B6803E05B6913F0800F3BD1CC
:10BE1000E36D03F01F03042202FA03F3334251D00F
:10BE20002268204820498A4218BF824246D01831F1
:10BE30008A4243D018318A4240D018318A423DD0DC
:10BE400018318A423AD018318A4237D018318A42A2
:10BE500034D001F556718A4230D018318A422DD043
:10BE600018318A422AD018318A4227D018318A42A2
:10BE700024D018318A4221D018318A421ED018317C
:10BE80008A421BD013681DE0012303FA02F2BA6054
:10BE9000636D43F002036365BAE700BF040000244A
:10BEA000B5814E1B100002402800024040000240B5
:10BEB000085402581C54025830540258126812F0A8
:10BEC000020F3DD1E36D03F01F03102202FA03F3CA
:10BED00033425FD022689B489B498A4218BF824206
:10BEE00034D018318A4231D018318A422ED01831DC
:10BEF0008A422BD018318A4228D018318A4225D064
:10BF000018318A4222D001F556718A421ED018316A
:10BF10008A421BD018318A4218D018318A4215D073
:10BF200018318A4212D018318A420FD018318A4211
:10BF30000CD018318A4209D01268C2F3800208E09E
:10BF4000BB60636D43F004036365BBE71268C2F333
:10BF5000C002FAB1BB6023681A6812F4802F0DD0BA
:10BF60001B6813F4002F04D1236C9BB12046984723
:10BF700010E0A36C73B1204698470BE01A6812F4E6
:10BF8000807F03D11A6822F008021A60236C0BB17B
:10BF900020469847E36D03F01F03202202FA03F3C3
:10BFA000334200F08E802268664867498A4218BF93
:10BFB00082422ED018318A422BD018318A4228D0A2
:10BFC00018318A4225D018318A4222D018318A424B
:10BFD0001FD018318A421CD001F556718A4218D000
:10BFE00018318A4215D018318A4212D018318A424B
:10BFF0000FD018318A420CD018318A4209D018313A
:10C000008A4206D018318A4203D01268C2F3400235
:10C0100002E01268C2F30012002A52D0BB6094F80A
:10C020003530DBB2042B0ED023681A6812F4802F4F
:10C0300035D01B6813F4002F2CD1636C002B40D03B
:10C04000204698473DE02268136823F016031360EA
:10C050002268536923F080035361236CB3B12268D3
:10C06000136823F008031360E36D03F01F023F23FE
:10C070009340BB60012384F83530002384F83430CA
:10C08000236D002B7FD0204698477CE0A36C002BCB
:10C09000E5D1E9E7E36BA3B12046984711E01A68C0
:10C0A00012F4807F09D11A6822F010021A6001236D
:10C0B00084F83530002384F83430E36B0BB120462C
:10C0C0009847636D002B5ED0636D13F0010F56D05F
:10C0D000042384F8353023681A491B4A934218BF59
:10C0E0008B4233D01832934230D0183293422DD045
:10C0F000183293422AD01832934227D018329342F2
:10C1000024D01832934221D002F5567293421DD0AA
:10C11000183293421AD01832934217D018329342F1
:10C1200014D01832934211D0183293420ED01832E4
:10C1300093420BD01832934208D01A6822F00102C1
:10C140001A6007E010000240280002401A6822F03E
:10C1500001021A60019B01330193AB4204D82368AA
:10C160001B6813F0010FF5D123681B6813F0010F52
:10C170000BD0032384F83530002384F83430E36C8B
:10C180000BB12046984703B0F0BD012384F8353049
:10C19000F2E7236C002BF6D020469847F3E712F025
:10C1A000200F3AD123686449644A934218BF8B42F6
:10C1B0002FD0183293422CD01832934229D0183203
:10C1C000934226D01832934223D01832934220D083
:10C1D000183293421DD002F55672934219D018328C
:10C1E000934216D01832934213D01832934210D093
:10C1F000183293420DD0183293420AD0183293422B
:10C2000007D01832934204D01A6822F004021A6050
:10C2100003E01A6822F008021A60236C002BB2D0E7
:10C2200020469847AFE70220884010EA0C0F60D004
:10C2300012F0020F5DD0786012F4004F0ED012F4AD
:10C24000803F05D1636C002B9DD0204698479AE72C
:10C25000E36B002B97D02046984794E712F0200F0D
:10C2600040D123683449354A934218BF8B422FD0BE
:10C27000183293422CD01832934229D0183293426C
:10C2800026D01832934223D01832934220D018324D
:10C2900093421DD002F55672934219D01832934240
:10C2A00016D01832934213D01832934210D018325D
:10C2B00093420DD0183293420AD01832934207D0DD
:10C2C0001832934204D01A6822F00A021A6003E07E
:10C2D0001A6822F014021A60012384F83530002312
:10C2E00084F83430E36B002B3FF44DAF2046984781
:10C2F00049E7082000FA01F111EA0C0F3FF443AFBF
:10C3000012F0080F3FF43FAF1A6822F00E021A60D5
:10C31000E36D03F01F03012202FA03F37B60626501
:10C3200084F83520002384F83430E36C002B3FF48C
:10C330002AAF2046984726E7100002402800024016
:10C3400030B4446B0268D2F88410704B194041EA53
:10C350008401C2F884100268D2F8841021F47F01AD
:10C36000856B41EA0541C2F88410826B224404685F
:10C37000D4F88810194041EA8201C4F88810046892
:10C38000D4F8881021F4FE01C56B41EA0541C4F8D8
:10C390008810C16B02EB41020468D4F8A010194068
:10C3A00041EA8201C4F8A0100468D4F8A01021F476
:10C3B000FE01056C41EA0541C4F8A010046C416C13
:10C3C00001FB04240268D2F8B010194041EA84014C
:10C3D000C2F8B0100268D2F8B01021F4FE01856CEA
:10C3E00041EA0541C2F8B010826CC16C01FB024405
:10C3F0000268D2F8AC10194041EA8401C2F8AC10CE
:10C40000026D416D01FB02420468D4F8F01019403E
:10C4100041EA8201C4F8F0100468D4F8F01021F465
:10C420007C11856D41EA0541C4F8F010816D02EB85
:10C4300041020468D4F8C0100B4043EA8202C4F8F9
:10C44000C0200268D2F8C03023F47C13C16D43EAE7
:10C450000143C2F8C0300268D2F8C03023F07C53E8
:10C46000016E43EA0163C2F8C030436B284A1A44A4
:10C470009200C266836B02EB83030367C16B03EB1D
:10C48000C1034367046C416C01FB04F103EB8103BE
:10C490008367846CC16C01FB04F103EB8103C36708
:10C4A000046D416D01FB04F103EB8103C0F88030A2
:10C4B000816D03EBC103C0F88430C46D856E05FB4C
:10C4C00004F403EB8403C0F88830016E01FB05F12E
:10C4D00003EB8103C0F890300E498B4207D8D0F8A7
:10C4E000903093420ED9002342F8043BF7E7D0F88E
:10C4F0009C3043F02003C0F89C30032380F8983030
:10C50000012000E0002030BC704700BF0300FFFFA7
:10C51000002B0010FCD30040F0B44C68002C30D14C
:10C520000E698C6826430C6846EA84460D6ACC691D
:10C5300044EA05648D692C434D692C43CD6844EA77
:10C540000544D0F88470806E03FB00F307EB83058D
:10C5500047F823606C6008350020CB680E4CE35C24
:10C56000834216D91418E678A3781B0443EA0663BD
:10C57000647843EA0423145C234345F8043B043005
:10C58000EBE70C698E6826430C68264346F080462C
:10C59000CCE7F0BC704700BF8025020830B595B0ED
:10C5A00004464C22A04901A8FCF722FB002C00F015
:10C5B000388123689D4A934220D094F898300BB379
:10C5C0002268936923F010039361FEF76FFA054622
:10C5D00023689A6912F0080F1AD0FEF767FA431B16
:10C5E0000A2BF5D9D4F89C3043F00103C4F89C30F1
:10C5F000032384F89830012015B030BD03F5807313
:10C600006360DAE784F899302046FCF773FED7E7D9
:10C610009A6942F001029A61FEF748FA05462368DA
:10C620009A6912F0010F0FD1FEF740FA401B0A2859
:10C63000F5D9D4F89C3043F00103C4F89C300323AF
:10C6400084F898300120D7E79A6942F002029A6193
:10C65000237C012B40D02268936943F0400393610F
:10C66000637C012B3ED02268936923F4804393615D
:10C67000A37C012B3CD02268936943F480539361DF
:10C680002268936923F44073A1680B439361226885
:10C69000936923F0A40393612268136923F01003C4
:10C6A0001361E368012B29D0002B2CD0022B00F062
:10C6B0009B802268936943F0800393612268136929
:10C6C00043F010031361E368032B1CD122689369C4
:10C6D00043F02003936116E02268936923F040033E
:10C6E0009361BDE72268936943F480439361BFE798
:10C6F0002268936923F480539361C1E722689369A8
:10C7000043F004039361A3695A1EE369013B1B02D2
:10C7100043EA4263226A013A13436269013A21689B
:10C7200043EA0243CB61A368B3F5407F62D0236E36
:10C7300033B12268D2F8C030616E0B43C2F8C0300A
:10C74000E36D226ED3420DD02168D1F8C83023F0BA
:10C750000703A26E14A800EB820252F84C2C13437C
:10C76000C1F8C830236C6BB12168D1F8BC3023F01C
:10C770000703626C14A800EB820252F84C2C13439E
:10C78000C1F8BC30A36C73B12168D1F8BC3023F080
:10C790007003E26C14A800EB820252F84C2C43EABE
:10C7A0000213C1F8BC30236D73B12168D1F8BC30DD
:10C7B00023F4E063626D14A800EB820252F84C2C63
:10C7C00043EA0223C1F8BC302268184B9A4222D0B7
:10C7D0000023C4F89430C4F89C30012384F89830C6
:10C7E0002046FFF7ADFD07E72268936943F0200379
:10C7F000936188E7A36A013BE26A013A43EA0223B4
:10C80000226B013A43EA0213626A013A216843EA61
:10C810000243CB608BE76268936823F00303936065
:10C82000D6E70120E8E600BFAC1C020800A00040EB
:10C8300090F89830013BDBB2012B07D9D0F89C303F
:10C8400043F00203C0F89C3001207047CB680A68AF
:10C85000D2B9072B0ED08A68DB0643EA82730A69D5
:10C8600043EA02434A691343C26E496842F82130E1
:10C87000002070470A69CB691B0243EA02438A69B8
:10C88000134343F06053EFE710B40A6942EA43727E
:10C89000072B0ED08C684B6943EA8473006F49689C
:10C8A00000EBC10440F83120636000205DF8044BC8
:10C8B00070478B69F2E710B490F89840E4B2012C0D
:10C8C00009D0D0F89C3043F00403C0F89C3001201C
:10C8D0005DF8044B7047920042EA011242EA4302BB
:10C8E000036801990A43C3F880200020F0E790F81C
:10C8F0009830DBB2012B07D0D0F89C3043F0040312
:10C90000C0F89C3001207047022380F898300268FC
:10C91000936923F0010393610023C0F89C3018460B
:10C92000704738B5044690F89830DBB2022B2BD113
:10C930000368D3F8C00010F07C5F0CD0D3F8C400BB
:10C9400010F4001F0FD0D4F89C3043F40073C4F8E7
:10C950009C3001201FE0D4F89C3043F02003C4F841
:10C960009C30012017E0D3F8C450C5F304452B4692
:10C970002046FFF7D1FD22680123AB40C2F8D0303A
:10C98000C4F89430002006E0D0F89C3043F008034F
:10C99000C0F89C30012038BDF0B490F89840E4B263
:10C9A000022C40F0D88040290CD041293FD0046DA2
:10C9B0008C4271D8D0F89C3043F02003C0F89C30F2
:10C9C0000120CFE00468D4F8A05015F4FE0F0CD07D
:10C9D000D4F8A45015F07F0F0FD1D0F89C3043F459
:10C9E0008073C0F89C300120BCE0D0F89C3043F04C
:10C9F0002003C0F89C300120B4E0D4F8A450C5F363
:10CA0000006C15F0807F06D0D4F8A0505FEAD57C8A
:10CA100001D14FF0000CD4F8A440C4F30524A44481
:10CA2000446F456C0CFB05F504EB85043CE00468A1
:10CA3000D4F8B05015F4FE0F0CD0D4F8B45015F063
:10CA40007F0F0FD1D0F89C3043F48073C0F89C3036
:10CA5000012087E0D0F89C3043F02003C0F89C30E0
:10CA600001207FE0D4F8B450C5F3006C15F0807F4E
:10CA700006D0D4F8B0505FEAD57C01D14FF0000C5D
:10CA8000D4F8B440C4F30524A444846FC56C0CFBF3
:10CA900005F504EB850407E0C46F456D01FB05F562
:10CAA00004EB85044FF0000C256805F080455560C7
:10CAB000002D2CD12568C5F38A451560256805F041
:10CAC00000559560256805F000451561A588D5617C
:10CAD000E58805F00F05D560656805F4801555619A
:10CAE000656805F400159561E57905F07F05156227
:10CAF0006568ED0F556204F108050024D6681A4FE9
:10CB0000BE5DA64208D92E5D1E550134F6E72568A4
:10CB100025F060451560D1E740290AD041290DD0A4
:10CB20001F290FD80268012303FA01F1C2F89810F7
:10CB300002E00368C3F8A8C0002013E00368C3F84C
:10CB4000B8C0F9E701F01F010268012303FA01F1FF
:10CB5000C2F89C10F0E7D0F89C3043F00803C0F80E
:10CB60009C300120F0BC704780250208402905D088
:10CB70000368D3F8B40000F07F0070470368D3F86F
:10CB8000A40000F07F0070470368D3F8C40000F0F1
:10CB90003F00704790F89830013BDBB2012B07D97A
:10CBA000D0F89C3043F00203C0F89C30012070475D
:10CBB00010B403689C6D0C4224D1DC6D44F0010478
:10CBC000DC6511F4007F05D00468D4F8E03013432D
:10CBD000C4F8E03011F4806F05D00468D4F8E43074
:10CBE0001A43C4F8E4200068436D0C4A0A4013431A
:10CBF00043650B4A536943EA9171516100205DF826
:10CC0000044B70479C6D31EA040402D00324DC65B8
:10CC1000D7E7DC6D44F00204DC65D2E7FFFFCF3FCD
:10CC200000A80040704770477047704770477047D2
:10CC3000704770477047704770477047704770473C
:10CC4000704700002DE9F04F83B00446B74B1A69D6
:10CC50005B699B0703EA8273019303681A6D02F410
:10CC6000704A5A6D0AEA020A1A6D02F00F095A6DEB
:10CC700009EA02091A6D02F0F0085A6D08EA020882
:10CC80001E6D06F071565A6D16401F6D07F06077E5
:10CC90005A6D17405D6DD3F850B015F4807F02D007
:10CCA0001BF4807F64D115F4806F02D01BF4806F79
:10CCB00067D1019B002B74D1BAF1000F7CD1B9F17F
:10CCC000000F40F08580B8F1000F40F08D8015F422
:10CCD000006F03D01BF4006F40F0928015F4007FCA
:10CCE00003D01BF4007F40F0968015F4002F03D092
:10CCF0001BF4002F40F09F8015F4803F03D01BF4FD
:10CD0000803F40F0A38015F4802F03D01BF4802FC8
:10CD100040F0A78015F4003F0FD01BF4003F0CD06B
:10CD200023684FF400321A65804B00221A61D4F850
:10CD30009C3043F08003C4F89C30002F40F09C806E
:10CD40004EB123681E65B20F784B1A61D4F89C303F
:10CD50001E43C4F89C602268754B9A4200F096808E
:10CD6000D4F89C30002B40F0F88003B0BDE8F08F81
:10CD70004FF480721A656D4B00221A61FFF75AFF5B
:10CD800091E72368D3F8DC10D3F8E4204FF48060F7
:10CD90001865664B0020186111402046FFF746FFDA
:10CDA00087E7236800221A6501998A0F5F4B1A6191
:10CDB0002046FFF737FF7FE72368C3F850A04FEA0C
:10CDC0009A725A4B1A6151462046FFF72CFF76E7BC
:10CDD0002368C3F850904FEA9972544B1A61494640
:10CDE000204609F053FF6EE72368C3F850804FEAEE
:10CDF00098724E4B1A614146204609F04CFF66E797
:10CE000023684FF400621A65484B00221A612046DD
:10CE1000FFF70AFF62E72368D3F8D810D3F8E020C1
:10CE20004FF400701865414B0020186111402046F6
:10CE3000FFF7FBFE59E723684FF400221A653B4BCE
:10CE400000221A612046FFF7F2FE55E723684FF4EF
:10CE500080321A65354B00221A612046FFF7E8FE42
:10CE600051E723684FF480221A65304B00221A6183
:10CE70002046FFF7DEFE4DE723681F65BA0F2B4BF8
:10CE80001A6139462046FFF7D7FE59E763689A686A
:10CE900012F0030F3FF464AF196A01F00F015A6AF0
:10CEA000186A00F03008586A08EA00081F6A07F498
:10CEB000C077586A07401E6A06F4FC46586A064066
:10CEC0001D6A05F4F025586A0540D3F82490D3F87C
:10CED00020A011401CD1B8F1000F1ED119F0400F55
:10CEE00002D01AF0400F25D187BB36B163681E62AD
:10CEF000D4F89C301E43C4F89C60002D3FF430AF42
:10CF000063681D62D4F89C301D43C4F89C5027E729
:10CF100019622046FFF791FEDDE76368C3F82080C1
:10CF200041462046FFF78AFED8E700BF00A8004030
:10CF300000A000406368D96BDA6B4020186202F0F1
:10CF40003F02090C2046FFF77AFECDE763681F62B7
:10CF500039462046FFF774FEC7E72046FFF76BFE11
:10CF600003E700BFF0B482B000235FE086685F0093
:10CF70000325BD4026EA0506CD68BD4035438560E2
:10CF8000466826EA04064D68C5F300149C40344305
:10CF9000446059E0DD08083550F8257003F00704B7
:10CFA000A6000F24B44027EA04070C69B4403C43B0
:10CFB00040F825405CE0092400E00024B4403C43F4
:10CFC00002355C4E46F825404FF0B0442568D44306
:10CFD00025EA02064F6817F4801F01D042EA0506D1
:10CFE0004FF0B0452E606E6804EA06054F6817F4EE
:10CFF000001F01D042EA06054FF0B04675604E4D65
:10D000006D6804EA05064F6817F4003F01D042EA54
:10D010000506494D6E602D682C404E6816F4803F21
:10D0200001D042EA0504444A146001330A6832FA26
:10D0300003F47BD001249C402240F6D04D6805F0DB
:10D040000305013D012D91D94C6804F00304032C24
:10D0500009D0C5685E000324B44025EA04058C6845
:10D06000B4402C43C4604C6804F00304022C91D0FB
:10D0700005685E000324B44025EA04054C6804F00A
:10D080000304B4402C4304604C6814F4403FCCD0FB
:10D090002A4CD4F8F45045F00205C4F8F450D4F802
:10D0A000F44004F002040194019C9D08AE1C214C44
:10D0B00054F8267003F00304A6000F24B44027EAB6
:10D0C00004071F4CA0423FF478AF04F58064A042EF
:10D0D0001ED004F58064A0421CD004F58064A042F8
:10D0E0001AD004F58064A04218D004F58064A042F0
:10D0F00016D004F58064A04214D004F58064A042E8
:10D1000012D004F50064A0423FF455AF0A2455E75D
:10D11000012453E7022451E703244FE704244DE799
:10D1200005244BE7062449E7072447E702B0F0BC93
:10D13000704700BF000400588000005800440258A7
:10D14000000002580369194201D0012070470020F5
:10D1500070470AB18161704709048161704700001E
:10D1600000285DD010B5044690F84130002B46D021
:10D17000242384F841302268136823F001031360EC
:10D180006368226823F0706313612268936823F454
:10D1900000439360E368012B36D0A368226843F410
:10D1A00004439360E368022B34D02268536823F46D
:10D1B00000635360226851681A4B0B435360226826
:10D1C000D36823F40043D360236962691343A169E0
:10D1D000226843EA0123D360E369216A22680B4392
:10D1E00013602268136843F0010313600020606439
:10D1F000202384F84130206384F8420010BD80F879
:10D200004030FCF7C9FAB3E7A368226843F400434F
:10D210009360C7E72268536843F400635360C9E72B
:10D22000012070470080000290F84130DBB2202BD3
:10D2300024D190F84030012B22D0012380F84030D7
:10D24000242380F841300268136823F0010313603F
:10D250000268136823F4805313600268136819434B
:10D2600011600268136843F001031360202380F803
:10D270004130002380F84030184670470220704744
:10D280000220704790F84130DBB2202B22D190F879
:10D290004030012B20D0012380F84030242380F837
:10D2A00041300268136823F00103136002681368B9
:10D2B00023F4706343EA012111600268136843F0AC
:10D2C00001031360202380F84130002380F84030B0
:10D2D0001846704702207047022070472DE9F0473A
:10D2E00082B0D0F8008001EBC10300EB83039A6A9F
:10D2F0005B6A9A4255D807460C46C1469B1A01EB19
:10D30000C10200EB8202D2699A4200D31A4602F1AE
:10D31000030A4FEA9A0A15E006F1030A4FEA9A0A4D
:10D32000BB7904EBC40507EB8505296A0093B3B20A
:10D33000E2B2404605F0C1FB2B6A33442B62AB6A74
:10D340001E44AE6209EB441303F510639B699BB264
:10D35000534512D304EBC40207EB8202916A536A6D
:10D3600099420AD24BB15B1A04EBC40207EB82026A
:10D37000D6699E42D0D31E46CEE704EBC40007EB2D
:10D3800080077A6ABB6A9A420FD804F00F0401231F
:10D39000A340D8F8344824EA0304C8F834480020ED
:10D3A00000E0012002B0BDE8F0870020FAE730B5C8
:10D3B00083B0002879D0044690F89534ABB10323AC
:10D3C00084F89534206805F035F9237C8DF8003019
:10D3D000231D0ECB206805F063F858B1022384F8B2
:10D3E00095340125284603B030BD80F8943408F008
:10D3F0004BF9E4E70021206805F074FD0246B8B956
:10D400000346207998422FD903EBC30104EB810135
:10D41000012048750B75CB8500200876C86108622D
:10D4200003EBC30104EB810148620133DBB2E8E79F
:10D43000022384F895340125D4E702EBC20304EB00
:10D440008303002183F8551283F8542283F858127D
:10D45000C3F85C12C3F8601202EBC20304EB83034F
:10D46000C3F864120132D2B29042E6D8237C8DF820
:10D470000030231D0ECB206805F032F9054658B95F
:10D4800000236374012384F89534237B012B08D097
:10D49000206805F0E4FCA5E7022384F89534012513
:10D4A000A0E7204600F082FDF2E701259AE7036835
:10D4B00090F89424012A1AD010B50446012280F86D
:10D4C0009424DA6812F0400F02D0427B012A09D07E
:10D4D000206805F0A9F8206805F0B3FC002084F866
:10D4E000940410BD9A6B42F480329A63F0E70220F4
:10D4F0007047000070B504460D460068066C00EBEE
:10D50000411303F530639A68A179012911D0384994
:10D510008E4256D03DB905EBC50304EB8303D3F827
:10D520006432002B5ED0E9B2204608F0FFF80020FC
:10D5300070BD12F0080F09D02E498E42F7D912F4AF
:10D54000004FF4D04FF400429A60F0E712F0200F41
:10D5500002D020229A60EAE712F0280FE7D125498D
:10D560008E4206D912F4004F03D04FF400429A6065
:10D57000DDE705EBC50204EB8202D2F874121B69E9
:10D58000C3F31203CB1AC2F868327DB905EBC502AA
:10D5900004EB8202D2F864226AB105EBC50204EB07
:10D5A0008202D2F860120B44C2F86032E9B220461F
:10D5B00008F0BCF8BBE704F29C42012105F0D4FC62
:10D5C000F4E712F4004F03D04FF400429A60AEE744
:10D5D00012F0200F01D020229A60E9B2204608F014
:10D5E000A5F8A4E704F29C42002105F0BDFC9AE7EF
:10D5F0000A31544F0A30544F38B5044603681D6C45
:10D6000003EB4113D3F8081B0E4A954207D903F5E3
:10D61000306311F4004F02D04FF400429A6020466C
:10D6200008F07CF8074B9D4202D9A379012B01D069
:10D63000002038BD04F29C420121206805F094FCD2
:10D64000F6E700BF0A30544F90F89434012B0CD009
:10D6500010B50446012380F894344174006805F045
:10D66000E0FB002084F8940410BD02207047F8B558
:10D6700007460C4611F0800F27D101F00F0505EB8E
:10D68000C506B60006F514760644311D05EBC50542
:10D6900000EB8505002085F8550204F00F040C709E
:10D6A0008A600B714A7802B14C83022B1CD097F828
:10D6B0009434012B1BD0012387F89434386805F08B
:10D6C000E7F8002087F89404F8BD01F00F0000EBA4
:10D6D000C001890010313944043100EBC00007EB70
:10D6E000800001254575D8E700234B71DFE7022054
:10D6F000EAE710B504460A4611F0800F20D101F088
:10D700000F0000EBC0039B0003F514732344191DA5
:10D7100000EBC00004EB8000002380F8553202F0DB
:10D720000F020A7094F89434012B18D0012384F866
:10D730009434206805F0F4F8002084F8940410BDB7
:10D7400001F00F0000EBC0039B0010332344191DB0
:10D7500000EBC00004EB800001234375DFE70220EB
:10D76000EDE770B5164601F00F0404EBC401890023
:10D7700001F514710144043104EBC40500EB850587
:10D78000C5F86022C5F864320023C5F8683285F810
:10D79000553285F854428279012A04D0006805F098
:10D7A000A1F9002070BDC5F87062F7E701F00F0124
:10D7B00001EBC10100EB8101D1F86802704770B53F
:10D7C000164601F00F0404EBC40189001031014436
:10D7D000043104EBC40500EB85052A626B6200236B
:10D7E000AB6201236B752C7582799A4204D0006874
:10D7F00005F078F9002070BD2E63F8E738B501F028
:10D800000F050279AA4238D304460B4611F0800F67
:10D810001FD101EBC101890001F5147101440431EC
:10D8200003EBC30300EB8303002283F8552201239B
:10D830008B700D7094F89434012B20D0012384F860
:10D840009434206805F092FA85B1002084F894049D
:10D8500038BD05EBC501890010310144043105EBE9
:10D86000C50300EB830301225A75E0E704F29C42F2
:10D87000A179206805F078FBE7E70120E8E70220BE
:10D88000E6E701F00F0302799A4230D310B504465F
:10D8900011F0800F1ED103EBC301890001F5147153
:10D8A0000144043103EBC30200EB8202002082F842
:10D8B000550200228A700B7094F89434012B18D012
:10D8C000012384F89434206805F07DFA002084F860
:10D8D000940410BD03EBC3018900103101440431ED
:10D8E00003EBC30200EB820201205075E1E7012047
:10D8F00070470220EDE708B511F0800F0CD101F060
:10D900000F0101EBC101890001F5147101440431DB
:10D91000006805F073F808BD01F00F0101EBC101CB
:10D920008900103101440431F2E72DE9F04F83B052
:10D9300004460668304605F0D1FA10B103B0BDE8E0
:10D94000F08F35460746206805F097FA0028F5D095
:10D9500006F5006BDBF80830C3F30D23C4F8D434AC
:10D96000206805F08AFA10F0020F04D0226853698B
:10D9700003F002035361206805F07FFA10F0100FE6
:10D9800014D02268936923F010039361D6F82080A5
:10D9900008F00F09C8F34343022B6AD0062B00F0AE
:10D9A00090802268936943F010039361206805F02A
:10D9B00064FA10F4002F40F09680206805F05DFABC
:10D9C00010F4802F40F00281206805F056FA0028FC
:10D9D000C0F28681206805F050FA10F4006F0AD07A
:10D9E000DBF8083013F0010F40F09481226853698E
:10D9F00003F400635361206805F03FFA10F0006FF4
:10DA000015D02268536903F00063536194F8CC3455
:10DA1000002B40F08381012184F8CC1423685B6DD6
:10DA2000C3F38303C4F8D034204600F0D3FA20684F
:10DA300005F023FA10F4805F40F07481206805F04F
:10DA40001CFA10F4005F40F0CA81206805F015FA56
:10DA500010F0080F40F0DB81206805F00EFA10F09E
:10DA6000800F00F0EE81B36923F08003B3610127DA
:10DA7000DBE147F6F07318EA030F92D04FEA181370
:10DA800000934FEAC902019209EBC90A04EB8A0A22
:10DA9000C8F30A12DAF86012304605F041F9009B2B
:10DAA000C3F30A02DAF860321344CAF86032019B09
:10DAB0004B4404EB8303D3F868321A44CAF8682253
:10DAC0006FE7082204F29C41304605F029F9C8F3BB
:10DAD0000A1809EBC90204EB8202D2F86832434407
:10DAE000C2F868325DE7206805F0CBF98046B94698
:10DAF00035E005EB49130122C3F8082B49462046BF
:10DB0000FFF7F8FC3DE005EB49130822C3F8082BAA
:10DB100049462046FFF770FD36E009EBC90304EBE8
:10DB2000830393F85732012B44D005EB49130222AB
:10DB3000C3F8082B1AF0200F04D005EB491320225C
:10DB4000C3F8082B1AF4005F05D005EB49134FF416
:10DB50000052C3F8082B09F101094FEA5808B8F13F
:10DB6000000F3FF42AAF18F0010FF4D05FFA89F3E9
:10DB700000931946206805F094F9824610F0010FD1
:10DB8000B7D11AF0080FBED11AF0100F04D005EB70
:10DB900049131022C3F8082B1AF0020FCAD0736978
:10DBA00013F0800FB9D0DBF8043043F48063CBF876
:10DBB0000430B2E709EBC90304EB8303002283F8C6
:10DBC00057220099204607F001FEAEE7206805F0D5
:10DBD00060F98046B94625E00099204607F0B2FD7D
:10DBE0001AF0080F04D005EB49130822C3F80829DE
:10DBF0001AF0100F04D005EB49131022C3F80829BE
:10DC00001AF0400F04D005EB49134022C3F808294D
:10DC10001AF0020F43D11AF0800F5CD109F101090B
:10DC20004FEA5808B8F1000F3FF4CEAE18F0010FDC
:10DC3000F4D05FFA89F300931946206805F03AF9A9
:10DC4000824610F0010FCBD009F00F03012101FA39
:10DC500003F2DBF8343023EA0203CBF8343005EB6F
:10DC60004913C3F80819A3798B42B5D109EBC9034D
:10DC700004EB8303D9691A6A0A441A62B9F1000FE6
:10DC8000AAD109EBC90304EB83035B6A002BA3D180
:10DC900004F29C420121206805F066F99CE74946A0
:10DCA000304604F0CDFC09EBC90304EB8303DB7DB4
:10DCB000012B05D005EB49130222C3F80829AAE776
:10DCC00009EBC90304EB83030022DA7500992046AF
:10DCD00007F082FDEEE749462046FFF7FFFA9DE791
:10DCE000DBF8043023F00103CBF8043094F8CC3493
:10DCF000012B08D0204607F063FD2268536903F02A
:10DD00000043536166E6002184F8CC14204600F0FD
:10DD100061F9F2E7204607F03BFD67E6204607F091
:10DD200037FD84E6DBF8043023F00103CBF8043040
:10DD30001021206804F084FC1AE005EB47134FF62D
:10DD40007F31C3F80819D3F8002922F40012C3F870
:10DD50000029C3F8081BD3F8002B22F40012C3F8E3
:10DD6000002BD3F8002B42F00062C3F8002B0137E0
:10DD70002379BB42E1D8DBF81C3043F00113CBF828
:10DD80001C30E37BEBB1DBF8843043F00B03CBF8C2
:10DD90008430DBF8443043F00B03CBF84430D6F842
:10DDA000003823F4FE63C6F8003804F29C42A179DF
:10DDB000206805F0D9F82268536903F48053536151
:10DDC0003CE6DBF8142042F22B031343CBF814306B
:10DDD000DBF8103043F00B03CBF81030DFE720689E
:10DDE00005F0B2F8206804F043FDE071276800F008
:10DDF0005FFE0146E279384604F0A4FB204607F0B6
:10DE0000B2FC2268536903F4005353611DE62046B7
:10DE100007F0A3FC2268536903F0080353611BE673
:10DE2000F9B22046FFF767FD01372379BB4208D9D5
:10DE300007EBC70304EB830393F85732012BF3D1AD
:10DE4000EEE7206805F019F810F4801F3AD1206839
:10DE500005F013F810F4001F71D1206805F00DF8DB
:10DE600010F0804F6DD1206805F007F810F0040F16
:10DE70003FF464AD23685D6815F0040F6AD1226831
:10DE800053682B43536059E501372379BB421BD9B3
:10DE900005EB4713D3F8002907EBC70304EB830313
:10DEA0001B7E012BF0D1002AEEDA07EBC70304EB4F
:10DEB00083030122DA7567F07F01C9B22046FFF7BC
:10DEC0001AFDE1E70127E0E72268536903F48013B4
:10DED0005361BCE7013322799A422AD905EB4312F8
:10DEE000D2F8001B03EBC30204EB820292F8582223
:10DEF000012AEFD10029EDDA01F48031D4F8D424DD
:10DF000002F001029142E5D103EBC30204EB82026D
:10DF1000012182F85712B26942F08002B26172693F
:10DF200012F0800FD6D1DBF8043043F40073CBF845
:10DF300004302268536903F4001353618DE7012311
:10DF4000C9E7204607F04EFC2268536903F080437E
:10DF5000536188E7204607F04BFC90E730B4046833
:10DF6000606A19B940EA0240A06218E00D46A36A4F
:10DF700000EB13400023691E8B4209D203F14001DC
:10DF800004EB8101496800EB11400133DBB2F2E799
:10DF900040EA024005F13F0104EB810148600020A6
:10DFA00030BC70470368596200207047034602681E
:10DFB0000121C0F8D814002083F8CC04936943F001
:10DFC00000639361516D024B0B435365704700BF73
:10DFD0000300001070470000134BDB6813F0040FC0
:10DFE00007D1114BDB6803F0070383421AD00120ED
:10DFF000704710B50C4AD36823F007031843D0606C
:10E00000FCF754FD0446084B5B6813F4005F07D12E
:10E01000FCF74CFD001BB0F57A7FF4D9012000E03D
:10E02000002010BD0020704700480258024AD36803
:10E0300043F08073D360704700480258002800F016
:10E04000D78238B50446036813F0010F25D0AA4AD9
:10E05000136903F03803926A102B15D0182B0FD0D8
:10E060006368B3F5803F3FD0002B53D1A24B1A68B1
:10E0700022F480321A601A6822F480221A6038E092
:10E0800002F00302022AEBD19B4B1B6813F4003F02
:10E0900003D06368002B00F0AD82236813F0020FF9
:10E0A00000F08880944A1369926A13F038035AD0BA
:10E0B000182B55D0E368002B00F0A9808E490A6820
:10E0C00022F0190213430B60FCF7F0FC05468A4B63
:10E0D0001B6813F0040F40F09180FCF7E7FC401B35
:10E0E0000228F4D903208CE2834A136843F4803376
:10E0F000136063682BB3FCF7D9FC05467E4B1B68A5
:10E1000013F4003FC9D1FCF7D1FC401B6428F5D9BA
:10E11000032076E2B3F5A02F09D0774B1A6822F4DA
:10E1200080321A601A6822F480221A60E1E7724B8A
:10E130001A6842F480221A601A6842F480321A6027
:10E14000D7E7FCF7B3FC05466B4B1B6813F4003FA5
:10E15000A3D0FCF7ABFC401B6428F5D9032050E2A8
:10E1600012F0030FA6D1644B1B6813F0040F03D009
:10E17000E368002B00F040825F4A136823F0190324
:10E18000E1680B431360FCF791FC05465A4B1B6892
:10E1900013F0040F06D1FCF789FC401B0228F5D9C7
:10E1A00003202EE2544A536823F0FE43216943EAD8
:10E1B00001635360236813F0100F51D04E4A136966
:10E1C00003F03803926A082B39D0182B33D0E36957
:10E1D000002B68D0484A136843F080031360FCF7B3
:10E1E00065FC0546444B1B6813F4807F52D1FCF755
:10E1F0005DFC401B0228F5D9032002E23E4A536829
:10E2000023F0FE43216943EA01635360D2E73A4AAF
:10E21000136823F001031360FCF748FC0546364BF6
:10E220001B6813F0040FC5D0FCF740FC401B02280C
:10E23000F5D90320E5E102F00302012AC7D12E4BF4
:10E240001B6813F4807F03D0E369802B40F0D681F4
:10E25000294AD36823F07C53216A43EA0163D360DF
:10E26000236813F0080F49D0636983B3224A536FC0
:10E2700043F001035367FCF719FC05461E4B5B6F27
:10E2800013F0020F3AD1FCF711FC401B0228F5D91C
:10E290000320B6E1184AD36823F07C53216A43EA8D
:10E2A0000163D360DCE7144A136823F08003136032
:10E2B000FCF7FCFB0546104B1B6813F4807FCFD0A6
:10E2C000FCF7F4FB401B0228F5D9032099E10A4A28
:10E2D000536F23F001035367FCF7E8FB0546064B39
:10E2E0005B6F13F0020F09D0FCF7E0FB401B022824
:10E2F000F5D9032085E100BF00440258236813F0DC
:10E30000200F29D0A3699BB1A84A136843F4805316
:10E310001360FCF7CBFB0546A44B1B6813F4005FAE
:10E320001AD1FCF7C3FB401B0228F5D9032068E192
:10E330009E4A136823F480531360FCF7B7FB05462D
:10E340009A4B1B6813F4005F06D0FCF7AFFB401B31
:10E350000228F5D9032054E1236813F0040F21D1DA
:10E36000636A002B00F04C81904A126902F0380277
:10E37000182A00F0EA80022B75D08C4A136823F02B
:10E3800080731360FCF792FB0446884B1B6813F004
:10E39000007F00F0D880FCF789FB001B0228F4D92D
:10E3A00003202EE1824A136843F480731360FCF764
:10E3B0007DFB05467E4B1B6813F4807F06D1FCF77E
:10E3C00075FB401B6428F5D903201AE1A368012BD3
:10E3D0000AD00BBB754B1A6F22F001021A671A6F35
:10E3E00022F004021A6704E0704A136F43F001033D
:10E3F0001367A36833B3FCF759FB05466B4B1B6FE0
:10E4000013F0020FACD1FCF751FB401B41F28833F3
:10E410009842F3D90320F4E0052B09D0634B1A6F1F
:10E4200022F001021A671A6F22F004021A67E0E76D
:10E430005E4B1A6F42F004021A671A6F42F0010233
:10E440001A67D6E7FCF732FB0546584B1B6F13F0F3
:10E45000020F85D0FCF72AFB401B41F2883398421B
:10E46000F3D90320CDE0514A136823F08073136081
:10E47000FCF71CFB05464D4B1B6813F0007F06D0D4
:10E48000FCF714FB401B0228F5D90320B9E0474BE9
:10E49000996A484A0A40A16AE06A41EA00110A43BF
:10E4A0009A62226B013AC2F30802616B0139490298
:10E4B00089B20A43A16B0139090401F4FE010A4340
:10E4C000E16B0139090601F0FE410A431A63DA6A79
:10E4D00022F00102DA62596B374A0A40A16C42EA23
:10E4E000C1025A63DA6A22F00C02216C0A43DA6232
:10E4F000DA6A22F00202616C0A43DA62DA6A42F4F2
:10E500008032DA62DA6A42F40032DA62DA6A42F4BB
:10E510008022DA62DA6A42F00102DA621A6842F0B4
:10E5200080721A60FCF7C2FA0446204B1B6813F095
:10E53000007F06D1FCF7BAFA001B0228F5D90320A8
:10E540005FE000205DE000205BE018498A6A086B0C
:10E55000012B57D002F00303A16A8B4254D1C2F3BE
:10E560000512E36A9A4251D1C0F30802236B013BC2
:10E570009A424DD1C0F34622636B013B9A4249D186
:10E58000C0F30642A36B013B9A4245D1C0F306603B
:10E59000E36B013B984241D1044B5B6BC3F3CC036B
:10E5A000A26C9A420AD100202BE000BF004402581E
:10E5B000004802580CFCFFFF0700FFFF184AD36A0F
:10E5C00023F00103D362FCF771FA0546FCF76EFAFB
:10E5D000A842FBD0124A516B124B0B40A16C43EA8C
:10E5E000C1035363D36A43F00103D362002008E000
:10E5F00001207047012004E0012002E0012000E03A
:10E60000002038BD0120FCE70120FAE70120F8E7EF
:10E610000120F6E70120F4E70120F2E70120F0E70E
:10E62000004402580700FFFF744B1B6903F03803D6
:10E63000102B00F0DF80182B10D00BB17048704702
:10E640006E4B1B6813F0200F00F0D6806B4B1868E0
:10E65000C0F3C1006B4B23FA00F0704710B4674A57
:10E66000916A01F00301946AC4F30510D36A03F0C0
:10E670000103526BC2F3CC0203FB02F307EE903AA4
:10E68000F8EE677A14F47C7F00F09480012966D05C
:10E69000022900F09280E1B107EE100AF8EE476A15
:10E6A0009FED596A86EE267A544B1B6BC3F3080321
:10E6B00006EE903AF8EE666A9FED546A67EE867A47
:10E6C00076EEA77AF7EE006A77EEA67A27EE277A3B
:10E6D00061E04A4B1B6813F0200F23D047490A68BA
:10E6E000C2F3C102474BD34007EE103AF8EE476A37
:10E6F00007EE100AB8EE476A86EE867A0B6BC3F314
:10E70000080306EE903AF8EE666A9FED406A67EEFF
:10E71000867A76EEA77AF7EE006A77EEA67A27EE8B
:10E72000277A38E007EE100AF8EE476A9FED386A5C
:10E7300086EE267A314B1B6BC3F3080306EE903A44
:10E74000F8EE666A9FED316A67EE867A76EEA77A12
:10E75000F7EE006A77EEA67A27EE277A1BE007EE3F
:10E76000100AF8EE476A9FED286A86EE267A234B58
:10E770001B6BC3F3080306EE903AF8EE666A9FED52
:10E78000236A67EE867A76EEA77AF7EE006A77EE6E
:10E79000A67A27EE277A194B1B6BC3F34623013366
:10E7A00007EE903AF8EE677AC7EE276AFCEEE67A53
:10E7B00017EE900A5DF8044B704707EE100AF8EE6A
:10E7C000476A9FED146A86EE267A0C4B1B6BC3F3E7
:10E7D000080306EE903AF8EE666A9FED0C6A67EE63
:10E7E000867A76EEA77AF7EE006A77EEA67A27EEBB
:10E7F000277AD0E70848704702487047004402581B
:10E8000000093D000090D0030024744A0000003944
:10E810000024744C20BCBE4B40787D01002800F0E1
:10E82000328170B50D4604469B4B1B6803F00F0305
:10E830008B420BD2984A136823F00F030B431360EB
:10E84000136803F00F038B4240F01F81236813F01D
:10E85000040F0CD02269914B9B6903F070039A421C
:10E8600005D98E498B6923F070031A438A612368A6
:10E8700013F0080F0CD06269884BDB6903F070035A
:10E880009A4205D98549CB6923F070031A43CA61BE
:10E89000236813F0100F0CD0A269804BDB6903F4DE
:10E8A000E0639A4205D97D49CB6923F4E0631A43BA
:10E8B000CA61236813F0200F0CD0E269774B1B6A02
:10E8C00003F070039A4205D974490B6A23F0700370
:10E8D0001A430A62236813F0020F0CD0E2686F4BF0
:10E8E0009B6903F00F039A4205D96C498B6923F0A9
:10E8F0000F031A438A61236813F0010F41D0674A5E
:10E90000936923F47063A1680B4393616368022BDE
:10E910000AD0032B27D0012B2CD0604A126812F0AA
:10E92000040F06D10120ADE0126812F4003F00F0A0
:10E93000AE805A490A6922F0070213430B61FCF7C3
:10E94000B5F80646554B1B6903F038036268B3EB14
:10E95000C20F16D0FCF7AAF8801B41F28833984208
:10E96000F0D903208EE04D4A126812F0007FE0D10A
:10E97000012087E0494A126812F4807FD9D1012032
:10E9800080E0236813F0020F0CD0E268434B9B69D0
:10E9900003F00F039A4205D240498B6923F00F031D
:10E9A0001A438A613C4B1B6803F00F03AB420AD940
:10E9B000394A136823F00F032B431360136803F0E5
:10E9C0000F03AB4265D1236813F0040F0CD022690A
:10E9D000324B9B6903F070039A4205D22F498B6931
:10E9E00023F070031A438A61236813F0080F0CD0D8
:10E9F00062692A4BDB6903F070039A4205D227490A
:10EA0000CB6923F070031A43CA61236813F0100F17
:10EA10000CD0A269214BDB6903F4E0639A4205D272
:10EA20001E49CB6923F4E0631A43CA61236813F0DB
:10EA3000200F0CD0E269194B1B6A03F070039A4255
:10EA400005D216490B6A23F070031A430A62FFF7D6
:10EA5000EBFD12498B69C3F30323114AD35C03F026
:10EA60001F03D8408B6903F00F03D35C03F01F032F
:10EA700020FA03F30B4A13600B4B18600B4B18681A
:10EA8000FBF728F970BD012070470120FAE701204B
:10EA9000F8E70120F6E700BF0020005200440258CA
:10EAA0006825020808000024040000241000002447
:10EAB00008B5FFF7B9FD0B4A9369C3F303230A496D
:10EAC000CB5C03F01F0320FA03F3926902F00F02FC
:10EAD000885C00F01F0023FA00F0044A1060044A2A
:10EAE000136008BD0044025868250208080000248D
:10EAF0000400002408B5FFF7DBFF054BDB69C3F317
:10EB00000213044AD35C03F01F03D84008BD00BFC2
:10EB1000004402586825020808B5FFF7C9FF054BF5
:10EB2000DB69C3F30223044AD35C03F01F03D8401C
:10EB300008BD00BF00440258682502083F23036057
:10EB4000114B1A6902F0070242609A6902F470627E
:10EB500082609A6902F00F02C2609A6902F0700244
:10EB60000261DA6902F070024261DA6902F4E0627D
:10EB700082611B6A03F07003C361044B1B6803F0DE
:10EB80000F030B60704700BF004402580020005282
:10EB9000404B9B6A03F00303032B79D070B5054605
:10EBA0000E463C4A136823F080631360FBF77EFF38
:10EBB0000446384B1B6813F0006F06D0FBF776FF56
:10EBC000031B022BF5D9032070BD324B9A6A22F445
:10EBD0007C32296842EA01329A626A68013AC2F3D9
:10EBE0000802A9680139490289B20A43E968013972
:10EBF000090401F4FE010A4329690139090601F0FB
:10EC0000FE410A439A63DA6A22F0C00269690A4344
:10EC1000DA62DA6A22F02002A9690A43DA62DA6A61
:10EC200022F01002DA62D96B1B4A0A40E96942EA13
:10EC3000C102DA63DA6A42F01002DA62C6B91A4631
:10EC4000DB6A43F40023D362124A136843F0806303
:10EC50001360FBF72BFF04460E4B1B6813F0006F8D
:10EC600014D1FBF723FF001B0228F5D90320ABE7E3
:10EC7000012E05D0074AD36A43F40013D362E3E7B9
:10EC8000044AD36A43F48013D362DDE700209BE794
:10EC900001207047004402580700FFFF404B9B6A69
:10ECA00003F00303032B79D070B505460E463C4AAA
:10ECB000136823F080531360FBF7F8FE0446384BCB
:10ECC0001B6813F0005F06D0FBF7F0FE031B022B5E
:10ECD000F5D9032070BD324B9A6A22F07C72296804
:10ECE00042EA01529A626A68013AC2F30802A968CC
:10ECF0000139490289B20A43E9680139090401F47A
:10ED0000FE010A4329690139090601F0FE410A435F
:10ED10001A64DA6A22F4406269690A43DA62DA6ADA
:10ED200022F40072A9690A43DA62DA6A22F4807274
:10ED3000DA62596C1B4A0A40E96942EAC1025A6424
:10ED4000DA6A42F48072DA62C6B91A46DB6A43F4C0
:10ED50008003D362124A136843F080531360FBF7B9
:10ED6000A5FE04460E4B1B6813F0005F14D1FBF7A1
:10ED70009DFE001B0228F5D90320ABE7012E05D02C
:10ED8000074AD36A43F08073D362E3E7044AD36A45
:10ED900043F40003D362DDE700209BE701207047C6
:10EDA000004402580700FFFFF8B50446016801F06F
:10EDB00000620023134330D0436EB3F5001F26D00A
:10EDC0000ED8EBB1B3F5801F07D102210830FFF751
:10EDD000DFFE054645B12E4621E0012635461EE000
:10EDE000B3F5401F09D10025A84A136D23F4401341
:10EDF000616E0B431365002611E0012635460EE0D7
:10EE0000A24AD36A43F40033D3620025ECE702211F
:10EE10002830FFF743FF0546DCE70026354621682A
:10EE200001F480720023134314D0A36D042B37D850
:10EE3000DFE803F003282F080800944AD36A43F45C
:10EE40000033D3627DBB914A136D23F00703A16D9C
:10EE50000B431365216801F480620023134336D00D
:10EE6000D4F8A430B3F5800F55D021D8002B4CD066
:10EE7000B3F5001F19D1002104F10800FFF788FE47
:10EE800005461BE0002104F10800FFF781FE05465E
:10EE9000D8E7002104F12800FFF700FF0546D1E77D
:10EEA00001263546D6E72E46D4E7012635460EE044
:10EEB000B3F5000F02D0B3F5200F20D195BB734AF4
:10EEC000936D23F46003D4F8A4100B439365216879
:10EED00001F400620023134339D0D4F8A830B3F111
:10EEE000007F5CD023D8002B53D0B3F1807F1BD19F
:10EEF000002104F10800FFF74BFE05461DE0B3F5C5
:10EF0000C00FDBD001263546E1E7604AD36A43F4FF
:10EF10000033D362D2E7002104F12800FFF7BEFEE0
:10EF20000546CBE72E46D2E7012635460FE0B3F182
:10EF3000806F02D0B3F1A06F25D1002D36D1534A96
:10EF4000936D23F0E063D4F8A8100B439365216818
:10EF500001F000720023134331D0E36C202B45D025
:10EF600029D833B1102B23D1484AD36A43F4003354
:10EF7000D362002D41D1454AD36C23F03003E16CBC
:10EF80000B43D3641BE0B3F1407FD6D00126354656
:10EF9000DDE73E4AD36A43F40033D362CDE7002174
:10EFA00004F12800FFF77AFE0546C6E72E46CEE7B5
:10EFB0000126354603E0302BDBD00126354621689B
:10EFC00001F48052002313432BD0E36DB3F5005FAF
:10EFD0004FD017D8002B46D0B3F5805F0FD100215A
:10EFE00004F10800FFF7D4FD054611E0022104F109
:10EFF0000800FFF7CDFD0546BBE72E46DFE70126FB
:10F0000035460EE0B3F5405F02D0B3F5804F27D10F
:10F01000002D35D11D4A136D23F4E043E16D0B4300
:10F020001365216801F40052002313433BD0236E83
:10F03000B3F5003F58D02BD843B1B3F5803F21D171
:10F04000012104F10800FFF7A3FD0546002D52D170
:10F050000E4A136D23F4E023216E0B43136522E067
:10F0600001263546DDE7094AD36A43F40033D3620B
:10F07000CEE7002104F12800FFF710FE0546C7E7A0
:10F080002E46CEE7012635460DE000BF004402586B
:10F09000B3F5802FDAD0B3F5A02FD7D0B3F5403F2A
:10F0A000D4D001263546216801F480420023134361
:10F0B00031D0D4F8AC30B3F1005F49D020D843B19F
:10F0C000B3F1805F19D1012104F10800FFF760FD61
:10F0D0000546002D43D1954A936D23F0E043D4F8C3
:10F0E000AC100B43936516E0012104F12800FFF7F3
:10F0F000D5FD0546AAE72E46D5E7012635460AE0A6
:10F10000B3F1804FE5D0B3F1A04FE2D0B3F1405F4F
:10F11000DFD001263546216801F400420023134365
:10F1200009D0E36EB3F1805F1BD0B3F1005F26D04E
:10F13000E3B101263546216801F0807200231343B4
:10F140003FD0A36C032B38D8DFE803F02722302709
:10F15000012104F12800FFF7A1FD0546B9E72E467D
:10F16000D9E7724AD36A43F40033D36275B96F4A60
:10F17000136D23F04053E16E0B431365DBE7012170
:10F1800004F10800FFF704FD0546EFE72E46D2E73D
:10F19000664AD36A43F40033D3628DB9634AD36CB1
:10F1A00023F00303A16C0B43D3640AE0022104F1B2
:10F1B0000800FFF7EDFC0546EFE70126354600E0C5
:10F1C0002E46216801F480020023134321D12168D7
:10F1D00001F001020023134300F09780A36F282B56
:10F1E00000F29180DFE803F07F8F8F8F8F8F8F8FFA
:10F1F000798F8F8F8F8F8F8F888F8F8F8F8F8F8F3C
:10F200007F8F8F8F8F8F8F8F7F8F8F8F8F8F8F8F2E
:10F210007F00474A136843F480731360FBF746FC92
:10F220000746434B1B6813F4807F05D1FBF73EFC78
:10F23000C01B6428F5D90325002D4AD13B4B1B6F19
:10F24000D4F8B020534013F4407F0CD0374B1A6FE2
:10F2500022F44072196F41F480311967196F21F45B
:10F26000803119671A67D4F8B030B3F5807F15D0B4
:10F270008DBBD4F8B03003F44072B2F5407F1ED09D
:10F280002A4A136923F47C53136128490B6FD4F87D
:10F29000B020C2F30B0213430B6798E7FBF706FCA1
:10F2A0000746224B1B6F13F0020FE1D1FBF7FEFB69
:10F2B000C01B41F288339842F3D90325D8E71B4895
:10F2C000026922F47C521B4901EA131313430361C0
:10F2D000DBE72E467BE72E4679E7012104F10800A3
:10F2E000FFF756FC0546F5B9104A536D23F0380375
:10F2F000A16F0B43536508E0012104F12800FFF7DB
:10F30000CDFC0546EFE701263546216801F00202F3
:10F31000002313432AD0636F052B23D8DFE803F0C3
:10F32000120C1B1212122E46EFE700BF00440258C7
:10F3300000480258CFFFFF00012104F10800FFF749
:10F3400027FC05468DB9B54A536D23F00703616F5D
:10F350000B4353650AE0012104F12800FFF79EFCEE
:10F360000546EFE70126354600E02E46216801F00C
:10F3700004020023134323D0D4F89030052B1BD86C
:10F38000DFE803F0090313090909012104F108006A
:10F39000FFF7FEFB054695B9A04A936D23F00703DE
:10F3A000D4F890100B4393650AE0012104F1280082
:10F3B000FFF774FC0546EEE70126354600E02E46D1
:10F3C000216801F020020023134328D0D4F88C30A8
:10F3D000B3F1005F44D017D843B1B3F1805F10D1CF
:10F3E000002104F10800FFF7D3FB0546002D3ED1B4
:10F3F0008A4A536D23F0E043D4F88C100B435365D5
:10F400000DE0012635460AE0B3F1804FEED0B3F1AE
:10F41000A04FEBD0B3F1405FE8D00126354621681C
:10F4200001F040020023134331D0D4F89830B3F5F3
:10F43000006F4FD020D843B1B3F5806F19D10021B0
:10F4400004F10800FFF7A4FB0546002D49D1734ADB
:10F45000936D23F4E053D4F898100B43936516E0B2
:10F46000022104F12800FFF719FC0546BEE72E46ED
:10F47000D5E7012635460AE0B3F5805FE5D0B3F560
:10F48000A05FE2D0B3F5406FDFD00126354621689A
:10F4900001F080020023134333D0D4F89C30B3F53D
:10F4A000804F00F0B28021D843B1B3F5005F1AD18C
:10F4B000002104F10800FFF76BFB0546002D40F02A
:10F4C000AB80564A936D23F46043D4F89C100B43F1
:10F4D000936516E0022104F12800FFF7DFFB0546E3
:10F4E000B3E72E46D3E7012635460AE0B3F5004FD1
:10F4F000E4D0B3F5204FE1D0B3F5C04FDED0012604
:10F500003546216801F00802002313430DD0D4F8DA
:10F510008030B3F5805F00F08380404A536D23F460
:10F520004053D4F880100B435365216801F010025A
:10F53000002313430CD0D4F89430B3F5807F79D0F6
:10F54000364A936D23F44073D4F894100B439365BB
:10F55000216801F40022002313430CD0D4F8A0301A
:10F56000B3F5803F00F08080B3F5003F72D0002BF0
:10F570006AD001263546216801F480220023134316
:10F580000DD0D4F88430B3F5001F00F08580B3F5BA
:10F59000401F77D0B3F5801F6FD001263546216814
:10F5A00001F480320023134308D0236D002B7CD05C
:10F5B000B3F5803F00F0878001263546216801F0D1
:10F5C00000520023134340F08780216801F4003289
:10F5D0000023134300F08D80E36FB3F5807F00F0CC
:10F5E000F78040F28380B3F5007F03D0B3F5407F0E
:10F5F00040F0EC80002D40F0F180084A536D23F478
:10F600004073E16F0B43536573E0022104F128005E
:10F61000FFF744FB054651E72E4672E700440258C7
:10F62000022104F12800FFF739FB00283FF475AFF1
:10F63000012672E7022104F12800FFF72FFB0028C2
:10F640003FF47EAF01267BE7002104F10800FFF7BD
:10F650009FFA05467DB97D4A936D23F44033D4F873
:10F66000A0100B43936586E7022104F12800FFF701
:10F6700015FB0546EEE72E467DE7744AD36A43F450
:10F680000033D3627DB9714A536D23F44013D4F82B
:10F6900084100B43536582E7012104F12800FFF732
:10F6A000FDFA0546EEE72E4679E7684AD36A43F449
:10F6B0000033D36275B9654AD36C23F48033216D6E
:10F6C0000B43D3647AE7022104F10800FFF760FAE4
:10F6D0000546EFE72E4671E7022104F12800FFF707
:10F6E000DDFA00283FF471AF01266EE7002B81D0D0
:10F6F0000126216801F480120023134306D0534AE7
:10F70000136D23F00043216F0B431365216801F44F
:10F7100000120023134306D04C4A136D23F080736C
:10F72000A16E0B431365216801F08042002313434F
:10F7300009D0464B1A6922F400421A611A69D4F8BA
:10F74000B4100A431A61216801F0004200231343F8
:10F7500006D03E4AD36C23F04053616D0B43D36413
:10F76000216801F400020023134307D0374A536D88
:10F7700023F44003D4F888100B43536561680022DA
:10F7800001F0010313432BD16168002201F0020351
:10F7900013432ED16168002201F00403134331D1D9
:10F7A0006168002201F00803134334D1616800222C
:10F7B00001F01003134337D16168002201F02003E8
:10F7C00013433AD106B101263046F8BD012690E731
:10F7D0001E4AD36A43F40033D3620BE72E4688E710
:10F7E000002104F10800FFF7D3F90028CCD0064629
:10F7F000CAE7012104F10800FFF7CAF90028C9D0BF
:10F800000646C7E7022104F10800FFF7C1F9002806
:10F81000C6D00646C4E7002104F12800FFF73EFAEF
:10F820000028C3D00646C1E7012104F12800FFF7F4
:10F8300035FA0028C0D00646BEE7022104F12800B0
:10F84000FFF72CFA0028BDD00646BBE7004402585B
:10F8500008B5FFF72DF9054B1B6AC3F30213044AE1
:10F86000D35C03F01F03D84008BD00BF004402581A
:10F870006825020830B4784A916A946AC4F3053561
:10F88000D36AC3F30013D26BC2F3CC0203FB02F3BF
:10F8900014F47C3F00F0DA8001F0030107EE903AA7
:10F8A000F8EE677A012966D0022900F0B280E1B152
:10F8B00007EE105AB8EE477A9FED686AC6EE076AFF
:10F8C000654B9B6BC3F3080307EE103AB8EE477A1B
:10F8D0009FED636A67EE867A77EE277AB7EE007A55
:10F8E00077EE877A66EEA76A61E05B4B1B6813F0E0
:10F8F000200F23D058490A68C2F3C102594BD340A4
:10F9000007EE103AB8EE477A06EE905AB8EE666AFD
:10F91000C7EE066A8B6BC3F3080307EE103AB8EE26
:10F92000477A9FED4F6A67EE867A77EE277AB7EED1
:10F93000007A77EE877A66EEA76A38E007EE105A0B
:10F94000B8EE477A9FED486AC6EE076A424B9B6B5A
:10F95000C3F3080307EE103AB8EE477A9FED406A0A
:10F9600067EE867A77EE277AB7EE007A77EE877AB7
:10F9700066EEA76A1BE007EE105AB8EE477A9FEDD5
:10F98000376AC6EE076A344B9B6BC3F3080307EE76
:10F99000103AB8EE477A9FED326A67EE867A77EED4
:10F9A000277AB7EE007A77EE877A66EEA76A2A4A58
:10F9B000936BC3F3462307EE103AB8EE477AB7EEDF
:10F9C000006A37EE067AC6EE877AFCEEE77AC0ED7B
:10F9D000007A936BC3F3064307EE103AB8EE477A0A
:10F9E00037EE067AC6EE877AFCEEE77AC0ED017A4A
:10F9F000936BC3F3066307EE903AF8EE677A77EEFF
:10FA0000867A86EEA77ABCEEC77A80ED027A30BCA1
:10FA1000704707EE105AB8EE477A9FED146AC6EEAB
:10FA2000076A0D4B9B6BC3F3080307EE103AB8EE61
:10FA3000477A9FED0B6A67EE867A77EE277AB7EE04
:10FA4000007A77EE877A66EEA76AB0E70023036054
:10FA500043608360DBE700BF004402580024744A1F
:10FA6000000000390090D0030024744C20BCBE4B31
:10FA700030B4784A916A946AC4F30555D36AC3F3E3
:10FA80000023526CC2F3CC0203FB02F314F07C7F20
:10FA900000F0DA8001F0030107EE903AF8EE677AA1
:10FAA000012966D0022900F0B280E1B107EE105AB8
:10FAB000B8EE477A9FED686AC6EE076A654B1B6C25
:10FAC000C3F3080307EE103AB8EE477A9FED636A76
:10FAD00067EE867A77EE277AB7EE007A77EE877A46
:10FAE00066EEA76A61E05B4B1B6813F0200F23D022
:10FAF00058490A68C2F3C102594BD34007EE103A85
:10FB0000B8EE477A06EE905AB8EE666AC7EE066A15
:10FB10000B6CC3F3080307EE103AB8EE477A9FED7B
:10FB20004F6A67EE867A77EE277AB7EE007A77EE3D
:10FB3000877A66EEA76A38E007EE105AB8EE477A81
:10FB40009FED486AC6EE076A424B1B6CC3F308037D
:10FB500007EE103AB8EE477A9FED406A67EE867A74
:10FB600077EE277AB7EE007A77EE877A66EEA76AA5
:10FB70001BE007EE105AB8EE477A9FED376AC6EEE3
:10FB8000076A344B1B6CC3F3080307EE103AB8EE58
:10FB9000477A9FED326A67EE867A77EE277AB7EE7C
:10FBA000007A77EE877A66EEA76A2A4A136CC3F367
:10FBB000462307EE103AB8EE477AB7EE006A37EE02
:10FBC000067AC6EE877AFCEEE77AC0ED007A136C0F
:10FBD000C3F3064307EE103AB8EE477A37EE067ADB
:10FBE000C6EE877AFCEEE77AC0ED017A136CC3F3B8
:10FBF000066307EE903AF8EE677A77EE867A86EE3D
:10FC0000A77ABCEEC77A80ED027A30BC704707EE67
:10FC1000105AB8EE477A9FED146AC6EE076A0D4B8C
:10FC20001B6CC3F3080307EE103AB8EE477A9FED5A
:10FC30000B6A67EE867A77EE277AB7EE007A77EE70
:10FC4000877A66EEA76AB0E70023036043608360AB
:10FC5000DBE700BF004402580024744A000000396A
:10FC60000090D0030024744C20BCBE4B10B402683A
:10FC70005369916941F00801916101688A6942F014
:10FC800010028A6101680A6822F001020A600168B4
:10FC90000C69294A22400A6101688A6822F44042BC
:10FCA0008A6090F88120D2B2042A0DD013F0200F80
:10FCB0000AD0D0F8842042F08002C0F88420016885
:10FCC0008A6942F020028A6190F88120D2B2032A28
:10FCD0000DD013F0400F0AD0D0F8842042F0040277
:10FCE000C0F8842001688A6942F040028A6113F4F6
:10FCF000007F0AD0D0F8842042F00102C0F88420AE
:10FD000001688A6942F400728A6113F4807F0AD024
:10FD1000D0F8843043F00803C0F884300268936957
:10FD200043F4807393610023A0F86230A0F86A3036
:10FD30005DF8044B704700BF90FCFFFFC36B5B098D
:10FD4000C0680830C00803FB00007047002800F0BE
:10FD5000B78070B504460023836205685C4B5D4E36
:10FD60009D4218BFB54214BF0126002607D0A3F557
:10FD700074439D4203D0C3680F2B00F2A38020463A
:10FD8000FFF7DCFF2EB1544B9D4202D0082800F251
:10FD90009B804F4A4F4B9D4218BF954203D003F5BD
:10FDA00080639D4202D1102800F2908094F8813047
:10FDB000F3B1022384F881302268136823F0010331
:10FDC000136021688A6802F4F812A369B3F1806FA6
:10FDD00014D0636813F4800F23D0E368062B20D976
:10FDE00021680B6823F48073206D03430B601DE0D2
:10FDF00084F880302046F9F755FEDAE76368B3F5FA
:10FE0000800F06D0002BE4D1A36BB3F1805FE0D16B
:10FE100002E0A06B0028F5D10B6843F480530B601F
:10FE2000D7E721680B6823F480730B60E369A16A4C
:10FE30000B431343E26B1343E16822680B43936067
:10FE4000636B626A1343A26B1343A2691343226973
:10FE5000134362691343226A134362681343E26CDB
:10FE60001343A2681343A26C1343A16D22680B4392
:10FE7000D36063686BB92268936823F4C05343F47A
:10FE8000006393602268936823F4C06343F4806343
:10FE900093602268136D23F001031365636813F404
:10FEA000800F06D02268D36823F00043616D0B43B6
:10FEB000D3600020C4F88400012384F8813070BD31
:10FEC000012070470120FAE70120F8E70120F6E75A
:10FED0000030014000380040003C0040704770474F
:10FEE00008B5806B0023A0F86A30A0F862300123C7
:10FEF00080F88130FFF7F3FF08BD70472DE9F84324
:10FF0000044606683269736902EA0305D6F8089068
:10FF100090F88170FFB213F4006F02D012F0080F56
:10FF20003FD105F06403042B42D0002305F04508BF
:10FF3000B8F1010F44D005F02602022A45D0002B6B
:10FF400046D115F0080F79D02268936943F0080371
:10FF500093612268936943F0100393612268936967
:10FF600043F4006393612268136923F0080313616B
:10FF700023689B6813F4404F3BD02046FFF776FE82
:10FF8000012384F88130D4F88430002B4AD1052F26
:10FF90004CD0042F4ED0032F1AD12046FFF79EFFDE
:10FFA00016E0B36943F40063B361FFF7A6FF0FE007
:10FFB000636F20469847236F204698470123B5E793
:10FFC000236F204698474346B5E7636F204698471E
:10FFD000BDE8F883072B1CD9636E328E1A80636EDE
:10FFE00002336366B4F86A309BB2013B9BB2A4F85B
:10FFF0006A30B4F86A309BB2002BBED0E3680F2B96
:020000040801F1
:10000000E8D92268636E126B1A60636E043363660C
:10001000E8E72268636E92F830201A70636E01334D
:100020006366DFE72046FFF75AFFD1E7204607F077
:1000300063F8CDE7204607F037F8C9E715F4587F95
:10004000C6D015F0400F0AD0D4F8843043F0040332
:10005000C4F884302268936943F04003936115F437
:10006000007F0AD0D4F8843043F00103C4F8843010
:100070002268936943F40073936115F4807F0AD07A
:10008000D4F8843043F00803C4F8843022689369BC
:1000900043F48073936115F0200F0AD0D4F88430B4
:1000A00043F08003C4F884302268936943F020034E
:1000B0009361D4F88430002B8AD02268136823F02F
:1000C00001031360226811691A4B0B40136109F494
:1000D0004049B9F5404F25D12268936823F4404345
:1000E0009360E36F5BB1144A1A65E06FFBF754FC51
:1000F00028B1D4F8843043F04003C4F88430A36FAF
:10010000002B3FF465AF0C4A1A65A06FFBF744FC67
:1001100000283FF45DAFD4F8843043F04003C4F8C6
:10012000843055E7012384F881302046FFF7D7FE5D
:100130004EE700BF94FCFFFFE1FE0008F0B4036A45
:10014000026A22F001020262446885691E4A2A405E
:100150000E68164323F002038D682B431B4A1C4D87
:10016000A84218BF90420CBF012200220CD005F516
:100170008045A84214BF00250125164FB84203D080
:1001800015B9154DA84205D123F00803CD682B43BE
:1001900023F004035AB9114A904214BF00220122ED
:1001A0000C4DA84203D012B90B4A904205D124F459
:1001B00040724C6914438A691443446086614A68FA
:1001C00042630362F0BC70478CFFFEFF00000140F9
:1001D000000401400040014000480140004401404B
:1001E00070B4036A026A22F4807202624468C569CC
:1001F0001A4A2A400E68164323F400738A6843EAB9
:100200000223174A174DA84218BF90420CBF012283
:10021000002206D123F40063CD6843EA052323F4CA
:1002200080635AB9104A904214BF002201220F4D38
:10023000A84203D012B90E4A904207D124F4405488
:100240004A6944EA02148A6944EA02144460C661B5
:100250004A68C263036270BC704700BF8CFFFEFF38
:100260000000014000040140004401400040014002
:100270000048014070B4036A026A22F480520262AC
:100280004468C569144A2A400D6842EA052223F4ED
:1002900000538D6843EA0533104E114DA84218BF34
:1002A000B0420DD005F58045A84214BF00250125B8
:1002B00006F58046B04203D015B90A4DA84204D1D4
:1002C00024F480444D6944EA85144460C2614A685C
:1002D0000264036270BC7047FF8CFFFE00000140A7
:1002E000000401400048014070B4036A026A22F42D
:1002F000803202624268456D144C2C400D682C43DC
:1003000023F400338D6843EA0543114E114DA84292
:1003100018BFB0420DD005F58045A84214BF002596
:10032000012506F58046B04203D015B90A4DA84212
:1003300004D122F480324D6942EA052242604465CC
:100340004A688265036270BC704700BF8FFFFEFF82
:1003500000000140000401400048014070B4036AFD
:10036000026A22F4801202624468456D144A2A40EF
:100370000D6842EA052223F400138D6843EA055311
:10038000104E114DA84218BFB0420DD005F5804562
:10039000A84214BF0025012506F58046B04203D0CF
:1003A00015B90A4DA84204D124F480244D6944EAC9
:1003B0008524446042654A68C265036270BC704728
:1003C000FF8FFFFE00000140000401400048014093
:1003D00030B4036A056A25F001050562846924F0DA
:1003E000F00444EA021423F00A030B43846103621D
:1003F00030BC704730B4036A056A25F01005056209
:10040000846924F4704444EA023423F0A00343EAEC
:1004100001138461036230BC7047000090F83D30E6
:10042000DBB2012B42D1022380F83D300268D36851
:1004300043F00103D36003681E4AB3F1804F18BF35
:10044000934225D0A2F57C42934221D002F58062EE
:1004500093421DD002F58062934219D002F5784292
:10046000934215D0A2F56C42934211D002F594321A
:1004700093420DD0A2F5C042934209D002F58062AA
:10048000934205D01A6842F001021A6000207047BA
:100490009968094A0A40062A18BFB2F5803F07D07A
:1004A0001A6842F001021A6000207047012070476C
:1004B00000207047000001400700010070477047AE
:1004C000704770B504460368DE681D6915F0020FB9
:1004D00010D016F0020F0DD06FF002021A61012346
:1004E000037703689B6913F0030F64D0FFF7E7FFFE
:1004F0000023237715F0040F12D016F0040F0FD04D
:1005000023686FF004021A610223237723689B6932
:1005100013F4407F55D02046FFF7D1FF0023237707
:1005200015F0080F12D016F0080F0FD023686FF0E7
:1005300008021A61042323772368DB6913F0030F91
:1005400046D02046FFF7BBFF0023237715F0100F9E
:1005500012D016F0100F0FD023686FF010021A613E
:10056000082323772368DB6913F4407F37D02046C4
:10057000FFF7A5FF0023237715F0010F02D016F037
:10058000010F33D115F4025F02D016F0800F35D180
:1005900015F4807F02D016F0800F37D115F0400F90
:1005A00002D016F0400F39D115F0200F02D016F00E
:1005B000200F3BD170BDFFF781FF204606F0A2FC63
:1005C00096E72046FFF77AFF204606F09BFCA5E75A
:1005D0002046FFF773FF204606F094FCB4E7204660
:1005E000FFF76CFF204606F08DFCC3E723686FF031
:1005F00001021A612046F9F747F9C3E723686FF44F
:1006000002521A61204600F04CFCC1E723686FF4E7
:1006100080721A61204600F045FCBFE723686FF046
:1006200040021A612046FFF74BFFBDE723686FF0D9
:1006300020021A61204600F033FCBBE770B4036867
:10064000404CA04214BF00240124B0F1804F14BFDD
:10065000224644F00102AAB93B4DA84214BF00252E
:1006600001253A4EB0420DD065B905F1804505F53A
:100670008235A84214BF0025012506F50066B04268
:1006800000D01DB123F070034D682B4362BB2E4A8E
:10069000904214BF002201222C4DA84224D01ABB44
:1006A00002F1804202F58232904214BF0022012200
:1006B00005F50065A84217D0B2B9254A904214BF8B
:1006C0000022012205F59A35A8420DD062B9214ACF
:1006D000904214BF0022012205F50065A84203D014
:1006E00012B91D4A904203D123F44073CA681343E0
:1006F00023F080034A69134303608A68C2620A6870
:100700008262164B984214BF234644F001035BB942
:100710000F4B984214BF00230123114A904203D08B
:1007200013B9104B984201D10B6903630123436154
:10073000036913F0010F03D0036923F00103036180
:1007400070BC7047000001400008004000040040F9
:100750000044014000E0004000E40040000401408B
:10076000004001400048014060B310B5044690F8D5
:100770003D3013B3022384F83D30214651F8040B79
:10078000FFF75CFF012384F8483084F83E3084F89A
:100790003F3084F8403084F8413084F8423084F8A7
:1007A000433084F8443084F8453084F8463084F887
:1007B000473084F83D30002010BD80F83C30F9F718
:1007C00045FCD7E70120704760B310B5044690F8A8
:1007D0003D3013B3022384F83D30214651F8040B19
:1007E000FFF72CFF012384F8483084F83E3084F86A
:1007F0003F3084F8403084F8413084F8423084F847
:10080000433084F8443084F8453084F8463084F826
:10081000473084F83D30002010BD80F83C30F9F7B7
:1008200053FCD7E70120704770B4036A026A22F0D4
:1008300010020262446885691A4A2A400E6842EA38
:10084000062623F020038A6843EA0213164A174D4E
:10085000A84218BF90420CBF0122002206D123F00B
:100860008003CD6843EA051323F040035AB9104AC8
:10087000904214BF002201220E4DA84203D012B9AB
:100880000D4A904207D124F440644A6944EA820444
:100890008A6944EA8204446086614A68826303622A
:1008A00070BC7047FF8CFFFE000001400004014057
:1008B00000440140004001400048014038B590F834
:1008C0003C30012B00F0958004460D46012380F852
:1008D0003C30142A00F28880DFE802F00B8686861E
:1008E0001F86868634868686488686865D868686C8
:1008F00071000068FFF722FC2268936943F0080347
:1009000093612268936923F00403936122689369D9
:1009100029690B439361002067E00068FFF784FFBB
:100920002268936943F4006393612268936923F416
:100930008063936122689369296943EA0123936183
:10094000002052E00068FFF74BFC2268D36943F0B7
:100950000803D3612268D36923F00403D3612268BA
:10096000D36929690B43D36100203EE00068FFF79B
:1009700081FC2268D36943F40063D3612268D369A0
:1009800023F48063D3612268D369296943EA012390
:10099000D361002029E00068FFF7A6FC2268536DB0
:1009A00043F0080353652268536D23F00403536535
:1009B0002268536D29690B435365002015E00068D8
:1009C000FFF7CCFC2268536D43F400635365226843
:1009D000536D23F4806353652268536D296943EA9C
:1009E00001235365002000E00120002384F83C30FF
:1009F00038BD0220FCE710B4846824F47F4442EA46
:100A000003220A43224382605DF8044B70470000D2
:100A100010B50468A3684C4A1A404B6813434B4A0C
:100A20001A400B681343A3604B68602B68D01CD836
:100A3000402B50D008D9502B15D10A69896800681D
:100A4000FFF7C6FC002035E0202B60D003D9302B07
:100A500007D001202EE0002B5BD0102B5BD10020B3
:100A600028E0002026E0012024E0702B2BD001D2CA
:100A700001201FE0364A93424FD008D9B3F5001F3A
:100A800057D018D9334A934259D1002012E0303A56
:100A9000934244D007D9304A934246D01032934211
:100AA00045D1002006E0B3F5801F3AD0B3F1101F06
:100AB00039D1002010BD294A93423CD010329342D4
:100AC0003BD10020F6E70B698A68C9680068FFF728
:100AD00092FF0020EEE70B68052B32D003681C6AFA
:100AE0001A6A22F001021A620268936923F0F00385
:100AF000096943EA0113936103681C620020D9E786
:100B00000A6989680068FFF775FC0020D2E70020B9
:100B1000D0E70020CEE70120CCE70020CAE7002084
:100B2000C8E70020C6E70120C4E70020C2E7012093
:100B3000C0E70020BEE70020BCE70120BAE70120A3
:100B4000B8E70120B6E700BF8FFFCFFFF8FFFEFF39
:100B50005000100010002000300010006000100055
:100B600090F83C30012B22D010B50446012380F8C8
:100B70003C30022380F83D30FFF74AFF80B92268FD
:100B8000D36823F04003D3602268D36823F4804302
:100B9000D360012384F83D30002384F83C3010BD3D
:100BA000012084F83D00002384F83C30F7E7022060
:100BB000704710B401F01F01012303FA01F4036A26
:100BC00023EA04030362036A02FA01F10B4303629E
:100BD0005DF8044B7047000010B504460846002934
:100BE00056D194F83E30DBB2013B18BF0123002BF5
:100BF00040F0A380002876D1022384F83E30012201
:100C000001462068FFF7D5FF23684E494E4A9342BC
:100C100018BF8B420BD002F57052934207D002F5F9
:100C20008062934203D002F58062934203D15A6CF2
:100C300042F400425A642368424AB3F1804F18BF1D
:100C400093426CD0A2F57C42934268D002F5806258
:100C5000934264D002F58062934260D002F57842FC
:100C600093425CD0A2F56C42934258D002F5943284
:100C7000934254D0A2F5C042934250D002F5806214
:100C800093424CD01A6842F001021A60002055E0ED
:100C900004290CD0082911D00C2916D010291BD0FA
:100CA00094F84330DBB2013B18BF01239FE794F86F
:100CB0003F30DBB2013B18BF012398E794F8403086
:100CC000DBB2013B18BF012391E794F84130DBB25E
:100CD000013B18BF01238AE794F84230DBB2013BA5
:100CE00018BF012383E7042809D008280BD00C285B
:100CF0000DD010280FD0022384F843307FE7022361
:100D000084F83F307BE7022384F8403077E7022302
:100D100084F8413073E7022384F842306FE7996822
:100D20000A4A0A40062A18BFB2F5803F07D01A685F
:100D300042F001021A60002000E0012010BD0020F6
:100D4000FCE700BF00000140000401400700010073
:100D500090F83C30012B4DD070B4012380F83C302A
:100D6000022380F83D3003685A689D68224E234C68
:100D7000A34218BFB34203D122F470024C6822434D
:100D800022F070020C6822435A6003681A4AB3F1D9
:100D9000804F18BF93421FD0A2F57C4293421BD0D4
:100DA00002F58062934217D002F58062934213D01D
:100DB00002F5784293420FD0A2F56C4293420BD0D9
:100DC00002F59432934207D0A2F5C042934203D079
:100DD00002F58062934204D125F080058A681543AC
:100DE0009D60012380F83D30002380F83C30184698
:100DF00070BC7047022070470000014000040140B1
:100E000090F83C30012B44D030B4012380F83C30C2
:100E1000CB6823F440738A68134323F480634A68E1
:100E2000134323F400630A68134323F480530A69CD
:100E3000134323F400534A69134323F480430A6B9A
:100E4000134323F470238A6943EA024323F0805357
:100E5000CA6913430268104D104CA24218BFAA423F
:100E600010D123F470038C6A43EA045323F0807397
:100E70000C6A234323F000734C6A234323F000538E
:100E8000C96A0B435364002380F83C30184630BCD9
:100E900070470220704700BF00000140000401407D
:100EA000704770477047026852E8003F23F0C00364
:100EB00042E800310029F6D1026802F1080353E844
:100EC000003F23F40003083242E800310029F3D147
:100ED0002023C0F888307047026852E8003F23F4AE
:100EE000907342E800310029F6D1026802F108034C
:100EF00053E8001F0D4B0B40083242E80031002937
:100F0000F3D1C36E012B06D02023C0F88C30002310
:100F1000C36643677047026852E8003F23F010033E
:100F200042E800310029F6D1EEE700BFFEFFFFEFF7
:100F3000D0F88830212B00D07047B0F856309BB2E3
:100F400093B9026852E8003F23F0800342E8003181
:100F50000029F6D1026852E8003F43F0400342E81E
:100F600000310029F6D17047036D1A7803689A6240
:100F7000036D01330365B0F856309BB2013B9BB261
:100F8000A0F85630D8E7D0F88830212B00D0704731
:100F9000B0F856309BB293B9026852E8003F23F094
:100FA000800342E800310029F6D1026852E8003F90
:100FB00043F0400342E800310029F6D17047036D49
:100FC0001B880268C3F308039362036D0233036551
:100FD000B0F856309BB2013B9BB2A0F85630D6E732
:100FE000D0F88830212B00D07047B0F86A3017E075
:100FF000026802F1080353E8003F23F400030832BB
:1010000042E800310029F3D1026852E8003F43F082
:10101000400342E800310029F6D17047013B9BB202
:10102000002BE1D0B0F8562092B2002AE0D002683E
:10103000D16911F0800FF1D0016D09789162026DD4
:1010400001320265B0F8562092B2013A92B2A0F88D
:101050005620E3E7D0F88830212B00D07047B0F855
:101060006A3017E0026802F1080353E8003F23F4F6
:101070000003083242E800310029F3D1026852E847
:10108000003F43F0400342E800310029F6D17047A9
:10109000013B9BB2002BE1D0B0F8562092B2002A5F
:1010A000E0D00268D16911F0800FF1D0016D09889C
:1010B000C1F308019162026D02320265B0F8562058
:1010C00092B2013A92B2A0F85620E1E7D0F8883007
:1010D000202B45D1B2FA82F35B09002908BF012316
:1010E000002B3FD10165A0F85420A0F85620C0F88D
:1010F00090302123C0F88830436EB3F1005F10D0E8
:101100008368B3F5805F25D0174B8367026852E888
:10111000003F43F0800342E800310029F6D100206F
:1011200070478368B3F5805F0ED0104B8367026809
:1011300002F1080353E8003F43F40003083242E899
:1011400000310029F3D1EAE70369002BEDD1084B08
:101150008367ECE70369002BD6D1064B8367D5E79D
:101160000220704701207047310F0108E10F01088C
:1011700055100108870F01081346D0F88820202A4F
:1011800040D110B50446B3FA83F25209002908BFD2
:101190000122002A38D10165A0F85430A0F8563059
:1011A000C0F890202122C0F88820C26FCAB1174928
:1011B000D163C26F16491164C26F1649D164C26F00
:1011C0000021116502682832016DC06FFAF7F8F846
:1011D00038B11023C4F890302023C4F8883001209F
:1011E0000FE0236840221A62226802F1080353E8E4
:1011F000003F43F08003083242E800310029F3D178
:10120000002010BD022070470120FAE71B120108E0
:101210008712010895120108704708B50346806BD4
:10122000DB69B3F5807F18D00023A0F85630026840
:1012300002F1080353E8003F23F08003083242E83C
:1012400000310029F3D1026852E8003F43F0400327
:1012500042E800310029F6D108BDFFF7DDFFFBE7CA
:1012600008B5026852E8003F23F0400342E800312D
:101270000029F6D12023C0F8883000238367FFF7C8
:10128000CBFF08BD704708B5806BFFF7FBFF08BDBB
:101290007047704738B5846BD4F88820D4F88C50E8
:1012A00023689B6813F0800F01D0212A10D0236897
:1012B0009B6813F0400F01D0222D10D0D4F890304D
:1012C00043F01003C4F89030204606F043F838BDD0
:1012D0000023A4F856302046FFF7E5FDE7E700239A
:1012E000A4F85E302046FFF7F7FDE7E708B5806B0E
:1012F0000023A0F85E30A0F8563006F02BF808BDA9
:1013000070B504460168CB6908688D6840F60F0225
:101310001A4008D113F0200F05D010F0200F34D15F
:1013200015F0805F31D12AB1B34A2A4033D1B34E90
:10133000304230D1E26E012A00F0C68013F4801FE3
:1013400003D015F4800F40F09B8113F0800F07D07D
:1013500010F0800F40F09B8115F4000F40F0978152
:1013600013F0400F03D010F0400F40F0978113F4BA
:10137000000F03D010F0804F40F0948113F0807F75
:1013800002D00028C0F2928170BD636F002BFBD0A9
:1013900020469847F8E713F0010F09D010F4807F3A
:1013A00006D001260E62D4F890103143C4F8901094
:1013B00013F0020F0BD015F0010F08D021680226A0
:1013C0000E62D4F8901041F00401C4F8901013F0AC
:1013D000040F0BD015F0010F08D0216804260E620F
:1013E000D4F8901041F00201C4F8901013F0080FE7
:1013F0000BD010F0200F00D13AB122680821116201
:10140000D4F890200A43C4F8902013F4006F0CD055
:1014100010F0806F09D022684FF400611162D4F897
:10142000902042F02002C4F89020D4F89020002AA6
:10143000AAD013F0200F09D010F0200F02D115F020
:10144000805F03D0636F0BB120469847D4F890209B
:1014500023689B6813F0400F02D112F0280F2CD0A4
:101460002046FFF739FD23689B6813F0400F20D01A
:10147000226802F1080353E8003F23F040030832DA
:1014800042E800310029F3D1D4F880306BB15C4AD6
:101490001A65D4F88000FAF77FFA00283FF474AF99
:1014A000D4F88000036D98476EE7204605F052FFA0
:1014B0006AE7204605F04EFF66E7204605F04AFF42
:1014C0000023C4F890305FE713F0100F3FF436AFFD
:1014D00010F0100F3FF432AF10230B6223689B68AB
:1014E00013F0400F00F09280D4F880201368454834
:1014F00045498B4218BF83422DD018318B422AD0E8
:1015000018318B4227D018318B4224D018318B42AE
:1015100021D018318B421ED018318B421BD001F5DF
:1015200056718B4217D018318B4214D018318B4230
:1015300011D018318B420ED018318B420BD018319C
:101540008B4208D018318B4205D018318B4202D023
:101550005B689BB201E05B689BB2002B3FF414AF69
:10156000B4F85C1099427FF60FAFA4F85E30D369EF
:10157000B3F5807F32D0226852E8003F23F48073B5
:1015800042E800310029F6D1226802F1080353E84D
:10159000003F23F00103083242E800310029F3D173
:1015A000226802F1080353E8003F23F040030832A9
:1015B00042E800310029F3D12023C4F88C30002305
:1015C000E366226852E8003F23F0100342E800314E
:1015D0000029F6D1D4F88000FAF73EF802232367F9
:1015E000B4F85C10B4F85E309BB2C91A89B22046D8
:1015F00005F040FEC8E600BF010000102001000415
:10160000ED1201081000024028000240B4F85C10FE
:10161000B4F85E309BB2C91A89B2B4F85E309BB29E
:10162000002B3FF4B1AE00293FF4AEAE226852E881
:10163000003F23F4907342E800300028F6D122687E
:1016400002F1080353E8000F1A4B0340083242E846
:1016500000300028F3D12023C4F88C300023E36647
:101660006367226852E8003F23F0100342E800302D
:101670000028F6D102232367204605F0FBFD83E610
:101680004FF480130B62204600F04EFE7CE6A36F01
:10169000002B3FF479AE2046984775E62046FFF7C9
:1016A000DFFD71E6204600F041FE6DE6204600F0C9
:1016B0003CFE69E6FEFFFFEF08B5806B0123036780
:1016C000C36E012B02D0FFF7E4FD08BDB0F85C103B
:1016D000490805F0CFFDF8E708B50346806BDB69E4
:1016E000B3F5807F29D00023A0F85E30026852E86D
:1016F000003F23F4807342E800310029F6D10268EC
:1017000002F1080353E8003F23F00103083242E8E6
:1017100000310029F3D1026802F1080353E8003FC9
:1017200023F04003083242E800310029F3D120239E
:10173000C0F88C30C36E012B07D000230367C36E43
:10174000012B0CD0FFF7A4FD08BD026852E8003F52
:1017500023F0100342E800310029F6D1EDE7B0F89C
:101760005C1005F087FDEFE72DE9F04186B00446F7
:10177000016883680269134342691343C2691343D2
:101780000868914A024013430B602268536823F4AF
:101790004053E1680B435360A16922688B4B9A4226
:1017A00001D0236A19439068894B03400B4393602F
:1017B0002268D36A23F00F03616A0B43D362226865
:1017C000844B9A4229D0844B9A4200F09480834BF8
:1017D0009A4200F0AA80824B9A4200F0C080814B6E
:1017E0009A4200F0D680804B9A4200F009817F4BEC
:1017F0009A4200F02E817E4B9A4200F041817D4B4F
:101800009A4200F054817C4B9A4200F079816F4BF0
:101810009A4200F09E81802333E0784B5B6D03F0A9
:101820003803282B65D8DFE813F029006400640032
:1018300064006400640064006400AC01640064003F
:10184000640064006400640064002B0064006400B1
:10185000640064006400640064005E00640064006E
:10186000640064006400640064006000640064005C
:10187000640064006400640064006200012300E00E
:10188000082352498A4200F09581E069B0F5004F83
:1018900000F00D82202B00F26682202B00F2BA822B
:1018A000DFE813F087028D02B802B8029002B80296
:1018B000B802B8029502B802B802B802B802B8027B
:1018C000B802B8029A02B802B802B802B802B80266
:1018D000B802B802B802B802B802B802B802B80238
:1018E000B802B802A6021023CBE72023C9E74023A1
:1018F000C7E78023C5E7414B5B6D03F00703052B6A
:1019000011D8DFE813F00600400108000A000C00BF
:101910000E000023B5E70823B3E71023B1E7202327
:10192000AFE74023ADE78023ABE7344B5B6D03F0BB
:101930000703052B11D8DFE813F006002801080083
:101940000A000C000E0000239BE7082399E71023F0
:1019500097E7202395E7402393E7802391E7274BE0
:101960005B6D03F00703052B11D8DFE813F00600C9
:10197000100108000A000C000E00002381E7082374
:101980007FE710237DE720237BE7402379E780234F
:1019900077E71A4B5B6D03F00703052B11D8DFE8DF
:1019A00013F00600F80008000A000C000E000023E7
:1019B00067E7082365E7102363E7202361E74023F7
:1019C0005FE780235DE700BFF369FFCF000C00589D
:1019D000FFF4FF11001001400044004000480040A7
:1019E000004C0040005000400014014000780040CE
:1019F000007C004000180140001C014000440258D7
:101A0000694B5B6D03F03803282B20D8DFE803F027
:101A1000151F1F1F1F1F1F1FC31F1F1F1F1F1F1F3C
:101A2000171F1F1F1F1F1F1F191F1F1F1F1F1F1FD4
:101A30001B1F1F1F1F1F1F1F1D00012321E708233E
:101A40001FE710231DE720231BE7402319E780230E
:101A500017E7554B5B6D03F00703052B0ED8DFE846
:101A600003F0039C0507090B00230AE7082308E796
:101A7000102306E7202304E7402302E7802300E742
:101A8000494B5B6D03F00703052B0ED8DFE803F02D
:101A900003870507090B0023F3E60823F1E610236B
:101AA000EFE62023EDE64023EBE68023E9E63E4B1C
:101AB0005B6D03F03803282B20D8DFE803F0151FF7
:101AC0001F1F1F1F1F1F721F1F1F1F1F1F1F171FDB
:101AD0001F1F1F1F1F1F191F1F1F1F1F1F1F1B1F20
:101AE0001F1F1F1F1F1F1D000123CAE60823C8E672
:101AF0001023C6E62023C4E64023C2E68023C0E6C6
:101B0000294B5B6D03F03803282B20D8DFE803F066
:101B1000151F1F1F1F1F1F1F4E1F1F1F1F1F1F1FB0
:101B2000171F1F1F1F1F1F1F191F1F1F1F1F1F1FD3
:101B30001B1F1F1F1F1F1F1F1D000123A1E60823BE
:101B40009FE610239DE620239BE6402399E6802311
:101B500097E603F50E339B6D03F00703052B0ED8B4
:101B6000DFE803F003260507090B022389E60823B3
:101B700087E6102385E6202383E6402381E6802341
:101B80007FE604237DE604237BE6042379E6042331
:101B900077E6042375E6042373E6042371E6042341
:101BA0006FE604236DE600BF00440258042368E694
:101BB000042366E6202B27D8022BC0F01D81023BB0
:101BC0001E2B00F21B81DFE813F0520019015800B0
:101BD0001901190119015D001901190119011901F2
:101BE00019011901190162001901190119011901DD
:101BF0001901190119011901190119011901190115
:101C00001901190119016E00402B2ED14FF400402B
:101C1000626A824B33F81220B0FBF2F3656805EB81
:101C20004501994200F2EC80B3EB053F00F2EA80F7
